:100000000C946D080C948C080C948C080C940C0BBC
:100010000C94420B0C948C080C948C080C948C0857
:100020000C948C080C948C080C948C080C948C0800
:100030000C948C080C948C080C948C080C94E30E93
:100040000C948C080C948C080C948C080C948C08E0
:100050000C94BD590C94C9500C948C080C948C08C9
:100060000C948C080C949F510C948C080C94935114
:100070000C948C080C948C080C948C080C948C08B0
:100080000C9480650C948C080C948C080C948C084F
:100090000C94DD510C948C080C94D1510C948C0868
:1000A0000C948C080C948C080C948C080C948C0880
:1000B0000C948C080C948C080C948C080C948C0870
:1000C0000C948C080C948C080C948C080C948C0860
:1000D0000C948C080C948C080C948C080C948C0850
:1000E0000C948C080C9476590C9480590C946C598F
:1000F0000C9426590C94B1590C94A2590C9496590D
:100100000C948A590C948C080C948C080C948C08D0
:100110000C948C080C948C080C948C080C948C080F
:10012000084AD73B3BCE016E84BCBFFDC12F3D6C5E
:1001300074319ABD56833DDA3D00C77F11BED9E4C4
:10014000BB4C3E916BAAAABE000000803F076342F1
:1001500036B79BD8A71A39685618AEBAAB558C1D5E
:100160003CB7CC5763BD6DEDFD753EF6177231BFE0
:10017000000000803F08000000BE922449123EAB00
:10018000AAAA2ABECDCCCC4C3E00000080BEABAAB1
:10019000AAAA3E00000000BF000000803F0000004F
:1001A0000000084178D3BB4387D1133D190E3CC3EF
:1001B000BD4282AD2B3E68EC8276BED98FE1A93E6E
:1001C0004C80EFFFBE01C4FF7F3F000000000050E5
:1001D0003A20256C642050612020252D372E326670
:1001E000206D0A002563002563004932433A200050
:1001F000256300256C642050612020252D372E3288
:1002000066206D00256C6420432000256300545F48
:1002100052483D252D342E3166200052483D252D73
:10022000342E3166200025630025630025630025F8
:10023000630043757272656E74207265706F7274BC
:1002400020696E74657276616C3D252D642073653E
:10025000630A004E6577207265706F727420696E54
:1002600074657276616C3D252D64207365630A00A8
:100270002563005573696E67207265706F72743DF7
:100280003078252D6C7820004E6577207265706F70
:1002900072743D3078252D6C78200025630025632D
:1002A00000256300256300204F534343414C3D2507
:1002B00064200020467573653A2065653D2530321F
:1002C000782068663D25303278206C663D253032D6
:1002D00078206C623D25303278004D43553D253005
:1002E000366C7800256300252D31306C7520252D66
:1002F00031306C7520252D31306C7520252D313035
:100300006C75200A007478206C656E2020202020F7
:100310007268206D697373202020207268207374C6
:10032000616C652020207268206D6973630A002566
:1003300063004F4B0A0025630025630025630025F9
:10034000630025630052454C41593D090930782529
:10035000780A00434F4D504153533D09307825787A
:100360000A00414343454C3D0909307825780A008D
:10037000505245533D0909307825780A00505F50A6
:1003800057523D0909307825780A004145533D0907
:1003900009307825780A0050315F4C45443D090901
:1003A000307825780A0050305F4C45443D090930CB
:1003B0007825780A004556454E543D090930782580
:1003C000780A004C45443D0909307825780A004FE9
:1003D000573D0909307825780A00504B543D0909EA
:1003E000307825780A0054583D0909307825780A74
:1003F0000052583D0909307825780A004F5045527F
:100400003D0909307825780A0043757272656E746B
:100410002064656275673D307825580A004E65771F
:100420002064656275673D307825580A0025730A97
:100430000025372E33662025372E33660025352ECE
:10044000326620004572726F72203020566F6C74D5
:10045000004E6F7420737570706F727465640A005B
:100460004572726F72203020566F6C740045727244
:100470006F72203020566F6C740025730A0073650C
:100480006E743D252D75207375707072657373657C
:10049000643D252D750A00545820506F7765723DD4
:1004A00025640A004368616E3D25640A0054657343
:1004B0007420362025730A00546573742035202576
:1004C000730A005465737420342025730A00546540
:1004D000737420332025730A00546573742032200E
:1004E00025730A005465737420312025730A002592
:1004F000730A0025730A00646565700A00666F72EE
:1005000063655F69646C650A006E6F6E650A0070F2
:100510007772733D005854414C5F5452494D3D250C
:10052000640025730A00696E74725F7365635F709F
:10053000313D252D372E33660A00696E74725F7067
:10054000313D252D6C640A00696E74725F736563BA
:100550005F70303D252D372E33660A00696E747248
:100560005F70303D252D6C640A00765F6D63753DCC
:10057000252D352E32660A00707077723D25730A7C
:100580000064656275673D3078252D780A00257313
:100590000A006175746F0A006C6F675F6D6F646548
:1005A0003D007573625F7077723D25730A00726556
:1005B000706F72745F6D61736B3D3078252D6C7850
:1005C00020007265706F72745F696E746572766117
:1005D0006C3D252D640A0072656C61793D25730AB6
:1005E0000052494D455F616464723D252D642E259E
:1005F0002D640A006E65696768626F725F7461627C
:100600006C655F73697A653D25640A0074785F7074
:100610006F7765723D25640A006368616E3D2564ED
:100620000A006932633D0069643D00537973746563
:100630006D2053756D6D6172790A0050413D090955
:100640003078256C7800503D09093078256C7800A9
:1006500041333D0909307825780041323D090930A0
:100660007825780041313D09093078257800565FBA
:10067000494E3D0909307825780052483D09093036
:1006800078257800555054494D453D090930782565
:10069000780050315F543D09093078257800503199
:1006A0003D0909307825780050305F543D09093004
:1006B0007825780050303D09093078257800565F5C
:1006C0004D43553D09093078257800545F4D435519
:1006D0003D0909307825780054313D0909307825E5
:1006E0007800543D090930782578004536343D09B5
:1006F00009307825780049443D090930782578008B
:100700005041200050200041332000413220004160
:10071000312000565F494E20005248200055505469
:10072000494D45200050315F542000503120005089
:10073000305F54200050302000565F4D435520005C
:10074000545F4D435520005431200054200045365D
:10075000342000494420002530327800765F6C69EF
:100760006768743D252D372E3366002000765F6163
:10077000323D252D372E3366002000765F61313DF6
:10078000252D372E3366002000765F696E3D252DBE
:10079000352E326600204E657665722D7573656460
:1007A00020737461636B203E202564206279746538
:1007B000730A00757074696D653D252D642D646143
:1007C00079732D253032643A253032643A2530323F
:1007D000642D686F7572730A0074657374205B6FA3
:1007E00066667C317C327C337C347C355D20202015
:1007F00020202020202D2074657374206D6F646587
:10080000730A0D00776474205B6F6E7C6F66667C84
:10081000746573745D20202020202020202020205B
:100820002D207761746368646F670A0D00757067C7
:100830007220202020202020202020202020202066
:100840002020202020202020202D207265626F6F24
:10085000742076696120626F6F746C6F6164657279
:100860000A0D00626F6F742020202020202020209D
:100870002020202020202020202020202020202D6B
:10088000207265626F6F740A0D0070777273205B5F
:10089000646565707C666F7263655F69646C657CB6
:1008A0006E6F6E655D202D206D637520736C6565C0
:1008B00070206D6F64650A0D007265737420656544
:1008C00070726F6D202020202020202020202020EA
:1008D00020202020202D20726573746F72652065A2
:1008E0006570726F6D0A0D0070707772205B6F6EAD
:1008F0007C6F66665D202020202020202020202084
:10090000202020202D2070726F6772616D6D6162F2
:100910006C65207077720A0D0074787077205B31F7
:10092000352D305D20202020202020202020202058
:1009300020202020202D205458205077722E20482F
:10094000696768657374203020283364426D290A12
:100950000D00737320202020202020202020202024
:1009600020202020202020202020202020202D207A
:1009700073797374656D2073756D6D6172790A0D8D
:1009800000727320202020202020202020202020E2
:10099000202020202020202020202020202D2072F8
:1009A0006164696F2073746174730A0D0072692049
:1009B0005B696E745D2020202020202020202020D4
:1009C0002020202020202020202D207265706F7292
:1009D0007420696E74657276616C0A0D0072652010
:1009E0005B6D61736B5D2020202020202020202063
:1009F0002020202020202020202D206D6F746520B5
:100A00007265706F72742073657474696E670A0D15
:100A1000006F772020202020202020202020202050
:100A2000202020202020202020202020202D206F6A
:100A30006E652D776972652073656E736F72730AC8
:100A40000D006C6F67205B6175746F7C6F6E7C6FDF
:100A500066665D20202020202020202020202D20C0
:100A60006D6F7465732064617461206F6E205553DF
:100A7000420A0D006E65205B666C7573685D202010
:100A80002020202020202020202020202020202066
:100A90002D206E65696768626F72207461626C6593
:100AA0000A0D0065727220202020202020202020A6
:100AB0002020202020202020202020202020202D29
:100AC000206572726F7220696E666F0A0D006D6329
:100AD00075202020202020202020202020202020C1
:100AE000202020202020202020202D206D63752014
:100AF000696E666F0A0D006964205B7265736574C8
:100B00005D202020202020202020202020202020A8
:100B10002020202D2069642068616E646C696E67F6
:100B20000A0D0068756D2020202020202020202024
:100B30002020202020202020202020202020202DA8
:100B40002068756D69646974792073656E736F725E
:100B50000A0D0072656C6179205B6F6E7C6F666652
:100B60007C73746174735D20202020202020202D50
:100B70002072656C6179206E6574776F726B20727C
:100B800065706F7274730A0D006465205B6D61732C
:100B90006B5D2020202020202020202020202020CD
:100BA00020202020202D2064656275670A0D0063D7
:100BB00068616E205B31312D32365D20202020208F
:100BC00020202020202020202020202D204368616C
:100BD0006E2031312D32362028322E3430352D32F0
:100BE000343830204D687A290A0D0063616C692021
:100BF0005B5B765F696E7C61317C61325D20766F14
:100C00006C747C72657365747C6E6F6E655D202D8F
:100C10002063616C6962726174650A0D00616463CE
:100C200020202020202020202020202020202020C4
:100C30002020202020202020202D2073686F772066
:100C4000765F696E2C2061312C20613220766F6CCA
:100C500074616765730A0D00752020202020202014
:100C60002020202020202020202020202020202084
:100C7000202020202D20757074696D650A0D007686
:100C80002020202020202020202020202020202064
:100C900020202020202020202020202D207665725A
:100CA00073696F6E0A0D006820202020202020200C
:100CB0002020202020202020202020202020202034
:100CC0002020202D2068656C700A0D0025630075BA
:100CD0006E6B6E6F776E20636D640A004E484443FE
:100CE000303231365F0058582D4D43503334323452
:100CF0005F004C334734323030445F00484D433559
:100D00003838335F004144584C3334355F00424D2E
:100D1000503038355F00484948363133305F004144
:100D20005432344D41435F00202573002025362E78
:100D300032662000253032780074656D705F65780A
:100D40007465726E3D252D362E32660020257300A7
:100D50002025362E3266204F6E2D426F6172640060
:100D6000253032780074656D705F626F6172643D2A
:100D7000252D362E3266000A00452025642E256476
:100D800020636C6F636B20256C7520637075202564
:100D90006C75206C706D20256C7520697271202532
:100DA0006C7520676C656420256C7520796C6564B2
:100DB00020256C7520726C656420256C7520747814
:100DC00020256C75206C697374656E20256C752008
:100DD00073656E736F727320256C7520736572690D
:100DE000616C20256C750A00532025642E25642033
:100DF000636C6F636B20256C7520747820256C758F
:100E000020727820256C752072747820256C7520EE
:100E100072727820256C75207265786D6974202552
:100E20006C752061636B747820256C75206E6F6122
:100E3000636B747820256C752061636B7278202554
:100E40006C752074696D65646F757420256C7520F0
:100E500062616461636B727820256C7520746F6FBA
:100E60006C6F6E6720256C7520746F6F73686F727E
:100E70007420256C752062616473796E6368202527
:100E80006C752062616463726320256C7520636FEA
:100E90006E74656E74696F6E64726F7020256C7508
:100EA0002073656E64696E6764726F7020256C755F
:100EB000206C6C747820256C75206C6C7278202501
:100EC0006C750A00257325730A004F6E6C696E6598
:100ED0000A000A002C20636865636B2072617465E8
:100EE00020257520487A0025732025732C206368FF
:100EF000616E6E656C20257520706F776572202598
:100F000075000A0025783A004D41432061646472FF
:100F1000657373200052616E646F6D2045554936CC
:100F20003420616464726573732067656E657261F5
:100F30007465640A000A2A2A2A2A2A2A2A426F6F1A
:100F400074696E672025732A2A2A2A2A2A2A0A0007
:100F5000020000FFFE00000141544D45474131327F
:100F60003872666131006C6F63616C686F73740016
:100F7000454550524F4D20697320636F72727570F2
:100F8000742C20726577726974696E672077697452
:100F9000682064656661756C74732E0A006E616EFC
:100FA00000696E660000407A10F35A00A0724E1875
:100FB000090010A5D4E80000E87648170000E40B0B
:100FC00054020000CA9A3B000000E1F505000080D1
:100FD000969800000040420F000000A0860100002B
:100FE00000102700000000E803000000006400007B
:100FF0000000000A00000000000100000000002CBA
:1010000076D888DC674F0823DFC1DFAE59E1B1B77E
:1010100096E5E3E453C63AE651997696E8E6C2844B
:1010200026EB898C9B62ED407C6FFCEFBC9C9F4063
:10103000F2BAA56FA5F490055A2AF75C936B6CF988
:10104000676DC11BFCE0E40D47FEF520E6B500D05E
:10105000ED902E0300943577050080841E08000073
:10106000204E0A000000C80C333333330F986E1241
:10107000831141EF8D2114893BE65516CFFEE6DB47
:1010800018D1844B381BF77C1D901DA4BBE4242091
:101090003284725E228100C9F124ECA1E53D27492A
:1010A0004E46494E4954594E414ECDCCCC3D0AD7BF
:1010B000233C17B7D13877CC2B329595E6241FB156
:1010C0004F0A000020410000C84200401C4620BCDE
:1010D000BE4CCA1B0E5AAEC59D7411241FBECFEF65
:1010E000D1E4DEBFCDBF16E0A0E0B2E0E8E2F2E07E
:1010F00001E00BBF02C007900D92A83CB107D9F7E1
:101100001DE2A8ECB6E001C01D92A639B107E1F7D7
:101110000E94834F0C9412810C94000029E0FC0182
:1011200020935700C895802D089500D08FE095E05A
:10113000EDB7FEB7928381830E94037E8091B20453
:101140009091B3040F900F9093FF04C000D089E0FA
:1011500095E009C092FF04C000D08DEF94E003C079
:1011600000D087EF94E0EDB7FEB7928381830E94B1
:10117000037E0F900F900895E091BB17F0E0EF71A0
:10118000F070E05FF74E80838091BB178F5F809394
:10119000BB178091D02488608093D02449ED54E01F
:1011A000CA0161E10E94CB4080E090E00895EF9297
:1011B000FF92CF93DF93E82EE7017E01F92EE7013E
:1011C0008091C8069091C90686FF2FC08DB79EB743
:1011D0000C970FB6F8949EBF0FBE8DBFEDB7FEB74C
:1011E000319680E092E0ADB7BEB712969C938E9395
:1011F00011978A81828313828B81848315828885EB
:10120000868317828C819D81918780878E819F81C3
:10121000938782870E94F17D2DB73EB7245F3F4FB1
:101220000FB6F8943EBF0FBE2DBF8DEE96E0BE0107
:101230000E94104282E495E0BE010E947C41DF9151
:10124000CF91FF90EF9008953F924F925F926F92EF
:101250007F928F929F92AF92BF92CF92DF92EF9246
:10126000FF920F931F93DF93CF93CDB7DEB76097B5
:101270000FB6F894DEBF0FBECDBF3B010E94A8554C
:10128000E82FF0E0EE0FFF1FEB57F84E80819181C1
:101290000196918380838091C8069091C90681FD53
:1012A00074980E9493474C018DEE96E00E94C241D3
:1012B00024C0C8010296B3010E94983E0097D1F065
:1012C000C8010D9660E074E647ED58E098010E9471
:1012D0008744D4019C91F80180859817A1F58091ED
:1012E000991790919A17019690939A17809399174E
:1012F00033242BC0C8010E948842082F192F0115E2
:101300001105B9F63EC1C8010296B3010E948F3E95
:10131000D4018C918150F801808780E091E0A0E0B9
:10132000B0E081879287A387B4878DEE96E0B801FD
:101330000E944942C8010D9660E074E647ED58E00E
:1013400098010E9487443324339484E00E94C74864
:10135000D80115969C938E93149783E00E94C748FA
:101360002C01F80197838683D401AC908085A81A5C
:10137000BB24CC24DD2486E0AA0CBB1CCC1CDD1CC9
:101380008A95D1F7618572858385948520EC30E05C
:1013900040E050E00E943A7A672F782F892F9927F2
:1013A000A60EB71EC81ED91EF801A186B286C38636
:1013B000D486D4018C9180878091C8069091C9060B
:1013C00081FD08C08091B20480FD04C081FFD1C0BE
:1013D0001D9BCFC0EDB7FEB772970FB6F894FEBF56
:1013E0000FBEEDBFEDB6FEB60894E11CF11C8FE216
:1013F00092E092838183C4010196D70113969C9356
:101400008E931297F301808114968C9314971596FE
:101410001C921597818116968C93169717961C929D
:10142000D4018C91F70180871186D80114968D9193
:101430009C9115979387828755864486BB27AD2D4F
:101440009C2D8B2D97878687C601B50124E630E059
:1014500040E050E00E943A7A672F782F892F992731
:101460000E94807AF701718B608B0E94F17D209140
:1014700095048DB79EB742960FB6F8949EBF0FBEE7
:101480008DBF2223A9F000D000D0EDB7FEB7319672
:1014900087EE91E0ADB7BEB712969C938E931197ED
:1014A000228313820E94037E0F900F900F900F9063
:1014B0008091B2049091B30496FF15C0332099F047
:1014C00089ED96E00E942F3F809197179091981791
:1014D000019690939817809397178091C8069091E2
:1014E000C90696FD73988091591C86FF42C00E94E0
:1014F000794DC40104960E94384DEDB7FEB73C9774
:101500000FB6F894FEBF0FBEEDBF31967E01089472
:10151000E11CF11CADB7BEB71296FC92EE9211978A
:1015200080E190E0938382838BE692E095838483CD
:10153000D80114968D919C91159797838683169662
:101540008D919C91179791878087D4018C91828788
:1015500013860E945A7EEDB7FEB73C960FB6F894FC
:10156000FEBF0FBEEDBF82E00E94554DC7010E9435
:10157000384D8091C8069091C90681FF0DC0749ABC
:101580000BC082E495E00E945641082F192F0115E7
:10159000110509F0B8CEEDCF60960FB6F894DEBF16
:1015A0000FBECDBFCF91DF911F910F91FF90EF90B4
:1015B000DF90CF90BF90AF909F908F907F906F9073
:1015C0005F904F903F90089587EE93E081159105CD
:1015D00011F00197F1F708958823B9F052985A98BD
:1015E0001DBA80916900806280936900EA9A5398DD
:1015F0005B98EB9A80916900806880936900809184
:1016000068008160809368000895109269005A9A7A
:10161000EA985B9AEB9808951F920F920FB60F927B
:1016200011248F939F93AF93BF938091680080FFA5
:1016300020C08091B0249091B124A091B224B091A7
:10164000B3240196A11DB11D8093B0249093B124C1
:10165000A093B224B093B3248091C8069091C90698
:1016600087FF07C0749882E090E09093880480938D
:101670008704BF91AF919F918F910F900FBE0F90F4
:101680001F9018951F920F920FB60F9211248F93EF
:101690009F93AF93BF938091680080FF20C080919B
:1016A000B4249091B524A091B624B091B7240196AA
:1016B000A11DB11D8093B4249093B524A093B624AA
:1016C000B093B7248091C8069091C90690FF07C0D7
:1016D000739882E090E09093880480938704BF9190
:1016E000AF919F918F910F900FBE0F901F90189503
:1016F00080937C0080917B00877F80937B0080912A
:101700007C00806C80937C0085E080937A008091DF
:101710007A00806880937A0080917B0087FFFCCFFD
:1017200080917B0085FFFCCF80917A00806480935C
:101730007A0080917A0086FDFCCF10927900109299
:10174000780084E090E060E070E020917A0020640E
:1017500020937A0020917A0026FDFCCF209178001A
:1017600030917900620F731F019779F710927C0016
:1017700080917A008F7780937A0076956795769539
:10178000679580E090E00E94BD77089580E00E9418
:10179000780B2091890430918A0440918B045091F8
:1017A0008C040E949B7821EE3AE744E95EE30E94B4
:1017B0008B76089580E1809351018093510190913F
:1017C000510195FF03C08F5F8F31B9F76BE4869F9E
:1017D000B0011124882777FD8095982F0E94BF774C
:1017E00020E030E64FE954E40E948B7620E030E0C0
:1017F0004AE754E40E94557708958091AC0484FF31
:101800004BC080917B00886080937B0089EC809343
:101810007C0085E080937A0080917A0080688093D4
:101820007A0080917B0087FFFCCF80917B0085FF51
:10183000FCCF80917A00806480937A0080917A0056
:1018400086FDFCCF80917A00806480937A0080913D
:101850007A0086FDFCCF609178007091790080E07D
:1018600090E00E94BD7727ED33EA40E95FE30E94F4
:101870009B7826E636E648E853E40E948A76609331
:101880008C1770938D1780938E1790938F1780917C
:101890007A008F7780937A0008956F927F928F926B
:1018A0009F92AF92BF92CF92DF92EF92FF920F93EF
:1018B0001F93DF93CF93CDB7DEB72A970FB6F89477
:1018C000DEBF0FBECDBF3C011092D0068FEF8983E3
:1018D0006CECC62E67E1D62E00E010E052E0E52E5B
:1018E000F12CEC0EFD1E4E010894811C911C4AE067
:1018F000A42EB12CAC0EBD1E3FC00830110509F45A
:1019000041C0C401B7012A870E94854A89812A857E
:101910008F3F11F08E3F19F48093D00634C06114CC
:10192000710479F4C7010E949F4A8093CD24F70186
:10193000A5ECB4E281918D93EA15FB05D9F721E07E
:1019400022C0C7010E949F4AF6018083D701F80197
:1019500033E0EE0FFF1F3A95E1F7E00FF11FEC5374
:10196000F84E8D918193AA15BB05D9F70F5F1F4FD4
:1019700089E090E0C80ED91E202F8981882309F0C4
:10198000BCCF01C028E0822F2A960FB6F894DEBFA4
:101990000FBECDBFCF91DF911F910F91FF90EF90C0
:1019A000DF90CF90BF90AF909F908F907F906F907F
:1019B000089500D087E79DE0EDB7FEB7928381835D
:1019C0000E94037E0F900F9008952F923F924F92A6
:1019D0005F926F927F928F929F92AF92BF92CF92BF
:1019E000DF92EF92FF920F931F93DF93CF9300D07C
:1019F00000D0CDB7DEB78C014B01009741F489E2EE
:101A000090E06BE270E04AE250E027E00AC08130EB
:101A1000910549F489E290E06BE270E04AE250E01F
:101A200026E00E946149C8010E944D0CF801E25372
:101A3000F94F80830115110581F0BCECCB2EB7E185
:101A4000DB2E00E010E03F01A4E34A2EADE05A2E69
:101A5000FCE22F2EFDE03F2E44C185EC94E20E9473
:101A6000D14B9C01B901882777FD8095982F0E9462
:101A7000BF77C82EE92E81149104A1F000D000D0C8
:101A800000D00DB71EB70F5F1F4F85E69DE0ADB7C5
:101A9000BEB712969C938E931197562F472F3C2DCD
:101AA0002E2D97C0E5ECAE2EE4E2BE2E00E61DE042
:101AB000D5018D915D0100D000D0EDB7FEB7319614
:101AC000ADB7BEB712961C930E9311978283138203
:101AD0006B837C830E94037E0F900F900F900F907A
:101AE0006B817C81BDECAB16B4E2BB0609F700D07C
:101AF00000D000D00DB71EB70F5F1F4F80E59DE0EF
:101B0000EDB7FEB7928381838C2D9E2D20E030E0CF
:101B100048EC52E40E945577D80112966D937D935C
:101B20008D939C9315970E94037EEDB7FEB7369672
:101B30000FB6F894FEBF0FBEEDBF8091CD24882371
:101B400019F08EE792E002C087E892E000D000D062
:101B50002CE43DE0ADB7BEB712963C932E9311979F
:101B600014969C938E9313970E94037E0F900F9070
:101B70000F900F9048C0780173E0EE0CFF1C7A952F
:101B8000E1F7E00EF11EE4ECF7E1EE0EFF1EC701F7
:101B90000E94D14B9C01B901882777FD8095982F31
:101BA0000E94BF775C018114910481F100D000D0C4
:101BB00000D00DB71EB70F5F1F4F89E39DE0ADB793
:101BC000BEB712969C938E931197562F472F3A2D9E
:101BD0002B2D652F742F832F922F20E030E048ECBF
:101BE00052E40E945577F80162837383848395835E
:101BF0000E94037E2DB73EB72A5F3F4F0FB6F89481
:101C00003EBF0FBE2DBF0E94D90C72C020E030E055
:101C1000D7018D917D0100D000D0EDB7FEB7319690
:101C2000ADB7BEB712965C924E9211978283138223
:101C300029833A836B837C830E94037E29813A81C6
:101C40002F5F3F4F0F900F900F900F906B817C8113
:101C500028303105E9F600D000D000D0EDB6FEB650
:101C60000894E11CF11CEDB7FEB7328221828A2D67
:101C70009B2D20E030E048EC52E40E945577D701DC
:101C800012966D937D938D939C9315970E94037E7E
:101C9000EDB7FEB736960FB6F894FEBF0FBEEDBF98
:101CA000D6018C91882319F08EE792E002C087E874
:101CB00092E000D000D028E23DE0EDB7FEB73283DD
:101CC0002183948383830E94037E0F900F900F9053
:101CD0000F900E94D90C0F5F1F4F89E090E0C80E53
:101CE000D91ED3018C9190E0081719070CF443CF4B
:101CF0000F900F900F900F90CF91DF911F910F9148
:101D0000FF90EF90DF90CF90BF90AF909F908F901B
:101D10007F906F905F904F903F902F900895DF934A
:101D2000CF9300D0CDB7DEB78091C6248983809150
:101D3000CC248A83CE0101960E94AA3E0F900F9078
:101D4000CF91DF910895CF93DF93EC018091C5246B
:101D50008F3FB1F58091C6248F3F91F58091C724C4
:101D60008F3F71F58091C8248F3F51F58091C92430
:101D70008F3F31F58091CA248F3F11F58091CB249C
:101D80008F3FF1F48091CC248F3FD1F489E290E031
:101D90006BE270E04AE250E027E00E94614980E097
:101DA00090E00E944D0CC253D94F888385EC94E299
:101DB00068E170E049E050E00E944C7F0E948F0E85
:101DC000DF91CF9108951F920F920FB60F920BB62D
:101DD0000F9211241F932F933F934F935F936F9311
:101DE0007F938F939F93AF93BF93EF93FF938091D4
:101DF000D02482608093D0248091B20486FD2B9AF7
:101E00008091B20487FD2B9A809187049091880479
:101E10001816190614F4749A739A8091C806909152
:101E2000C90685FF02C07498739880914A05909105
:101E30004B05019790934B0580934A05009709F055
:101E40007EC08091FC069091FD0601969093FD0660
:101E50008093FC0620915B2030915C2040915D20B6
:101E600050915E202F5F3F4F4F4F5F4F20935B207D
:101E700030935C2040935D2050935E2020E130E061
:101E800030934B0520934A052091B20420FD02C0F7
:101E90001D9B05C01092CC061092CB0606C021E017
:101EA00030E03093CC062093CB066091B004709163
:101EB000B1046115710599F001960E94597A009755
:101EC00071F477988091C8069091C90692FF07C077
:101ED000749884E090E090938804809387046091E4
:101EE000B0047091B1046115710579F08091FC0620
:101EF0009091FD060E94597A009739F485EF94E09D
:101F000062E140E050E00E94CB408091B20486FD47
:101F10002B988091B2049091B30491FF10C00E945D
:101F2000A8558A3119F0182F1F5F01C01BE00E94CD
:101F3000EC53812F90E00E94C0550E948A5484E6A1
:101F400095E060E040E050E00E94CB40FF91EF91CF
:101F5000BF91AF919F918F917F916F915F914F91C1
:101F60003F912F911F910F900BBE0F900FBE0F90BE
:101F70001F9018958091BB1790916F20891B089531
:101F80000E94BA0F882379F0E0916F20F0E0EF71A2
:101F9000F070E05FF74E208130E080916F208F5F1E
:101FA00080936F2002C02FEF3FEFC9010895CF93B8
:101FB000DF93EC011092F0061092EF068881998170
:101FC000009731F022E08B3E920709F0B9C009C0BA
:101FD0000E94BA0F882341F48BEE92E099838883A4
:101FE000B3C0613109F0B0C0F89478940E94C00F7A
:101FF00090E09093F4068093F3068D3009F47CC052
:102000008F3F31F38231910569F18F37910521F0CE
:102010008830910509F053C08091F7069091F80639
:10202000181619060CF060C06091902D7091912DDA
:1020300088E090E00E94C57D6091902D7091912D77
:1020400080E290E00E94C57D6091902D7091912D6D
:1020500088E090E00E94C57D8091F7069091F80697
:1020600001973EC06091902D7091912D8DE090E090
:102070000E94C57D1092F6061092F50614C0805994
:102080009F4DFC0180816091902D7091912D90E089
:102090000E94C57D8091F5069091F6060196909379
:1020A000F6068093F5068091F5069091F60620914C
:1020B000F7063091F806821793070CF315C060916C
:1020C000902D7091912D0E94C57D8091F706909181
:1020D000F8062091F306FC01E059FF4D208301969C
:1020E0009093F8068093F7068091F7069091F80692
:1020F0008F33910509F06CCF10926F2080916F2083
:102100008093BB178091F7069091F806FC01E05987
:10211000FF4D10829093F0068093EF061092F80620
:102120001092F7068091CE249091CF24009709F465
:102130004FCF6091F10640E050E00E94CB4048CF85
:102140001982188283E001C081E0DF91CF91089568
:1021500078948091CB069091CC060097C9F080913D
:10216000B2049091B30493FD13C092FF03C083B7F0
:10217000817F03C083B7817F866083BFF89483B774
:10218000816083BF7894889583B78E7F83BF78946E
:102190000895CF93DF93EC0188819981009721F016
:1021A0002BE08130920799F40E94DA520E94A81025
:1021B0008091820E9091830E65E840E050E00E948D
:1021C000CB4081E09BE09983888381E003C0198242
:1021D000188283E0DF91CF910895CF93DF930E941F
:1021E000DA5280EB0E94514C8823B1F40E94B74C24
:1021F0008091591C90915A1C816090935A1C809335
:10220000591C00D08FE19DE0EDB7FEB7928381832A
:102210000E94037E0F900F908EB1C82FD0E0C47043
:10222000D070729A0E94DA528EE40E94514C882338
:10223000B1F40E94B74C8091591C90915A1C826055
:1022400090935A1C8093591C00D086E19DE0EDB715
:10225000FEB7928381830E94037E0F900F90209798
:1022600009F472980E94DA528EEE0E94514C882333
:10227000B1F40E94B74C8091591C90915A1C846013
:1022800090935A1C8093591C00D08EE09DE0EDB7CE
:10229000FEB7928381830E94037E0F900F9086EA9F
:1022A0000E94514C8823B1F40E94B74C8091591C74
:1022B00090915A1C886090935A1C8093591C00D0AE
:1022C00085E09DE0EDB7FEB7928381830E94037E97
:1022D0000F900F900E94DA528CE30E94514C882399
:1022E000B1F40E94B74C8091591C90915A1C8061A6
:1022F00090935A1C8093591C00D08CEF9CE0EDB752
:10230000FEB7928381830E94037E0F900F900E94FC
:10231000DA5282ED0E94514C8823B1F40E94B74CEE
:102320008091591C90915A1C806290935A1C809302
:10233000591C00D082EF9CE0EDB7FEB792838183F9
:102340000E94037E0F900F900E94DA5280ED0E944F
:10235000514C8823B1F40E94B74C8091591C909144
:102360005A1C806890935A1C8093591C00D086EEAA
:102370009CE0EDB7FEB7928381830E94037E0F90AD
:102380000F90C7E0D0E00E94DA528CE70E94514CD7
:102390008823B9F40E94B74C8091591C90915A1C23
:1023A000806490935A1C8093591C00D08CED9CE063
:1023B000EDB7FEB7928381830E94037E0F900F904A
:1023C00002C0219701F70E94B74C0E94D90CDF91FF
:1023D000CF910895DF93CF9300D0CDB7DEB74A8376
:1023E00069830E948D4C6981862F0E94BF4C4A816F
:1023F000842F0E94BF4C0E94B74C0F900F90CF913A
:10240000DF910895AF92BF92DF92EF92FF920F9308
:102410001F93DF93CF9300D00F92CDB7DEB7082F75
:10242000D22E4A835B8369830E948D4C6981862FFB
:102430000E94BF4C802F81600E94B44C4A815B8116
:10244000042F152FAA24BB24ED2CFF240894E108A7
:10245000F1080FC0AE14BF0419F40E94DA4C02C098
:102460000E94D04CF80180830894A11CB11C0F5F1E
:102470001F4FAD1478F30E94B74C0F900F900F9040
:10248000CF91DF911F910F91FF90EF90DF90BF9060
:10249000AF900895AF92BF92CF92DF92EF92FF92EA
:1024A0000F931F93DF93CF93CDB7DEB760970FB62F
:1024B000F894DEBF0FBECDBFB82EA42E662309F45C
:1024C00055C0AE014F5F5F4F80E1DA011D928A95E2
:1024D000E9F780EB68E928E00E940212BB2059F07E
:1024E00000D088E892E0EDB7FEB7928381830E9426
:1024F000F17D0F900F908E010F5F1F4F38E0E32E9C
:10250000F12CEC0EFD1E2FE8C22E22E0D22ED801B7
:102510008D918D0100D000D0EDB7FEB73196ADB7EB
:10252000BEB71296DC92CE921197828313820E94DC
:10253000F17D0F900F900F900F900E151F0539F73A
:1025400000D000D0EDB7FEB7319684E992E0ADB788
:10255000BEB712969C938E931197888582831382BF
:102560000E94F17D0F900F900F900F90AA2009F418
:1025700057C0AE014F5F5F4F80E1FA0111928A951B
:10258000E9F780EB60E828E00E940212BB2069F0C6
:1025900000D08AE992E0ADB7BEB712969C938E93B5
:1025A00011970E94F17D0F900F908E010F5F1F4FCA
:1025B00090E1E92EF12CEC0EFD1E8FE8C82E82E092
:1025C000D82EF80181918F0100D000D0EDB7FEB771
:1025D0003196ADB7BEB71296DC92CE921197828338
:1025E00013820E94F17D0F900F900F900F900E15A7
:1025F0001F0539F700D000D0EDB7FEB7319684E95A
:1026000092E0ADB7BEB712969C938E9311978885D2
:10261000828313820E94F17D0F900F900F900F9094
:1026200060960FB6F894DEBF0FBECDBFCF91DF919D
:102630001F910F91FF90EF90DF90CF90BF90AF90E0
:1026400008950F931F93DF93CF9300D0CDB7DEB7DC
:102650001A8219828EEE6AEA8E010F5F1F4FA8015F
:1026600022E00E940212398120E08A8190E0822BD0
:10267000932B90933118809330188EEE6CEAA8015A
:1026800022E00E940212398120E08A8190E0822BB0
:10269000932B90933318809332188EEE6EEAA80134
:1026A00022E00E940212398120E08A8190E0822B90
:1026B000932B90933518809334188EEE60EBA8011D
:1026C00022E00E940212398120E08A8190E0822B70
:1026D000932B90934318809342188EEE62EBA801DF
:1026E00022E00E940212398120E08A8190E0822B50
:1026F000932B90934518809344188EEE64EBA801B9
:1027000022E00E940212398120E08A8190E0822B2F
:10271000932B90934718809346188EEE66EBA80192
:1027200022E00E940212398120E08A8190E0822B0F
:10273000932B90933718809336188EEE68EBA80190
:1027400022E00E940212398120E08A8190E0822BEF
:10275000932B90933918809338188EEE6AEBA8016A
:1027600022E00E940212398120E08A8190E0822BCF
:10277000932B90933D1880933C188EEE6CEBA80140
:1027800022E00E940212398120E08A8190E0822BAF
:10279000932B90933F1880933E188EEE6EEBA8011A
:1027A00022E00E940212398120E08A8190E0822B8F
:1027B000932B90934118809340180F900F90CF91D6
:1027C000DF911F910F9108952F923F924F925F9248
:1027D0006F927F928F929F92AF92BF92CF92DF9231
:1027E000EF92FF920F931F93DF93CF93CDB7DEB796
:1027F0006C970FB6F894DEBF0FBECDBFA82E4A8BE4
:102800002B8FFE01319683E0DF011D928A95E9F757
:1028100080915418882339F46C8F0E94211381E031
:10282000809354186C8D662309F475C08EEE64EFA6
:102830004EE20E94EA1169E07AE180E090E00E94B5
:102840003E4C8EEE66EFAE014F5F5F4F22E00E947E
:102850000212698170E080E090E0982F872F762F38
:1028600066272A8130E040E050E0622B732B842BF6
:10287000952B209146183091471840E050E0621B9C
:10288000730B840B950B209144183091451840E050
:1028900050E00E943A7A7B018C013FE01595079544
:1028A000F794E7943A95D1F760913E1870913F18EC
:1028B000882777FD8095982F2BE0660F771F881F5C
:1028C000991F2A95D1F7209140183091411844273B
:1028D00037FD4095542F2E0D3F1D401F511F0E9464
:1028E000A27A2E0D3F1D30933B1820933A18285F93
:1028F0003F4F14E0359527951A95E1F779010027A8
:10290000F7FC0095102FE0924818F09249180093B8
:102910004A1810934B18BA2DB295BB0FBB0FB07C61
:10292000BC5CB9872A2D30E03E8B2D8B63E070E0D4
:102930000A2C02C0660F771F0A94E2F7882777FDFA
:102940008095982F25E335E040E050E00E943A7AE8
:10295000DC01CB010296A11DB11D8A879B87AC8744
:10296000BD8720E533EC40E050E004C05595479525
:1029700037952795AA94D2F72E873F87488B598B96
:1029800018861C821D821E821F8248E050E08D89BD
:102990009E89481B590B5C8B4B8B69C18EEE64EF93
:1029A00049850E94EA116A857B858C859D850E94F8
:1029B0003E4C8EEE66EFAE014F5F5F4F23E00E940C
:1029C000021280913A1890913B18805A9F401C0146
:1029D000442437FC4094542CC201B101A20191015E
:1029E0000E943A7A6F8B788F898F9A8F2091341852
:1029F00030913518442737FD4095542FC201B1015D
:102A00000E943A7A7B018C01BDE015950795F794F9
:102A1000E794BA95D1F722E030E040E050E0E20ED2
:102A2000F31E041F151F6F89788D898D9A8DACE078
:102A30009595879577956795AA95D1F72091361842
:102A400030913718442737FD4095542F0E943A7A29
:102A5000BC01992777FD9095892FE60EF71E081F78
:102A6000191FE2E015950795F794E794EA95D1F7D9
:102A700080E090E8A0E0B0E0E80EF91E0A1F1B1FFE
:102A8000209142183091431840E050E0C801B7014E
:102A90000E943A7A3B014C017FE0969487947794A8
:102AA00067947A95D1F7A980BB24CC24DD246501F5
:102AB000BB24AA248A8190E0A0E0B0E0BA2FA92F1D
:102AC000982F8827A82AB92ACA2ADB2A8B8190E066
:102AD000A0E0B0E0A82AB92ACA2ADB2A0B8804C0E1
:102AE000D594C794B794A7940A94D2F7209132183A
:102AF00030913318442737FD4095542FC201B1015E
:102B00000E943A7A7B018C014BE015950795F7946A
:102B1000E7944A95D1F78091301890913118AA27FF
:102B200097FDA095BA2F32E0880F991FAA1FBB1FEF
:102B30003A95D1F7E80EF91E0A1F1B1F209138188D
:102B400030913918442737FD4095542F6F89788D7F
:102B5000898D9A8D0E943A7A27E195958795779588
:102B600067952A95D1F7E60EF71E081F191F0D88E5
:102B700004C0EE0CFF1C001F111F0A94D2F722E0C4
:102B800030E040E050E0E20EF31E041F151F82E02B
:102B900015950795F794E7948A95D1F7AE18BF0875
:102BA000C00AD10AC601B5012E853F8548895989D9
:102BB0000E943A7A97FD0BC0660F771F881F991FF6
:102BC000A40193010E94807A79018A010AC0A401BC
:102BD00093010E94807A79018A01EE0CFF1C001F8C
:102BE000111F552717FD5A95412F302F2F2DCA0140
:102BF000B9010E943A7A2EED3BE040E050E00E949D
:102C00003A7A5B016C01C801B70123E433EE4FEF60
:102C10005FEF0E943A7ABC01992777FD9095892F42
:102C20006153714F8F4F9F4F5601DD24B7FCD094F5
:102C3000CD2C6A0D7B1D8C1D9D1D44E095958795BF
:102C4000779567954A95D1F76E0D7F1D801F911F6F
:102C50002C813D814E815F81260F371F481F591FF0
:102C60002C833D834E835F8338853F5F388748855B
:102C70005A89451708F492CE552391F0252F30E05C
:102C800040E050E06C817D818E819F810E94807A3E
:102C900020934C1830934D1840934E1850934F1872
:102CA0008B8D8823C9F160914C1870914D188091DB
:102CB0004E1890914F18611571058105910561F1CC
:102CC0000E94BF7720E836EE45EC57E40E94557726
:102CD00021E03EED42E45EE30E94FE78562F472F4E
:102CE000382F292F60E070E080E89FE3DA01F901D6
:102CF0002B2F3A2F4F2F5E2F0E948A762BE43AE338
:102D00004DEB57E30E94557760935018709351181C
:102D100080935218909353186C960FB6F894DEBFB8
:102D20000FBECDBFCF91DF911F910F91FF90EF901C
:102D3000DF90CF90BF90AF909F908F907F906F90DB
:102D40005F904F903F902F900895DF93CF9300D0E6
:102D500000D000D0CDB7DEB7FE01319686E0DF01AE
:102D60001D928A95E9F780919617882399F486EA4F
:102D700061E340E00E94EA1186EA6CE24AE00E94C8
:102D8000EA1181E0809396176CE77EE380E090E0A3
:102D90000E943E4C86EA6DE248E00E94EA116CE730
:102DA0007EE380E090E00E943E4C86EA62E3AE0162
:102DB0004F5F5F4F26E00E94021286EA6DE247E015
:102DC0000E94EA119A8180E0498150E0482B592BFA
:102DD00050939117409390179C8180E02B8130E0B5
:102DE000282B392B30939317209392177E8160E024
:102DF0008D8190E0862B972B909395178093941755
:102E00006DB77EB7685070400FB6F8947EBF0FBEA6
:102E10006DBFEDB7FEB731966EE972E0ADB7BEB7E4
:102E200012967C936E931197538342833583248348
:102E3000978386830E94F17D6DB77EB7685F7F4F71
:102E40000FB6F8947EBF0FBE6DBF26960FB6F894EE
:102E5000DEBF0FBECDBFCF91DF910895CF92DF923D
:102E6000EF92FF920F931F93DF93CF9300D000D088
:102E700000D0CDB7DEB78E010F5F1F4F86E0F8019F
:102E800011928A95E9F78CE362E041E00E94EA1131
:102E90008CE360E048E50E94EA1162E174E380E0BF
:102EA00090E00E943E4C8CE363E0A80126E00E9483
:102EB00002128CE362E043E00E94EA11998180E013
:102EC0000A8110E0082B192B1093771700937617BF
:102ED0009B8180E06C8170E0682B792B709379176F
:102EE000609378173D8120E08E8190E0822B932BB8
:102EF00090937B1780937A17882777FD8095982F7A
:102F00000E94BF776B017C01B801882777FD80950F
:102F1000982F0E94BF779B01AC01C701B6010E94A8
:102F2000FE762DB73EB72C5030400FB6F8943EBF1A
:102F30000FBE2DBF0DB71EB70F5F1F4F2CEA32E03B
:102F4000EDB7FEB732832183209176173091771742
:102F5000F8013383228320917817309179173583D4
:102F6000248320917A1730917B173783268320EEB4
:102F70003EE245E652E40E949B7820E030E044E3E4
:102F800053E40E948B76F80160877187828793876C
:102F90000E94F17D2DB73EB7245F3F4F0FB6F894E6
:102FA0003EBF0FBE2DBF26960FB6F894DEBF0FBEF4
:102FB000CDBFCF91DF911F910F91FF90EF90DF90E8
:102FC000CF900895CF93DF93EC018881998100978A
:102FD00031F02AE08A3E920709F071C00BC081ED02
:102FE00096E060E870E00E9481438AEE9AE099835F
:102FF000888369C081ED96E00E94AC43009709F494
:1030000062C08091C8069091C90693FF3FC080912D
:10301000591C82FF3BC083E061E048E021E00E9450
:10302000E4138DB79EB70A970FB6F8949EBF0FBEF4
:103030008DBFEDB7FEB731968FEC91E0ADB7BEB75F
:1030400012969C938E93119780914C1890914D18E5
:10305000A0914E18B0914F1882839383A483B583B7
:103060008091501890915118A0915218B091531816
:1030700086839783A087B1870E94037E8DB79EB712
:103080000A960FB6F8949EBF0FBE8DBF8091C806FA
:103090009091C90694FF06C08091591C83FF02C01D
:1030A0000E94A5168091C8069091C90695FF97CFFA
:1030B0008091591C84FF93CF0E942E1790CF1982C4
:1030C000188283E001C081E0DF91CF910895CF9213
:1030D000DF92FF920F931F93CF93DF93729A8091A9
:1030E000B20483FD06C0C0E5D0E00E94E40A219747
:1030F000E1F78EE40E94514C8823B1F080915F206B
:1031000090916020A0916120B09162200196A11D54
:10311000B11D80935F2090936020A0936120B093B5
:10312000622021E030E084C0C0E5D0E00E94E40AE3
:103130002197E1F78FE40E94514C0E94D04CF82E69
:1031400082958695869583708130A9F420916320BD
:103150003091642040916520509166202F5F3F4F51
:103160004F4F5F4F2093632030936420409365203E
:103170005093662016C08230A0F0209167203091D5
:1031800068204091692050916A202F5F3F4F4F4F38
:103190005F4F2093672030936820409369205093BD
:1031A0006A200E94D04C1F2D1F7300E0080F111DD4
:1031B0000E94D04C0E94DA4C20E0E901C80FD11DDA
:1031C000D695C795D695C7950E94B74C8091B20405
:1031D00083FF7298B80180E090E00E94BD7720E103
:1031E00034E048EC5BE30E949B7860935518709341
:1031F00056188093571890935818BE0180E090E0BD
:103200000E94BD7724EA3CEF44E25CE30E949B7895
:1032100020E030E040E252E40E948A766093D124BC
:103220007093D2248093D3249093D42420E030E070
:10323000C901DF91CF911F910F91FF90DF90CF9047
:1032400008957298729A8EE40E94514C80EA0E940E
:10325000BF4C80E00E94BF4C80E00E94BF4C8FE4D6
:103260000E94514C0E94D04C829586958695837021
:103270008130A9F420916320309164204091652031
:10328000509166202F5F3F4F4F4F5F4F2093632039
:1032900030936420409365205093662016C082309E
:1032A000A0F02091672030916820409169205091D2
:1032B0006A202F5F3F4F4F4F5F4F2093672030931F
:1032C00068204093692050936A2000D000D0EDB769
:1032D000FEB7319621EC32E0ADB7BEB712963C9303
:1032E0002E931197828313820E94F17D0F900F908D
:1032F0000F900F908EE40E94514C80E80E94BF4CCA
:1033000080E00E94BF4C80E00E94BF4C0E94B74CFE
:1033100080E090E0089500D08FEC9CE0ADB7BEB7A0
:1033200012969C938E9311970E94037E2091950490
:103330000F900F902223A9F000D000D0EDB7FEB778
:1033400031968CEC9CE0ADB7BEB712969C938E93F1
:103350001197228313820E94037E0F900F900F908B
:103360000F90089500D087EA9CE0EDB7FEB79283F6
:1033700081830E94037E8FE79CE0EDB7FEB79283C6
:1033800081830E94037E88E59CE0EDB7FEB79283BF
:1033900081830E94037E8DE19CE0EDB7FEB79283AE
:1033A00081830E94037E8BEE9BE0EDB7FEB7928394
:1033B00081830E94037E8FEA9BE0EDB7FEB7928384
:1033C00081830E94037E89E89BE0EDB7FEB792837C
:1033D00081830E94037E83E59BE0EDB7FEB7928375
:1033E00081830E94037E83E29BE0EDB7FEB7928368
:1033F00081830E94037E87EF9AE0EDB7FEB7928348
:1034000081830E94037E8EEC9AE0EDB7FEB7928333
:1034100081830E94037E83EA9AE0EDB7FEB7928330
:1034200081830E94037E84E79AE0EDB7FEB7928322
:1034300081830E94037E82E49AE0EDB7FEB7928317
:1034400081830E94037E81E19AE0EDB7FEB792830B
:1034500081830E94037E8DED99E0EDB7FEB79283E4
:1034600081830E94037E8DEA99E0EDB7FEB79283D7
:1034700081830E94037E81E899E0EDB7FEB79283D5
:1034800081830E94037E82E599E0EDB7FEB79283C7
:1034900081830E94037E89E199E0EDB7FEB79283B4
:1034A00081830E94037E88EE98E0EDB7FEB7928399
:1034B00081830E94037E89EB98E0EDB7FEB792838B
:1034C00081830E94037E8AE898E0EDB7FEB792837D
:1034D00081830E94037E83E698E0EDB7FEB7928376
:1034E00081830E94037E8DE298E0EDB7FEB7928360
:1034F00081830E94037E84E098E0EDB7FEB792835B
:1035000081830E94037E89ED97E0EDB7FEB7928339
:1035100081830E94037E0F900F90089581ED92E0C9
:103520000E94237E08952F923F924F925F926F9256
:103530007F928F929F92AF92BF92CF92DF92EF9243
:10354000FF920F931F93CF93DF9360915B20709155
:103550005C2080915D2090915E20A0905B20B090D7
:103560005C20C0905D20D0905E2060905B207090C9
:103570005C2080905D2090905E2020905B203090B9
:103580005C2040905D2050905E202DB73EB72A50C1
:1035900030400FB6F8943EBF0FBE2DBFCDB7DEB79B
:1035A000219623EB37E0EDB7FEB732832183A0E805
:1035B000EA2EA1E5FA2EA1E00A2F112DA80197010C
:1035C0000E94807A3B832A83C601B501A801970136
:1035D0000E94807AF0E1EF2EFEE0FF2E012D112DEA
:1035E000A80197010E94807A332727FD30953D83FB
:1035F0002C83C401B301A80197010E94807AECE3F7
:10360000EE2EF12C012D112DA80197010E94807A38
:10361000332727FD30953F832E83C201B101A801D6
:1036200097010E94807A772767FD70957987688770
:103630000E94037E2DB73EB7265F3F4F0FB6F8942A
:103640003EBF0FBE2DBFDF91CF911F910F91FF9015
:10365000EF90DF90CF90BF90AF909F908F907F9032
:103660006F905F904F903F902F900895E6E9FDE2B4
:103670008081918122E482349207B9F000D000D099
:1036800085E997E0ADB7BEB712969C938E931197DC
:10369000E659FD421496FC93EE9313970E94037E25
:1036A0000F900F900F900F9008953A96B1E4E53F78
:1036B000FB07F0F208950F931F93CF93DF93EC0174
:1036C0008C9A0E94C60B00D000D000D029E837E0C9
:1036D000EDB7FEB73283218363837483858396833A
:1036E0000E94037E8DB79EB706960FB6F8949EBFD4
:1036F0000FBE8DBF209719F00E94D90C0BC000D0CF
:1037000087E897E0EDB7FEB7928381830E94037E3E
:103710000F900F9081E00E94780B00D000D000D075
:103720000DB71EB70F5F1F4F2BE737E0EDB7FEB7A2
:103730003283218320918D0430918E0440918F0437
:10374000509190040E949B78F80162837383848374
:1037500095830E94037E8DB79EB706960FB6F894A8
:103760009EBF0FBE8DBF209719F00E94D90C0BC0D1
:1037700000D089E797E0EDB7FEB7928381830E947E
:10378000037E0F900F9082E00E94780B00D000D053
:1037900000D00DB71EB70F5F1F4F2DE637E0EDB716
:1037A000FEB732832183209191043091920440919D
:1037B0009304509194040E949B78F8016283738370
:1037C000848395830E94037E8DB79EB706960FB6BD
:1037D000F8949EBF0FBE8DBF209719F00E94D90CA0
:1037E0000BC000D08BE697E0EDB7FEB792838183E4
:1037F0000E94037E0F900F9083E00E94780B00D010
:1038000000D000D02CE537E0EDB7FEB7328321833E
:1038100063837483858396830E94037E8C988DB71F
:103820009EB706960FB6F8949EBF0FBE8DBF0E943E
:10383000D90CDF91CF911F910F9108950F931F9392
:10384000CF93DF93882389F085EC94E26FEF70E0EB
:1038500049E050E00E947B7D85EC94E268E170E0F5
:1038600049E050E00E944C7F1CC0C5ECD4E207E563
:1038700017E0899100D000D0EDB7FEB73196ADB713
:10388000BEB712961C930E931197828313820E94E7
:10389000037E0F900F900F900F90B4E2CD3CDB07AA
:1038A00041F70E94D90CDF91CF911F910F9108959C
:1038B000EF92FF920F931F9360919A0470919B0473
:1038C00080E090E00E946D7D6CEE72E00E94827D4F
:1038D000009709F09EC086E294E9A0E0B0E08093F2
:1038E000AC049093AD04A093AE04B093AF048CEA03
:1038F00094E06EE070E044E050E00E944C7F8CE386
:1039000090E09093B1048093B00480EB94E062E186
:1039100070E042E050E00E944C7F8AE090E090939B
:10392000B3048093B20482EB94E064E170E042E07F
:1039300050E00E944C7F1092C9061092C80688EC95
:1039400096E060E070E042E050E00E944C7F0F2E75
:10395000F2E2EF2EFFEFFF2EFCEC0F2FFBE31F2F09
:10396000F02DE0928D04F0928E0400938F0410935A
:1039700090048DE894E066E070E044E050E00E943E
:103980004C7FE0929104F092920400939304109380
:10399000940481E994E06AE070E044E050E00E9421
:1039A0004C7F87ED94E3AFEEBCE380938904909362
:1039B0008A04A0938B04B0938C0489E894E062E0BD
:1039C00070E044E050E00E944C7F1092CD0680E011
:1039D00090E00E9433578DEC96E066E170E041E0A4
:1039E00050E00E944C7F8AE18093B4048AE190E029
:1039F0000E94AB5584EB94E067E170E041E050E059
:103A00000E944C7F81E00E941E1C80E090E00E949A
:103A1000A30E1F910F91FF90EF900895882309F452
:103A20004BC18091AC0480FF0BC000D083E597E0D0
:103A3000EDB7FEB7928381830E94037E0F900F90B3
:103A40008091AC0481FF0BC000D08EE497E0EDB70D
:103A5000FEB7928381830E94037E0F900F90809126
:103A6000AC0482FF0BC000D08BE497E0EDB7FEB74B
:103A7000928381830E94037E0F900F908091AC040B
:103A800083FF0BC000D087E497E0EDB7FEB79283C9
:103A900081830E94037E0F900F908091AC0484FF7D
:103AA0000BC000D080E497E0EDB7FEB7928381832E
:103AB0000E94037E0F900F908091AC0485FF0BC095
:103AC00000D089E397E0EDB7FEB7928381830E942F
:103AD000037E0F900F908091AC0486FF0BC000D046
:103AE00085E397E0EDB7FEB7928381830E94037E62
:103AF0000F900F908091AC0487FF0BC000D08FE235
:103B000097E0EDB7FEB7928381830E94037E0F900A
:103B10000F908091AC049091AD04A091AE04B0914F
:103B2000AF0490FF0BC000D08BE297E0EDB7FEB77B
:103B3000928381830E94037E0F900F908091AC044A
:103B40009091AD04A091AE04B091AF0491FF0BC071
:103B500000D085E297E0EDB7FEB7928381830E94A3
:103B6000037E0F900F908091AC049091AD04A091D2
:103B7000AE04B091AF0492FF0BC000D08DE197E08E
:103B8000EDB7FEB7928381830E94037E0F900F9062
:103B90008091AC049091AD04A091AE04B091AF04BB
:103BA00093FF0BC000D089E197E0EDB7FEB7928399
:103BB00081830E94037E0F900F908091AC049091BE
:103BC000AD04A091AE04B091AF0494FF0BC000D03F
:103BD00083E197E0EDB7FEB7928381830E94037E75
:103BE0000F900F908091AC049091AD04A091AE0421
:103BF000B091AF0495FF0BC000D08FE097E0EDB718
:103C0000FEB7928381830E94037E0F900F90809174
:103C1000AC049091AD04A091AE04B091AF0496FFB6
:103C20000BC000D08BE097E0EDB7FEB792838183A5
:103C30000E94037E0F900F908091AC049091AD0490
:103C4000A091AE04B091AF0497FF0BC000D087E005
:103C500097E0EDB7FEB7928381830E94037E0F90B9
:103C60000F908091AC049091AD04A091AE04B091FE
:103C7000AF04A0FF0BC000D084E097E0EDB7FEB723
:103C8000928381830E94037E0F900F908091AC04F9
:103C90009091AD04A091AE04B091AF04A1FF14C205
:103CA00000D080E097E0EDB7FEB7928381830E9459
:103CB000037E0F900F9008C200D000D000D086EF96
:103CC00096E0EDB7FEB79283818381E090E0A0E0BB
:103CD000B0E083839483A583B6830E94037E8DB76F
:103CE0009EB706960FB6F8949EBF0FBE8DBF0E947A
:103CF000D90C00D000D000D08BEE96E0EDB7FEB727
:103D00009283818382E090E0A0E0B0E0838394839B
:103D1000A583B6830E94037E8DB79EB706960FB625
:103D2000F8949EBF0FBE8DBF0E94D90C00D000D06A
:103D300000D082EE96E0EDB7FEB79283818384E0F7
:103D400090E0A0E0B0E083839483A583B6830E94D3
:103D5000037E8DB79EB706960FB6F8949EBF0FBE32
:103D60008DBF0E94D90C00D000D000D088ED96E025
:103D7000EDB7FEB79283818388E090E0A0E0B0E0E9
:103D800083839483A583B6830E94037E8DB79EB7F9
:103D900006960FB6F8949EBF0FBE8DBF0E94D90C39
:103DA00000D000D000D08BEC96E0EDB7FEB7928348
:103DB000818380E190E0A0E0B0E083839483A583D9
:103DC000B6830E94037E8DB79EB706960FB6F89411
:103DD0009EBF0FBE8DBF0E94D90C00D000D000D076
:103DE0008EEB96E0EDB7FEB79283818380E290E0A0
:103DF000A0E0B0E083839483A583B6830E94037E12
:103E00008DB79EB706960FB6F8949EBF0FBE8DBFB6
:103E10000E94D90C00D000D000D084EB96E0EDB722
:103E2000FEB79283818380E490E0A0E0B0E08383DA
:103E30009483A583B6830E94037E8DB79EB70696B2
:103E40000FB6F8949EBF0FBE8DBF0E94D90C00D054
:103E500000D000D088EA96E0EDB7FEB79283818368
:103E600080E890E0A0E0B0E083839483A583B683EC
:103E70000E94037E8DB79EB706960FB6F8949EBF3C
:103E80000FBE8DBF0E94D90C00D000D000D08EE9AB
:103E900096E0EDB7FEB79283818380E091E0A0E0E9
:103EA000B0E083839483A583B6830E94037E8DB79D
:103EB0009EB706960FB6F8949EBF0FBE8DBF0E94A8
:103EC000D90C00D000D000D082E996E0EDB7FEB763
:103ED0009283818380E092E0A0E0B0E083839483CA
:103EE000A583B6830E94037E8DB79EB706960FB654
:103EF000F8949EBF0FBE8DBF0E94D90C00D000D099
:103F000000D084E896E0EDB7FEB79283818380E02D
:103F100094E0A0E0B0E083839483A583B6830E94FD
:103F2000037E8DB79EB706960FB6F8949EBF0FBE60
:103F30008DBF0E94D90C00D000D000D08AE796E057
:103F4000EDB7FEB79283818380E098E0A0E0B0E017
:103F500083839483A583B6830E94037E8DB79EB727
:103F600006960FB6F8949EBF0FBE8DBF0E94D90C67
:103F700000D000D000D08EE696E0EDB7FEB7928379
:103F8000818380E090E1A0E0B0E083839483A58307
:103F9000B6830E94037E8DB79EB706960FB6F8943F
:103FA0009EBF0FBE8DBF0E94D90C00D000D000D0A4
:103FB00084E696E0EDB7FEB79283818380E090E2DD
:103FC000A0E0B0E083839483A583B6830E94037E40
:103FD0008DB79EB706960FB6F8949EBF0FBE8DBFE5
:103FE0000E94D90C00D000D000D08AE596E0EDB751
:103FF000FEB79283818380E090E4A0E0B0E0838309
:104000009483A583B6830E94037E8DB79EB70696E0
:104010000FB6F8949EBF0FBE8DBF0E94D90C00D082
:1040200000D000D080E596E0EDB7FEB792838183A3
:1040300080E090E8A0E0B0E083839483A583B6831A
:104040000E94037E8DB79EB706960FB6F8949EBF6A
:104050000FBE8DBF0E94D90C00D000D000D086E4E6
:1040600096E0EDB7FEB79283818380E090E0A1E017
:10407000B0E083839483A583B6830E94037E8DB7CB
:104080009EB706960FB6F8949EBF0FBE8DBF0E94D6
:10409000D90C00D000D000D08BE396E0EDB7FEB78E
:1040A0009283818380E090E0A2E0B0E083839483F8
:1040B000A583B6830E94037E8DB79EB706960FB682
:1040C000F8949EBF0FBE8DBF0E94D90C089500D0FA
:1040D0008BE296E0ADB7BEB712969C938E93119784
:1040E0000E94037E0F900F900E948E1A00D087E2EC
:1040F00096E0EDB7FEB7928381830E94037E0F9016
:104100000F9080E00E941E1C00D082E296E0ADB7C6
:10411000BEB712969C938E9311970E94037E0F90C8
:104120000F900E94ED108091591C80FF05C081E026
:1041300061E041E00E944A120E94931A00D000D030
:10414000EDB7FEB7319689E196E0ADB7BEB71296EE
:104150009C938E9311978091B404828313820E9462
:10416000037EEDB7FEB731968CE096E0ADB7BEB7F3
:1041700012969C938E9311978091CD068283138221
:104180000E94037E84EF95E0EDB7FEB792838183B2
:1041900080E490E0948383830E94037E00D0EDB797
:1041A000FEB7319681EE95E0ADB7BEB712969C93FF
:1041B0008E9311978091D524828313828091D62487
:1041C000848315820E94037E8091B2049091B3048F
:1041D000EDB7FEB736960FB6F894FEBF0FBEEDBF33
:1041E00096FF03C083EF92E002C086EF92E000D01A
:1041F00000D027ED35E0ADB7BEB712963C932E93B5
:10420000119714969C938E9313970E94037E82ECD1
:1042100095E0EDB7FEB7928381838091B0049091D1
:10422000B104948383830E94037E00D08EEA95E0DC
:10423000ADB7BEB712969C938E9311978091AC0444
:104240009091AD04A091AE04B091AF04EDB7FEB76C
:1042500083839483A583B6830E94037E2DB73EB7E4
:104260002A5F3F4F0FB6F8943EBF0FBE2DBF81E0CF
:104270000E940E1D1D9B03C083EF92E002C086EFDB
:1042800092E000D000D022EA35E0ADB7BEB712967A
:104290003C932E93119714969C938E9313970E94A0
:1042A000037E0F900F9088E995E0EDB7FEB79283FB
:1042B00081830E94037E8091B2040F900F9081FF52
:1042C0000EC000D082E995E0ADB7BEB712969C93C0
:1042D0008E9311970E94037E0F900F9017C080FF5E
:1042E00003C083EF92E002C086EF92E000D000D0DE
:1042F0002EE835E0EDB7FEB73283218394838383C4
:104300000E94037E0F900F900F900F908091C8062F
:104310009091C90600D000D021E835E0ADB7BEB716
:1043200012963C932E93119714969C938E93139709
:104330000E94037E0F900F900F900F90779903C00B
:1043400083EF92E002C086EF92E000D000D028E731
:1043500035E0EDB7FEB732832183948383830E94D7
:10436000037E0F900F900F900F900E9495080E946F
:10437000FD0B0E94DA0B00D000D000D02AE635E019
:10438000ADB7BEB712963C932E931197EDB7FEB71B
:1043900063837483858396830E94037E2DB73EB723
:1043A0002A5F3F4F0FB6F8943EBF0FBE2DBF81E08E
:1043B00090E00E945B1B8091B0249091B124A09169
:1043C000B224B091B32400D000D000D02CE535E069
:1043D000EDB7FEB73283218383839483A583B683AD
:1043E0000E94037E88E495E0ADB7BEB712969C9319
:1043F0008E9311978091BD249091BE24A091BF24EB
:10440000B091C024EDB7FEB783839483A583B683B0
:104410000E94037E8091B4249091B524A091B6248B
:10442000B091B7242AE335E0EDB7FEB7328321839C
:1044300083839483A583B6830E94037E86E295E0FE
:10444000ADB7BEB712969C938E9311978091C124FD
:104450009091C224A091C324B091C424EDB7FEB7BB
:1044600083839483A583B6830E94037E2DB73EB7D2
:104470002A5F3F4F0FB6F8943EBF0FBE2DBF80E0BE
:1044800090E061E070E00E94E50C81E090E061E086
:1044900070E00E94E50C08952F923F924F925F9238
:1044A0006F927F928F929F92AF92BF92CF92DF9244
:1044B000EF92FF920F931F93DF93CF9300D0CDB76E
:1044C000DEB79A838983DC018D919C9111970097C7
:1044D00011F00C94EA3360919A0470919B0480E788
:1044E00090E20E946D7D80E790E260E470E00E94BF
:1044F0008B7D009759F46091902D7091912D8AE0F9
:1045000090E00E94C57D81E00C94EF3381309105ED
:1045100049F42090702033244424552466247724C1
:104520004301BFC18230910599F4309170202091F0
:104530007120932F80E0820F911D1C01892F880F1D
:10454000880B482E582E682E782E882E982EA9C1BA
:104550008330910509F09CC020917020A0907120BB
:104560008090722030E040E050E060E070E080E059
:1045700090E000E10E942772F22E132FE42ED52E38
:10458000C62EB72E282E992E2A2D30E040E050E07E
:1045900060E070E080E090E008E00E9427722F0D5C
:1045A000B1E02F1508F0B0E0310FE1E0311708F06D
:1045B000E0E0B30FF1E0B31708F0F0E0EF2B4E0DA1
:1045C00031E04E1508F030E0E40FF1E0E41708F0B8
:1045D000F0E03F2B5D0D41E05D1508F040E0A32FBA
:1045E000A50F31E0A51708F030E0432B6C0D31E04A
:1045F0006C1508F030E0F42FF60F41E0F61708F0E4
:1046000040E0342B7B0D41E07B1508F040E0532F58
:10461000570F31E0571708F030E0432B820D31E09F
:10462000821508F030E0480F61E0481708F060E0BC
:10463000362B990D930F022F080D11E0021708F089
:1046400010E01B0F81E01B1708F080E0B82FBE0FB1
:1046500071E0BE1708F070E07A0F61E07A1708F099
:1046600060E06F0F31E06F1708F030E0350F21E0A8
:10467000351708F020E0240F81E0241708F080E0CF
:1046800018014B2E572E662E732E822E982EFEC0AA
:10469000843091050CF4FCC020917020A090712012
:1046A000709072208090732030E040E050E060E035
:1046B00070E080E090E008E10E942772F22E132F54
:1046C000E42ED52EC62EB72E282E992E2A2D30E078
:1046D00040E050E060E070E080E090E000E10E94A7
:1046E00027722F0DF1E02F1508F0F0E0310FE1E017
:1046F000311708F0E0E0F30FA1E0F31708F0A0E0B5
:10470000EA2B4E0D31E04E1508F030E0E40FA1E049
:10471000E41708F0A0E03A2B5D0D41E05D1508F0CC
:1047200040E0B32FB50F31E0B51708F030E0432B70
:104730006C0D31E06C1508F030E0A42FA60F41E0BD
:10474000A61708F040E0342B7B0D41E07B1508F004
:1047500040E0532F570F31E0571708F030E0432B5C
:10476000820D31E0821508F030E0480F61E0481713
:1047700008F060E0362B990E930E122F180D81E091
:10478000121708F080E0282E2F0E81E02F1608F077
:1047900080E0F82EFE0E81E0FE1608F080E0E82EA4
:1047A000EB0E81E0EB1608F080E0D82EDA0E81E007
:1047B000DA1608F080E0C82EC50E81E0C51608F0B4
:1047C00080E0B82EB40E81E0B41608F080E0980EB8
:1047D000272D30E040E050E060E070E080E090E0C5
:1047E00008E00E942772210FE1E0211708F0E0E0C5
:1047F000320DF1E0321508F0F0E0E30FA1E0E3172D
:1048000008F0A0E0FA2B4F0D31E04F1508F030E032
:10481000F40FA1E0F41708F0A0E03A2B5E0D41E0A0
:104820005E1508F040E0A32FA50F31E0A51708F0B2
:1048300030E0432B6D0D31E06D1508F030E0542F62
:10484000560F41E0561708F040E0342B7C0D41E054
:104850007C1508F040E0632F670F31E0671708F020
:1048600030E0432B8B0D31E08B1508F030E0480F22
:1048700071E0481708F070E0372B990D222E3E2E7C
:104880004F2E5A2E652E762E842E932E990E09C009
:10489000AAE02A2E3324442455246624772488242D
:1048A00099240E94D90CB22DB43691F4E32DE3364D
:1048B00079F4F42DFC3661F4552051F4662041F46E
:1048C000772031F4882021F4992011F40C947A2F68
:1048D0009101A201B301C401F4E6AF2EE3E6BE2EBE
:1048E0000CE6C02EDD24EE24FF2400E010E00E9440
:1048F0009872823008F061C2822D853689F4932D3A
:10490000923771F4442061F4552051F4662041F44B
:10491000772031F4882021F4992011F40C949931F6
:104920009101A201B301C40115E6A12EB2E7BB2E8D
:10493000CC24DD24EE24FF2400E010E00E949872D5
:10494000823008F0F6C0A22DA53681F4B32DB4361E
:1049500069F4442059F4552049F4662039F477204D
:1049600029F4882019F4992009F4C4C69101A20100
:10497000B301C401A5E6AA2EF4E6BF2ECC24DD24A3
:10498000EE24FF2400E010E00E949872823008F0CC
:1049900064C0E22DE53781F4332071F4442061F4E2
:1049A000552051F4662041F4772031F4882021F419
:1049B000992011F40C94632D9101A201B301C4015B
:1049C000E5E7AE2EBB24CC24DD24EE24FF2400E05A
:1049D00010E00E949872823010F5F22DF83611F036
:1049E0000C94E833332011F00C94E833442011F098
:1049F0000C94E833552011F00C94E833662011F044
:104A00000C94E833772011F00C94E833882011F0EF
:104A10000C94E833992011F00C94E83388C7822D68
:104A2000863781F4332071F4442061F4552051F429
:104A3000662041F4772031F4882021F4992011F484
:104A40000C94722D922D943611F00C94E833A32D12
:104A5000A13611F00C94E83367C0B22DB53689F455
:104A6000E32DEE3671F4442061F4552051F46620B4
:104A700041F4772031F4882021F4992011F40C942A
:104A8000D7309101A201B301C40105E6A02E1EE6B4
:104A9000B12ECC24DD24EE24FF2400E010E00E949F
:104AA0009872823018F5F22DF43611F00C94E83338
:104AB000832D893611F00C94E833442011F00C94C6
:104AC000E833552011F00C94E833662011F00C9473
:104AD000E833772011F00C94E833882011F00C941F
:104AE000E833992011F00C94E833CDC7922D973715
:104AF00089F4A32DAF3671F4442061F4552051F4AC
:104B0000662041F4772031F4882021F4992011F4B3
:104B10000C94AD30B22DB33311F00C94E833E32D87
:104B2000E13711F00C94E833442011F00C94E83391
:104B300095C0F22DF83789F4832D843671F4942DC5
:104B4000913659F4552049F4662039F4772029F438
:104B5000882019F4992009F4FBC39101A201B30143
:104B6000C401B8E7AB2EA4E6BA2EF1E6CF2EDD24C1
:104B7000EE24FF2400E010E00E949872823008F0DA
:104B800083C0A22DA33789F4B32DB23771F444202A
:104B900061F4552051F4662041F4772031F48820E7
:104BA00021F4992011F40C9465329101A201B30112
:104BB000C401E3E7AE2E02E7B02ECC24DD24EE24C0
:104BC000FF2400E010E00E949872823020F5E22D70
:104BD000E93611F00C94E833F32DF23711F00C9410
:104BE000E833442011F00C94E833552011F00C9474
:104BF000E833662011F00C94E833772011F00C9420
:104C0000E833882011F00C94E833992011F00C94CB
:104C1000E8330C941232822D833789F4932D933725
:104C200071F4442061F4552051F4662041F477205A
:104C300031F4882021F4992011F40C947432A22DBF
:104C4000A33611F00C94E833B32DB43611F00C9464
:104C5000E833E42DE13611F00C94E833552011F0DF
:104C60000C94E833662011F00C94E833772011F0AF
:104C70000C94E833882011F00C94E833992011F05B
:104C80000C94E8330C948332F22DF33689F4832D9F
:104C90008D3671F4942D983659F4552049F46620D8
:104CA00039F4772029F4882019F4992009F458C39D
:104CB0009101A201B301C40113E6A12EBDE6BB2EF2
:104CC000A8E6CA2EDD24EE24FF2400E010E00E94B6
:104CD00098728230C8F5A22DA23689F4B32DB5366C
:104CE00071F4E42DE43659F4552049F4662039F482
:104CF000772029F4882019F4992009F4FBC4F22DB7
:104D0000F23711F00C94E833832D823711F00C94B4
:104D1000E833942D953611F00C94E833552011F0BA
:104D20000C94E833662011F00C94E833772011F0EE
:104D30000C94E833882011F00C94E833992011F09A
:104D40000C94E8330C94D02FA22DAD3691F4B32DF2
:104D5000B53779F4E42DE83661F4552051F4662036
:104D600041F4772031F4882021F4992011F40C9437
:104D70009432F22DF33611F00C94E833832D823304
:104D800011F00C94E833942D993611F00C94E8331B
:104D9000552011F00C94E833662011F00C94E833A0
:104DA000772011F00C94E833882011F00C94E8334C
:104DB000992011F00C94E833CFC2A22DA03791F4C2
:104DC000B32DBC3679F4E42DE53661F4F52DF836D3
:104DD00049F4662039F4772029F4882019F49920C1
:104DE00009F4A5C59101A201B301C401F0E7AF2EFA
:104DF000ECE6BE2E05E6C02E18E6D12EEE24FF24EA
:104E000000E010E00E949872823008F04DC1822DBF
:104E1000803791F4932D953679F4A42DA23761F45F
:104E2000552051F4662041F4772031F4882021F494
:104E3000992011F40C9499319101A201B301C4019C
:104E4000B0E7AB2EA5E6BA2EF2E7CF2EDD24EE2496
:104E5000FF2400E010E00E949872823008F087C0C2
:104E6000B22DB53791F4E32DE33679F4F42DFD3608
:104E700061F4552051F4662041F4772031F4882004
:104E800021F4992011F40C9433309101A201B30163
:104E9000C401E5E7AE2E03E6B02E1DE6C12EDD24EB
:104EA000EE24FF2400E010E00E949872823028F582
:104EB000822D873611F00C94E833932D9F3611F034
:104EC0000C94E833A42DAC3611F00C94E833552043
:104ED00011F00C94E833662011F00C94E83377203D
:104EE00011F00C94E833882011F00C94E8339920E9
:104EF00011F00C94E8330C947D2FB22DB03391F463
:104F0000E32DE13379F4F42DF13761F4552051F4B8
:104F1000662041F4772031F4882021F4992011F49F
:104F20000C94D02F822D813311F00C94E833932D03
:104F3000913311F00C94E833A42DA13711F00C94A7
:104F4000E833552011F00C94E833662011F00C94EE
:104F5000E833772011F00C94E833882011F00C949A
:104F6000E833992011F00C94E8330C943330B22DCF
:104F7000B93691F4E32DEC3679F4F42DF13661F481
:104F8000852D833649F4662039F4772029F488206A
:104F900019F4992009F411C29101A201B301C401CD
:104FA000B9E6AB2EACE6BA2EF1E6CF2EE3E6DE2E66
:104FB000EE24FF2400E010E00E9498728230D0F5C9
:104FC000922D943791F4A32DA43679F4B42DB737EC
:104FD00061F4552051F4662041F4772031F48820A3
:104FE00021F4992011F40C947533E22DE43711F07B
:104FF0000C94E833F32DFF3611F00C94E833842D34
:105000008F3611F00C94E833952D923611F00C94F4
:10501000E833662011F00C94E833772011F00C94FB
:10502000E833882011F00C94E833992011F00C94A7
:10503000E833B8C5A22DAE3691F4B32DB13679F46C
:10504000E42DE83661F4F52DF33649F4662039F4A1
:10505000772029F4882019F4992009F478C5822D45
:10506000863311F00C94E833932D993611F00C949B
:10507000E833A42DA53711F00C94E833B52DB536DF
:1050800011F00C94E833662011F00C94E83377208B
:1050900011F00C94E833882011F00C94E833992037
:1050A00011F00C94E83346C4E22DE13691F4F32D6F
:1050B000FC3679F4842D853661F4952D923749F4C8
:1050C000662039F4772029F4882019F4992009F40E
:1050D00047C49101A201B301C40101E6A02E1CE660
:1050E000B12EB5E6CB2EA2E7DA2EEE24FF2400E0A7
:1050F00010E00E949872823008F08BC0A22DA23777
:1051000091F4B32DB73779F4E42DE03761F4F52D40
:10511000F03749F4662039F4772029F4882019F40F
:10512000992009F421C19101A201B301C401F2E760
:10513000AF2EE7E7BE2E00E7C02E10E7D12EEE24FB
:10514000FF2400E010E00E949872823030F5822D3A
:10515000813611F00C94E833932D9D3611F00C94A8
:10516000E833A42DA53711F00C94E833B52DB836EB
:1051700011F00C94E833662011F00C94E83377209A
:1051800011F00C94E833882011F00C94E833992046
:1051900011F00C94E8330C94C630E22DE33799F407
:1051A000F32DF53681F4842D823769F4952D9037EF
:1051B00051F4662041F4772031F4882021F49920BD
:1051C00011F40C94DE32A22DA33711F00C94E833C5
:1051D000B32DB23711F00C94E833E42DE73711F01A
:1051E0000C94E833F52DF03711F00C94E833662079
:1051F00011F00C94E833772011F00C94E8338820F8
:1052000011F00C94E833992011F00C94E8330C94CD
:105210006531822D873791F4932D903779F4A42D41
:10522000A83761F4B52DB43749F4662039F47720F6
:1052300029F4882019F4992009F463C49101A2018A
:10524000B301C401B7E7AB2EA0E7BA2EF8E7CF2E23
:10525000E4E7DE2EEE24FF2400E010E00E949872C6
:105260008230D8F5E22DE43799F4F32DF33781F449
:10527000842D853669F4952D923751F4662041F4DA
:10528000772031F4882021F4992011F40C946231B4
:10529000A22DA43711F00C94E833B32DB33711F0DD
:1052A0000C94E833E42DE53611F00C94E833F52D39
:1052B000F43711F00C94E833662011F00C94E833C5
:1052C000772011F00C94E833882011F00C94E83327
:1052D000992011F00C94E83368C4822D823791F440
:1052E000932D973679F4A42DA03761F4B52DB537F9
:1052F00049F4662039F4772029F4882019F499209C
:1053000009F4C7C5E22DEC3611F00C94E833F32D07
:10531000F13611F00C94E833842D843711F00C949D
:10532000E833952D983711F00C94E833662011F08E
:105330000C94E833772011F00C94E833882011F0B6
:105340000C94E833992011F00C94E8330C94393321
:105350000E94A5160C94EA330E94ED100C94EA33D7
:105360000E942E170C94EA3360919A0470919B046A
:1053700080E090E00E946D7D8C0163EF72E00E94FE
:10538000827D009719F477980C94EA33C80166EF90
:1053900072E00E94827D009719F4779A0C94EA33A8
:1053A000779903C083EF92E002C086EF92E000D0CD
:1053B00000D02DE234E00C94D73360919A047091C0
:1053C0009B0480E090E00E946D7D8C016AEF72E0AA
:1053D0000E94827D009709F052C060919A047091FA
:1053E0009B0480E090E00E946D7D8C01009711F499
:1053F0000C94EA336DEF72E00E94827D009729F4ED
:1054000082E29FEFACECBBE30BC0C80163E073E04A
:105410000E94827D009789F482E29FEFACECBAE3B0
:1054200080938D0490938E04A0938F04B093900486
:105430008DE894E066E070E0DCC0C8010E94607C0A
:105440007B018C0120E030E0A9010E945177882384
:1054500091F081E00E94780B9B01AC01C801B7017B
:105460000E94557760938D0470938E0480938F040F
:1054700090939004DDCF00D08DE694E08CC0C801FD
:1054800068E073E00E94827D009709F052C060914D
:105490009A0470919B0480E090E00E946D7D8C01E5
:1054A000009711F40C94EA336DEF72E00E94827D54
:1054B000009729F482E29FEFACECBBE30BC0C8017C
:1054C00063E073E00E94827D009769F482E29FEFBF
:1054D000ACECBAE38093910490939204A09393046C
:1054E000B09394041DC0C8010E94607C7B018C01B4
:1054F00020E030E0A9010E9451778823B1F082E0DA
:105500000E94780B9B01AC01C801B7010E9455773E
:105510006093910470939204809393049093940405
:1055200081E994E06AE070E064C000D080E694E035
:1055300067C0C8016BE073E00E94827D009709F0AC
:105540006BC060919A0470919B0480E090E00E948F
:105550006D7D8C01009711F40C94EA336DEF72E0CD
:105560000E94827D009769F487ED94E3AFEEBCE37F
:105570008093890490938A04A0938B04B0938C0445
:1055800034C0C80163E073E00E94827D009741F45B
:1055900000D081E594E0EDB7FEB79283818336C0F9
:1055A000C8010E94607C1B012C0120E030E0A901B1
:1055B0000E945177882309F180E00E94780B7B01DB
:1055C0008C01C201B10121EE3AE744E95EE30E9499
:1055D0008A76A80197010E94557760938904709399
:1055E0008A0480938B0490938C0489E894E062E0B1
:1055F00070E044E050E00C94B83300D084E494E0D0
:10560000ADB7BEB712969C938E9311970E94037EFE
:105610000F900F900C94EA330E94C60B00D000D07C
:1056200000D02DE334E0EDB7FEB732832183ADB770
:10563000BEB713966D937D938D939C9316970E949E
:10564000037EEDB7FEB736960FB6F894FEBF0FBED9
:10565000EDBF81E00E94780B20918D0430918E0483
:1056600040918F04509190040E949B787B018C01A3
:1056700082E00E94780B9B01AC018DB79EB70A9720
:105680000FB6F8949EBF0FBE8DBFCDB6DEB60894A0
:10569000C11CD11C81E394E0ADB7BEB712969C93B8
:1056A0008E9311978E2D9F2DA02FB12FF6018283FF
:1056B0009383A483B583CA01B901209191043091E9
:1056C000920440919304509194040E949B78D601D7
:1056D00016966D937D938D939C9319970E94037EEC
:1056E000EDB7FEB73A960FB6F894FEBF0FBEEDBF0A
:1056F0000C94723360919A0470919B0480E090E066
:105700000E946D7D009761F160E070E040E150E043
:105710000E94527B2091C8063091C9062617370790
:1057200099F17093C9066093C80688EC96E060E032
:1057300070E042E050E00E944C7F8091C80690915A
:10574000C90600D000D02DE134E0ADB7BEB7129647
:105750003C932E93119714969C938E9313970EC09F
:105760008091C8069091C90600D000D029E034E0AD
:10577000EDB7FEB732832183948383830E94037E37
:105780000F900F900F900F900E94D90C00D000D076
:105790008CEF93E0ADB7BEB712969C938E931197A2
:1057A00081E090E014969C938E9313970E94037E61
:1057B00081EF93E0EDB7FEB79283818382E090E0C2
:1057C000948383830E94037E86EE93E0ADB7BEB7D9
:1057D00012969C938E93119784E090E014969C937C
:1057E0008E9313970E94037E8AED93E0EDB7FEB788
:1057F0009283818388E090E0948383830E94037E78
:105800008FEC93E0ADB7BEB712969C938E93119731
:1058100080E190E014969C938E9313970E94037EF0
:1058200083EC93E0EDB7FEB79283818380E290E052
:10583000948383830E94037E85EB93E0ADB7BEB76C
:1058400012969C938E93119780E490E014969C930B
:105850008E9313970E94037E86EA93E0EDB7FEB71E
:105860009283818380E890E0948383830E94037E07
:1058700087E993E0ADB7BEB712969C938E931197CC
:1058800080E091E014969C938E9313970E94037E80
:105890008BE893E0EDB7FEB79283818380E092E0DE
:1058A000948383830E94037E8DE793E0ADB7BEB7F8
:1058B00012969C938E93119780E094E014969C939B
:1058C0008E9313970E94037E80E793E0EDB7FEB7B7
:1058D0009283818380E098E0948383830E94037E97
:1058E00082E693E0ADB7BEB712969C938E93119764
:1058F00080E090E114969C938E9313970E94037E10
:1059000083E593E0EDB7FEB79283818380E090E278
:10591000948383830E94037E85E493E0ADB7BEB792
:1059200012969C938E93119780E090E446C70E9454
:10593000B21950C780917420843329F480E061E06B
:1059400040E00E944A1220919504222309F442C7A4
:1059500000D000D0EDB7FEB7319682E493E08AC064
:1059600080917420893709F079C060919A04709110
:105970009B0480E090E00E946D7D8C0163EF72E0FB
:105980000E94827D009731F48091B2049091B3041B
:1059900090640CC0C80166EF72E00E94827D00979F
:1059A00091F48091B2049091B3049F7B9093B304DF
:1059B0008093B20482EB94E064E170E042E050E056
:1059C0000E944C7F4BC0C80160E173E00E94827D61
:1059D000009729F500D000D000D0EDB7FEB7319682
:1059E0008EE794E0ADB7BEB712969C938E93119755
:1059F000809197179091981793838283809199173C
:105A000090919A17958384830E94037EEDB7FEB729
:105A100036960FB6F894FEBF0FBEEDBF1FC0809143
:105A2000B2049091B30496FF03C083EF92E002C0EA
:105A300086EF92E000D000D02AE734E0ADB7BEB7E1
:105A400012963C932E93119714969C938E931397D2
:105A50000E94037E0F900F900F900F90209195045D
:105A6000222309F4B7C600D000D0EDB7FEB73196B7
:105A70008FE393E0ADB7BEB712969C938E931197C8
:105A8000228313829EC660919A0470919B0480E0E9
:105A900090E00E946D7D6DEF72E00E94827D009724
:105AA00011F481E001C080E00E941E1C2091950449
:105AB000222309F48FC600D000D0EDB7FEB731968F
:105AC0008CE393E0D7CF0E94931A20919504222370
:105AD00009F480C600D000D0EDB7FEB7319689E357
:105AE00093E0C8CF0E948E1A20919504222309F4D6
:105AF00071C600D000D0EDB7FEB7319686E393E0D3
:105B0000B9CF60919A0470919B0480E090E00E946C
:105B10006D7D0E94647C803150F48093CD0690E0CE
:105B20000E9433578DEC96E066E170E027C000D00C
:105B300000D0EDB7FEB7319687E994E0ADB7BEB7B8
:105B400012969C938E9311978091CD0629C06091F7
:105B50009A0470919B0480E090E00E946D7D0E9409
:105B6000647C982F9B50903160F48093B40490E053
:105B70000E94AB5584EB94E067E170E041E050E0B7
:105B8000F7C500D000D0EDB7FEB7319684EA94E0B7
:105B9000ADB7BEB712969C938E9311978091B404C3
:105BA00082836FCF0C94000015C660919A047091A7
:105BB0009B0480E090E00E946D7D8C0166E173E0C3
:105BC0000E94827D009739F4219A8091B2049091CD
:105BD000B3048061C3C5C80168E173E00E94827D9F
:105BE000009739F4229A8091B2049091B3048062B4
:105BF000B5C5C8016AE173E00E94827D009739F45F
:105C0000239A8091B2049091B3048064A7C5C8011F
:105C10006CE173E00E94827D009739F4239A8091B1
:105C2000B2049091B304806899C5C8016EE173E035
:105C30000E94827D0097C9F48091B2049091B304D0
:105C400091609093B3048093B20482EB94E064E19A
:105C500070E042E050E00E944C7F85EF94E062E10A
:105C600040E050E00E94CB40B5C5C80160E273E05F
:105C70000E94827D009771F4EBE9F7E11192119295
:105C8000B7E1EB3BFB07D1F78091B2049091B304ED
:105C9000926064C5C80166EF72E00E94827D9C013B
:105CA0008091B2049091B30421153105A9F48F704D
:105CB0009C7F9093B3048093B2042B9A82EB94E080
:105CC00064E170E042E050E00E944C7F8091BC248F
:105CD00090E00E94C0557EC584FF03C083EF92E030
:105CE00002C086EF92E000D000D024EE34E0EDB7A1
:105CF000FEB732832183948383830E94037E809145
:105D0000B2040F900F900F900F9085FF03C083EFA8
:105D100092E002C086EF92E000D000D029ED34E09E
:105D2000ADB7BEB712963C932E93119714969C93E1
:105D30008E9313970E94037E8091B2040F900F9070
:105D40000F900F9086FF03C083EF92E002C086EFB2
:105D500092E000D000D02EEC34E0EDB7FEB73283F5
:105D60002183948383830E94037E8091B2040F90E9
:105D70000F900F900F9087FF03C083EF92E002C057
:105D800086EF92E000D000D023EC34E0ADB7BEB790
:105D900012963C932E93119714969C938E9313977F
:105DA0000E94037E8091B2049091B3040F900F90F3
:105DB0000F900F9090FF03C083EF92E002C086EF38
:105DC00092E000D000D028EB34E0EDB7FEB732838C
:105DD0002183948383830E94037E8091B2049091F7
:105DE000B3040F900F900F900F9091FF03C083EFBB
:105DF00092E002C086EF92E000D000D02DEA34E0BD
:105E0000ADB7BEB712963C932E93119714969C9300
:105E10008E9313970E94037E8091B2049091B304F5
:105E20000F900F900F900F9091FFD4C482E293E0F7
:105E30000E94237E0BE917E18BE0C82ED12CBAE239
:105E4000EB2EB3E0FB2EF801819191918F0100D0F0
:105E500000D000D0EDB7FEB73196ADB7BEB7129601
:105E6000FC92EE921197D382C282958384830E9422
:105E7000F17D0894C11CD11CEDB7FEB736960FB664
:105E8000F894FEBF0FBEEDBFFBE1CF16D104D9F6EB
:105E9000A1C400D082E393E0ADB7BEB712969C9345
:105EA0008E9311970E94037E209195040F900F907E
:105EB0002223A9F000D000D0EDB7FEB731968FE2D3
:105EC00093E0ADB7BEB712969C938E931197228341
:105ED00013820E94037E0F900F900F900F9088E125
:105EE0000FB6F89480936000109260000FBE0C947F
:105EF000007C70C40E94DD4D6DC460919A04709165
:105F00009B0480E090E00E946D7D1C0163EF72E0D5
:105F10000E94827D009749F40E948A548091B204C5
:105F20009091B30481608D7F19C4C10166EF72E066
:105F30000E94827D009741F40E94EC538091B2044C
:105F40009091B3048C7F0AC405E313E0C101B8014A
:105F50000E94827D009749F40E94EC538091B20424
:105F60009091B3048E7F8260F9C38091B20481FF67
:105F70000BC000D000D083EF94E0EDB7FEB7928362
:105F80008183148303831DC480FF03C083EF92E0E9
:105F900002C086EF92E000D000D02FEE34E007C4BC
:105FA00000D085E093E0EDB7FEB7928381830E9435
:105FB000037E8DB79EB740970FB6F8949EBF0FBE75
:105FC0008DBFEDB7FEB7319687EE92E0ADB7BEB7A5
:105FD00012969C938E93119780916B2090916C20D8
:105FE000A0916D20B0916E2082839383A483B583AA
:105FF00080915F2090916020A0916120B0916220FB
:1060000086839783A087B1878091632090916420D5
:10601000A0916520B091662082879387A487B58779
:106020008091672090916820A0916920B0916A20AA
:1060300086879787A08BB18B0E94037E2091950461
:10604000EDB7FEB772960FB6F894FEBF0FBEEDBF68
:10605000222309F4BFC300D000D0EDB7FEB73196BC
:1060600084EE92E007CDF89481E090E00E948E08E3
:10607000182F80E090E00E948E08082F7894F89402
:1060800083E090E00E948E08F82E82E090E00E946B
:106090008E08E82E789400D000D000D02AED32E0AF
:1060A000EDB7FEB73283218320910C1830910D1883
:1060B00040910E1850910F18ADB7BEB713962D939F
:1060C0003D934D935C9316970E94037E00D000D0C1
:1060D000EDB7FEB7319623EB32E0ADB7BEB71296FF
:1060E0003C932E931197E2821382F48215820683E9
:1060F0001782108711860E94037EEDB7FEB73A968D
:106100000FB6F894FEBF0FBEEDBF0E94361B209164
:10611000660000D000D0EDB7FEB7319687EA92E076
:10612000ADB7BEB712969C938E93119722831382BC
:106130000E94037E0F900F900F900F900E94D90C39
:1061400020919504222309F445C300D000D0EDB777
:10615000FEB7319684EA92E08DCC80E090E060E07A
:1061600070E00E94E50C81E090E060E070E00E9449
:10617000E50C20919504222309F42CC300D000D013
:10618000EDB7FEB7319681EA92E074CC0E942119F6
:106190000E94D90C20919504222309F41BC300D03E
:1061A00000D0EDB7FEB731968EE992E063CC6091F6
:1061B0009A0470919B0480E090E00E946D7D6AE3F8
:1061C00073E00E94827D009741F5F8948DEE96E091
:1061D0000E94C2410CC0C8010D960E940E4582E487
:1061E00095E0B8010E947C41C8010E948842082FB6
:1061F000192F0115110579F704C08DEE96E00E9464
:1062000003428DEE96E00E9468420097B1F78DEE52
:1062100096E00E94BE41789448C08DEE96E00E94C0
:10622000C241482F592F7A0100E413E03BC0EDB77B
:10623000FEB73C970FB6F894FEBF0FBEEDBF319688
:10624000ADB7BEB712961C930E931197D701129655
:106250008C9112978283138213968C911397848367
:10626000158218968C9118978683178214968D91B3
:106270009C9115979187808716968D919C91179781
:10628000938782870E94F17DEDB7FEB73C960FB6EB
:10629000F894FEBF0FBEEDBFC7010E948842482F91
:1062A000592F7A01E114F10411F62091950422236B
:1062B00009F490C200D000D0EDB7FEB731968BE95B
:1062C00092E0D8CB0E94581C85C260919A047091CC
:1062D0009B0480E090E00E946D7D8C0167E673E096
:1062E0000E94827D009731F48091B2049091B304B2
:1062F000937F34C2C80163E073E00E94827D0097FF
:1063000039F48091B2049091B304937F986026C2CF
:10631000C8016CE673E00E94827D009739F4809199
:10632000B2049091B304937F946018C20E949508C0
:1063300051C260919A0470919B0480E090E00E94A9
:106340006D7D0097A9F160E070E040E150E00E94AF
:10635000527B6093AC047093AD048093AE04909331
:10636000AF0400D000D000D028E832E0EDB7FEB78F
:1063700032832183ADB7BEB713966D937D938D9312
:106380009C9316970E94037EEDB7FEB736960FB624
:10639000F894FEBF0FBEEDBF8CEA94E06EE070E0B3
:1063A00044E050E00E944C7F81E00E940E1D12C22A
:1063B00080E00E940E1D0E94D90C00D000D000D0B9
:1063C00083E792E0ADB7BEB712969C938E93119778
:1063D0008091AC049091AD04A091AE04B091AF0453
:1063E000EDB7FEB783839483A583B6830E94037EB3
:1063F0008DB79EB706960FB6F8949EBF0FBE8DBFA1
:1064000081E00E940E1D0E94D90C20919504222348
:1064100009F4E0C100D000D0EDB7FEB7319680E7B7
:1064200092E028CB60919A0470919B0480E090E008
:106430000E946D7D009741F160E070E04AE050E01D
:106440000E94527B7093B1046093B00400D000D0DE
:10645000EDB7FEB7319623E532E0ADB7BEB7129681
:106460003C932E931197738362830E94037E0F9057
:106470000F900F900F9080EB94E062E170E042E0AB
:1064800050E00E944C7F14C000D000D082E392E024
:10649000EDB7FEB7928381838091B0049091B104EF
:1064A000948383830E94037E0F900F900F900F9030
:1064B00020919504222309F48DC100D000D0EDB7BE
:1064C000FEB731968FE292E0D5CA0E944B452091EB
:1064D0009504222309F47EC100D000D0EDB7FEB7A9
:1064E00031968CE292E0C6CA0E9467202091950402
:1064F000222309F46FC100D000D0EDB7FEB731966A
:1065000089E292E0B7CA80E090E00E945B1B209194
:106510009504222309F45EC100D000D0EDB7FEB788
:10652000319686E292E0A6CA0E9467180097B9F5F4
:1065300000D000D000D08BE192E0EDB7FEB792839F
:1065400081838091551890915618A0915718B09159
:10655000581883839483A583B6830E94037E8EE0BC
:1065600092E0ADB7BEB712969C938E93119780912F
:10657000D1249091D224A091D324B091D424EDB70A
:10658000FEB783839483A583B6830E94037E8DB771
:106590009EB706960FB6F8949EBF0FBE8DBF0E94A1
:1065A000D90C20919504222309F414C100D000D005
:1065B000EDB7FEB731968BE092E05CCA83E061E014
:1065C00048E021E00E94E41300D000D000D084E035
:1065D00092E0EDB7FEB79283818380914818909145
:1065E0004918A0914A18B0914B1883839483A583CE
:1065F000B6830E94037E00D000D0EDB7FEB731967F
:1066000083EF91E0ADB7BEB712969C938E9311972E
:1066100080914C1890914D18A0914E18B0914F1840
:1066200082839383A483B5838091501890915118ED
:10663000A0915218B091531886839783A087B18791
:106640000E94037EEDB7FEB73A960FB6F894FEBFF0
:106650000FBEEDBF0E94D90C20919504222309F4AE
:10666000B9C000D000D0EDB7FEB7319680EF91E011
:1066700001CA60919A0470919B0480E090E00E94AE
:106680006D7D67E773E00E94827D0097B1F46091B1
:106690009A0470919B0480E090E00E946D7D0097C9
:1066A00009F498C00E94647C803108F093C09091F6
:1066B0005201982B909352018DC08091520100D0CD
:1066C00000D025E135E0EDB7FEB73283218390E0BD
:1066D0008F709070948383830E94037E0F900F903D
:1066E0000F900F900E94D90C75C060919A04709120
:1066F0009B0480E090E00E946D7D8C0163EF72E06E
:106700000E94827D009741F40E94CE528091B20493
:106710009091B304906122C0C80166EF72E00E94BC
:10672000827D009741F5F8940E94DC5288E10FB613
:10673000F89480936000109260000FBE84B7877F4A
:1067400084BF809160008861809360001092600037
:1067500078948091B2049091B3049F7E9093B30497
:106760008093B20482EB94E064E170E042E050E098
:106770000E944C7F2FC0C8016CE773E00E94827DAD
:106780009C018091B2049091B3042115310521F44C
:1067900094FF20C0F894FFCF94FF03C083EF92E0F2
:1067A00002C086EF92E000D000D022E235E0ADB723
:1067B000BEB712963C932E93119714969C938E938A
:1067C00013970E94037E0F900F900F900F9002C0BE
:1067D0000E948B19E981FA811182108283E00F9067
:1067E0000F90CF91DF911F910F91FF90EF90DF906D
:1067F000CF90BF90AF909F908F907F906F905F9061
:106800004F903F902F900895F89491E2E0E0F0E0EF
:10681000909357008491E2E0F0E090935700249128
:10682000E4E0F0E090935700E49190E0A0E0B0E065
:10683000DC019927882730E040E050E0542F432FB7
:10684000322F2227820F931FA41FB51F8E0F911D79
:10685000A11DB11D80930C1890930D18A0930E18D4
:10686000B0930F1878940895DF93CF93CDB7DEB728
:1068700027970FB6F894DEBF0FBECDBFCE010496AA
:106880006EE070E044E050E00E942E7F8C819D819C
:10689000AE81BF818F3F2FEF92072FEFA2072FEF1F
:1068A000B20749F48CEA94E06EE070E044E050E016
:1068B0000E944C7F08C08093AC049093AD04A093D9
:1068C000AE04B093AF04CE01029662E170E042E004
:1068D00050E00E942E7F8A819B812FEF8F3F92078D
:1068E00079F48CE390E09093B1048093B00480EB52
:1068F00094E062E170E042E050E00E944C7F04C00E
:106900009093B1048093B004CE01029664E170E0EC
:1069100042E050E00E942E7F8A819B812FEF8F3FC3
:10692000920779F48AE090E09093B3048093B204E4
:1069300082EB94E064E170E042E050E00E944C7F22
:1069400004C09093B3048093B204CE01029660E039
:1069500070E042E050E00E942E7F8A819B812FEF01
:106960008F3F920769F41092C9061092C80688EC0E
:1069700096E060E070E042E050E00E944C7F04C08E
:106980009093C9068093C80685EC94E268E170E0B4
:1069900049E050E00E942E7F0E948F0ECE010496A7
:1069A00066E070E044E050E00E942E7F8C819D8183
:1069B000AE81BF818F3F2FEF92072FEFA2072FEFFE
:1069C000B20749F48DE894E066E070E044E050E0FE
:1069D0000E944C7F08C08DE894E066E070E044E0DF
:1069E00050E00E942E7FCE0104966AE070E044E001
:1069F00050E00E942E7F8C819D81AE81BF818F3FB0
:106A00002FEF92072FEFA2072FEFB20749F481E98A
:106A100094E06AE070E044E050E00E944C7F08C0DF
:106A200081E994E06AE070E044E050E00E942E7F4B
:106A3000CE01049662E070E044E050E00E942E7FB8
:106A40008C819D81AE81BF818F3F2FEF92072FEF09
:106A5000A2072FEFB20749F489E894E062E070E002
:106A600044E050E00E944C7F08C089E894E062E076
:106A700070E044E050E00E942E7FCE01019666E176
:106A800070E041E050E00E942E7F89818F3F49F401
:106A90008DEC96E066E170E041E050E00E944C7FB2
:106AA00008C08DEC96E066E170E041E050E00E94A5
:106AB0002E7FCE01019667E170E041E050E00E9438
:106AC0002E7F89818F3F49F484EB94E067E170E089
:106AD00041E050E00E944C7F08C084EB94E067E105
:106AE00070E041E050E00E942E7F27960FB6F894A8
:106AF000DEBF0FBECDBFCF91DF9108950E94C2527D
:106B00006C9A6B9A6A9A6F9A729A749A739A779A35
:106B1000809880B3897F80BB8398849887E0809336
:106B20007E00549A0E9404340E94343481E00E9412
:106B3000EC0A80E090E00E94A30E0E944B4C8091F2
:106B4000B20486FD239A0895CF93DF93EC018881E8
:106B50009981009731F02AE08B3D920709F099C0A6
:106B60008FC00E947E358091B20480FD06C081FFF7
:106B700002C01D9902C00E94EC53809170008C7F6E
:106B8000809370008091B60080628093B60010926E
:106B9000B20082E08093B1008091B60090E08770EF
:106BA00090700097C9F780917000816080937000A9
:106BB00080E090E06CEB78E00E94A5520E948E1A73
:106BC00080E00E941E1C00D08AEE91E0ADB7BEB7F7
:106BD00012969C938E9311970E94037E0F900F90B4
:106BE0000E94ED108091591C86FF02C00E94884DC2
:106BF0008091CD0690E00E9433578091B40490E0DC
:106C00000E94AB550E94A8558093FB068091B40466
:106C100090E00E94AB5500D000D000D0EDB7FEB799
:106C2000319681E893E0ADB7BEB712969C938E93F0
:106C300011978091FB06828313828091CD06848315
:106C400015820E94F17D1092FA061092F906EDB7B6
:106C5000FEB736960FB6F894FEBF0FBEEDBF81ECBF
:106C600094E09093CF248093CE2483E290E090939D
:106C7000F2068093F1068BED9AE0998388830DC02C
:106C8000633259F489EF96E060E070E00E944C2294
:106C9000E6CF1982188283E001C081E0DF91CF91B5
:106CA00008958536910564F12091C8063091C90692
:106CB00020FF10C000D000D023E933E0EDB7FEB7CD
:106CC00032832183948383830E94F17D0F900F9000
:106CD0000F900F9080916B2090916C20A0916D206F
:106CE000B0916E200196A11DB11D80936B209093F1
:106CF0006C20A0936D20B0936E2021E030E002C0A4
:106D000020E030E0C90108954F925F926F927F9228
:106D10008F929F92AF92BF92CF92DF92EF92FF92AB
:106D20000F931F93DF93CF93CDB7DEB7CB58D040EF
:106D30000FB6F894DEBF0FBECDBF2C01633871F4DF
:106D400089ED96E0C557DF4F6883CB58D0400E944D
:106D5000023FC557DF4F6881CB58D040D2012D91FB
:106D60003C911197BAE02E383B0709F469C7EAE075
:106D70002F383E0748F42115310589F0F9E02E3807
:106D80003F0709F0A9C716C04AE02F39340709F4B4
:106D90007DC75AE0263A350709F09EC78FC789EDAF
:106DA00096E061E870E04EE355E00E94E73E8EE831
:106DB00099E041C7623109F095C78091B204909182
:106DC000B30491FDF4CF8091AC049091AD04A091F7
:106DD000AE04B091AF0497FD8C9A0E94FD0B809198
:106DE000AC049091AD04A091AE04B091AF0493FFB8
:106DF00002C00E9467188091AC049091AD04A091EC
:106E0000AE04B091AF0494FF0AC00E94C60B609319
:106E1000B8247093B9248093BA249093BB248091B2
:106E2000AC0480FF5DC042E1C42ED12CCC0EDD1E2F
:106E300000D000D000D0EDB7FEB73196ADB7BEB7E9
:106E40001296DC92CE92119788E790E0938382832A
:106E500087EA93E0958384830E945A7E082F192F36
:106E600035ECE32E34E2F32EEDB7FEB736960FB6CF
:106E7000F894FEBF0FBEEDBF28E7A22EB12C9FE80D
:106E8000892E92E0992ED7012D917D01EDB7FEB7A5
:106E900038970FB6F894FEBF0FBEEDBF3196C6010E
:106EA000800F911FADB7BEB712969C938E9311972A
:106EB000B382A28295828482268317820E945A7EA0
:106EC000080F191FEDB7FEB738960FB6F894FEBF3E
:106ED0000FBEEDBFFDECEF16F4E2FF06A1F602C017
:106EE00000E010E08091AC0481FF6EC082E1C82E0A
:106EF000D12CCC0EDD1E00D000D000D0EDB7FEB7F7
:106F00003196C601800F911FADB7BEB712969C9304
:106F10008E93119788E790E0938382838BEA93E0C6
:106F2000958384830E945A7E080F191F7E0108945E
:106F3000E11CF11C80E1F70111928A95E9F72DB768
:106F40003EB72A5F3F4F0FB6F8943EBF0FBE2DBF2E
:106F500080EB68E9A70128E00E940212B9E0AB2E9D
:106F6000B12CAC0EBD1EA8E78A2E912CFFE86F2E27
:106F7000F2E07F2ED7012D917D01EDB7FEB7389756
:106F80000FB6F894FEBF0FBEEDBF3196C601800F5D
:106F9000911FADB7BEB712969C938E9311979382B3
:106FA000828275826482268317820E945A7E080F2D
:106FB000191FEDB7FEB738960FB6F894FEBF0FBE97
:106FC000EDBFEA14FB04B1F68091AC049091AD04DE
:106FD000A091AE04B091AF040097A105B10581F175
:106FE0002DB73EB7285030400FB6F8943EBF0FBEC5
:106FF0002DBFEDB7FEB73196CE014296800F911F9F
:10700000ADB7BEB712969C938E93119788E790E028
:107010009383828380EB93E0958384838091CB0676
:107020009091CC06978386830E945A7E080F191F81
:10703000EDB7FEB738960FB6F894FEBF0FBEEDBFA2
:107040008091AC0482FF50C089E290E06BE270E076
:107050004AE250E027E00E94614985EC94E20E94F8
:10706000D14B2DB73EB72A5030400FB6F8943EBFF3
:107070000FBE2DBFEDB6FEB60894E11CF11C9E01BB
:107080002E5E3F4F200F311FADB7BEB712963C9317
:107090002E93119728E730E0F7013383228327EB03
:1070A00033E0358324839C01B901882777FD8095DF
:1070B000982F0E94BF7720E030E048EC52E40E9415
:1070C0005577D70116966D937D938D939C93199761
:1070D0000E945A7E080F191FEDB7FEB73A960FB6F9
:1070E000F894FEBF0FBEEDBF8091AC0483FF56C085
:1070F00089E290E06BE270E04AE250E026E00E9414
:10710000614981E090E00E944D0C8093CF0684ECB1
:1071100097E10E94D14B2DB73EB72A5030400FB6B1
:10712000F8943EBF0FBE2DBFEDB6FEB60894E11C2D
:10713000F11C9E012E5E3F4F200F311FADB7BEB731
:1071400012963C932E93119728E730E0F701338392
:10715000228321EC33E0358324839C01B901882705
:1071600077FD8095982F0E94BF7720E030E048ECB3
:1071700052E40E945577D70116966D937D938D93B7
:107180009C9319970E945A7E080F191FEDB7FEB7FE
:107190003A960FB6F894FEBF0FBEEDBF8091AC04D7
:1071A00084FF36C02DB73EB72A5030400FB6F89452
:1071B0003EBF0FBE2DBFEDB7FEB73196CE01429652
:1071C000800F911FADB7BEB712969C938E93119707
:1071D00088E790E0938382838CEC93E095838483AB
:1071E00080918C1790918D17A0918E17B0918F1769
:1071F00086839783A087B1870E945A7E080F191F44
:10720000EDB7FEB73A960FB6F894FEBF0FBEEDBFCE
:107210008091AC0485FF31C00E94DA0B2DB73EB7D8
:107220002A5030400FB6F8943EBF0FBE2DBFEDB7C9
:10723000FEB731969E012E5E3F4F200F311FADB736
:10724000BEB712963C932E93119728E730E0338314
:1072500022832AED33E03583248366837783808716
:1072600091870E945A7E080F191FEDB7FEB73A9614
:107270000FB6F894FEBF0FBEEDBF8091AC0486FF41
:107280003AC0F8948091B0249091B124A091B22496
:10729000B091B32478942DB73EB72A5030400FB642
:1072A000F8943EBF0FBE2DBF4DB75EB74F5F5F4F27
:1072B0009E012E5E3F4F200F311FEDB7FEB7328388
:1072C000218328E730E0FA013383228328EE33E07C
:1072D0003583248386839783A087B1870E945A7E53
:1072E000080F191F2DB73EB7265F3F4F0FB6F89412
:1072F0003EBF0FBE2DBF8091AC0487FF92C080912E
:10730000B0049091B104009709F48BC0F894C09038
:10731000B024D090B124E090B224F090B3247894BB
:107320008091BC179091BD17A091BE17B091BF1767
:10733000A7019601281B390B4A0B5B0BCA01B90147
:107340000E94BD77862EA72E682EB92E6091B004BC
:107350007091B10480E090E00E94BD779B01AC0188
:10736000682D7A2D862D9B2D0E9455775C014DB797
:107370005EB74A5050400FB6F8945EBF0FBE4DBF87
:10738000EDB7FEB73196CE014296800F911FADB793
:10739000BEB712969C938E93119788E790E09383E3
:1073A000828381EF93E095838483262F372F4A2DA4
:1073B0005B2D2683378340875187C557DF4F68830E
:1073C000CB58D040C657DF4F7883CA58D0400E9470
:1073D0005A7E080F191FC557DF4F6881CB58D04020
:1073E000C657DF4F7881CA58D040862F972FAA2DD5
:1073F000BB2D8093BD249093BE24A093BF24B09353
:10740000C024C092BC17D092BD17E092BE17F09274
:10741000BF17EDB7FEB73A960FB6F894FEBF0FBE92
:10742000EDBF8091AC049091AD04A091AE04B091F9
:10743000AF0490FF40C0F8948091B4249091B5249B
:10744000A091B624B091B72478942DB73EB72A50B6
:1074500030400FB6F8943EBF0FBE2DBF4DB75EB79C
:107460004F5F5F4F9E012E5E3F4F200F311FEDB7E4
:10747000FEB73283218328E730E0FA013383228389
:107480002EEF33E03583248386839783A087B187EB
:107490000E945A7E080F191F2DB73EB7265F3F4F37
:1074A0000FB6F8943EBF0FBE2DBFC8010E945136E3
:1074B000009709F07CCC8091AC049091AD04A09130
:1074C000AE04B091AF0491FF92C08091B00490914E
:1074D000B104009709F48BC0F894C090B424D09004
:1074E000B524E090B624F090B72478948091C0172A
:1074F0009091C117A091C217B091C317A70196012F
:10750000281B390B4A0B5B0BCA01B9010E94BD77DE
:10751000862EA72E682EB92E6091B0047091B1040A
:1075200080E090E00E94BD779B01AC01682D7A2D30
:10753000862D9B2D0E9455775C014DB75EB74A5052
:1075400050400FB6F8945EBF0FBE4DBFEDB7FEB70B
:107550003196CE014296800F911FADB7BEB71296FD
:107560009C938E93119788E790E09383828387E0C2
:1075700094E095838483262F372F4A2D5B2D268315
:10758000378340875187C557DF4F6883CB58D0403A
:10759000C657DF4F7883CA58D0400E945A7E080FE2
:1075A000191FC557DF4F6881CB58D040C657DF4FF2
:1075B0007881CA58D040862F972FAA2DBB2D809353
:1075C000C1249093C224A093C324B093C424C09236
:1075D000C017D092C117E092C217F092C317EDB74F
:1075E000FEB73A960FB6F894FEBF0FBEEDBF80917E
:1075F000AC049091AD04A091AE04B091AF0492FFA1
:107600003EC080915B2090915C20A0915D20B09164
:107610005E202DB73EB72A5030400FB6F8943EBFDB
:107620000FBE2DBF4DB75EB74F5F5F4F9E012E5E01
:107630003F4F200F311FEDB7FEB73283218328E77C
:1076400030E0FA013383228324E134E0358324835C
:1076500086839783A087B1870E945A7E080F191FDF
:107660002DB73EB7265F3F4F0FB6F8943EBF0FBE13
:107670002DBFC8010E945136009709F098CB809128
:10768000AC049091AD04A091AE04B091AF0493FF0F
:107690003CC04DB75EB74A5050400FB6F8945EBF3D
:1076A0000FBE4DBFEDB7FEB73196CE014296800FAB
:1076B000911FADB7BEB712969C938E93119788E732
:1076C00090E0938382838DE194E09583848380911D
:1076D000551890915618A0915718B0915818868354
:1076E0009783A087B1870E945A7E080F191FEDB7B4
:1076F000FEB73A960FB6F894FEBF0FBEEDBFC801B5
:107700000E945136009709F052CB8091AC049091C1
:10771000AD04A091AE04B091AF0494FF3CC02DB76E
:107720003EB72A5030400FB6F8943EBF0FBE2DBF73
:10773000EDB7FEB73196CE014296800F911FADB7DF
:10774000BEB712969C938E93119788E790E093832F
:10775000828388E294E0958384838091B824909119
:10776000B924A091BA24B091BB2486839783A087C3
:10777000B1870E945A7E080F191FEDB7FEB73A96DF
:107780000FB6F894FEBF0FBEEDBFC8010E94513680
:10779000009709F00CCB8091AC049091AD04A091BE
:1077A000AE04B091AF0495FF48C081E00E94780B11
:1077B0002DB73EB72A5030400FB6F8943EBF0FBEEB
:1077C0002DBFEDB6FEB60894E11CF11C9E012E5EA5
:1077D0003F4F200F311FADB7BEB712963C932E938B
:1077E000119728E730E0F7013383228325E334E063
:1077F0003583248320918D0430918E0440918F0431
:10780000509190040E949B78D70116966D937D93BA
:107810008D939C9319970E945A7E080F191FEDB7FC
:10782000FEB73A960FB6F894FEBF0FBEEDBFC80183
:107830000E945136009709F0BACA8091AC04909129
:10784000AD04A091AE04B091AF0496FF48C082E0B1
:107850000E94780B2DB73EB72A5030400FB6F894EF
:107860003EBF0FBE2DBFEDB6FEB60894E11CF11C65
:107870009E012E5E3F4F200F311FADB7BEB712964F
:107880003C932E93119728E730E0F701338322834E
:1078900022E434E0358324832091910430919204D2
:1078A00040919304509194040E949B78D7011696BE
:1078B0006D937D938D939C9319970E945A7E080F28
:1078C000191FEDB7FEB73A960FB6F894FEBF0FBE7C
:1078D000EDBFC8010E945136009709F068CA809137
:1078E000AC049091AD04A091AE04B091AF0497FFA9
:1078F00039C083E00E94780B2DB73EB72A50304044
:107900000FB6F8943EBF0FBE2DBFEDB7FEB7319650
:107910009E012E5E3F4F200F311FADB7BEB71296AE
:107920003C932E93119728E730E0338322832FE492
:1079300034E03583248366837783808791870E9430
:107940005A7E080F191F8C98EDB7FEB73A960FB6FE
:10795000F894FEBF0FBEEDBFC8010E9451360097DC
:1079600009F025CA8091AC049091AD04A091AE04B9
:10797000B091AF04A0FF06C083E061E046E020E0E4
:107980000E94E4138091AC049091AD04A091AE04E8
:10799000B091AF04A1FF06C083E061E046E021E0C2
:1079A0000E94E4138091AC049091AD04A091AE04C8
:1079B000B091AF04A0FF3CC02DB73EB72A50304075
:1079C0000FB6F8943EBF0FBE2DBFEDB7FEB7319690
:1079D000CE014296800F911FADB7BEB712969C9311
:1079E0008E93119788E790E0938382838CE594E0EF
:1079F0009583848380914C1890914D18A0914E18D6
:107A0000B0914F1886839783A087B1870E945A7ED2
:107A1000080F191FEDB7FEB73A960FB6F894FEBFE0
:107A20000FBEEDBFC8010E945136009709F0BFC9D3
:107A30008091AC049091AD04A091AE04B091AF04DC
:107A4000A1FF3CC02DB73EB72A5030400FB6F89486
:107A50003EBF0FBE2DBFEDB7FEB73196CE014296A9
:107A6000800F911FADB7BEB712969C938E9311975E
:107A700088E790E09383828384E694E0958384830F
:107A80008091501890915118A0915218B0915318AC
:107A900086839783A087B1870E945A7E080F191F9B
:107AA000EDB7FEB73A960FB6F894FEBF0FBEEDBF26
:107AB000C8010E945136009709F079C9779A8091E0
:107AC000C8069091C90692FD749A8091C80690915B
:107AD000C90682FD08C08091B20480FD04C081FF08
:107AE00031C01D9B2FC000D000D08FE694E0ADB711
:107AF000BEB712969C938E931197CE014296149620
:107B00009C938E9313970E94F17D209195040F9082
:107B10000F900F900F902223A9F000D000D0EDB766
:107B2000FEB7319684EE91E0ADB7BEB712969C9346
:107B30008E931197228313820E94037E0F900F90E1
:107B40000F900F908091EC06898BFE01E00FF11FE2
:107B5000128A0F5F1F4F8091C8069091C90680FF5F
:107B600012C000D000D086E794E0EDB7FEB7928354
:107B70008183C8010196948383830E94F17D0F90D5
:107B80000F900F900F9068010894C11CD11CE1E187
:107B9000EE2EF12CEC0EFD1EC701B6010E945F48CF
:107BA0008091B20482FF08C08CE994E0B701A6017D
:107BB00020EB30E20E94E44C8091C8069091C90607
:107BC00082FD73980E948A5489ED96E00E94053FD9
:107BD0008091B2049091B30490FF43C0E090B00450
:107BE000F090B1040E94A855C82E1092B1041092D2
:107BF000B00489E190E00E94C05524C07398809140
:107C0000EC068F5F8093EC06898BB8016F5F7F4F26
:107C1000CE0141960E945F4889ED96E00E94053FA3
:107C20008091820E9091830E65E840E050E00E94C2
:107C3000CB408EE89AE0D20111969C938E9352C06D
:107C400000E010E02091B2043091B30430FDD6CFB3
:107C50008C2D90E00E94C055F092B104E092B004E7
:107C6000739A8091CB069091CC06009711F00E94F8
:107C7000EC538091EC068F5F8093EC068091C806F0
:107C80009091C90682FF93C8739A91C884EE96E0DA
:107C90000E94AC43009731F10E948A548091B20453
:107CA00087FD2B9884EE96E060E470E00E948143AB
:107CB00086EA9AE0F2019183808314C084EE96E014
:107CC0000E94AC43009771F00E94EC538091B20483
:107CD00087FF6DC82B9A6BC8D20111961C921E9219
:107CE00083E001C081E0C557DF4F0FB6F894DEBFD7
:107CF0000FBECDBFCF91DF911F910F91FF90EF90FD
:107D0000DF90CF90BF90AF909F908F907F906F90BB
:107D10005F904F9008950E942F3F08950895FC01B1
:107D2000DB018C91808311968C911197818308954A
:107D3000FC01DB0190818C91981741F421E030E047
:107D4000918111968C911197981711F020E030E0F5
:107D5000C9010895FC0180818093D524818180939D
:107D6000D6240895DC011996ED91FC911A970280B2
:107D7000F381E02D309709F009950895EF92FF9275
:107D80000F931F93DF93CF9300D0CDB7DEB78C0155
:107D900088E10E94DA48BC017E010894E11CF11CD4
:107DA000C7010E948F3ED8011996ED91FC911A9758
:107DB0000190F081E02DC801B70109950F900F9057
:107DC000CF91DF911F910F91FF90EF900895EF9267
:107DD000FF920F931F93CF93DF93EC018B017A01F6
:107DE0004EE455E00E94133FFA86E986C80162E539
:107DF00075E00E94723FDF91CF911F910F91FF902C
:107E0000EF9008950E942C3F0895CF93DF93EC01EB
:107E100088E165ED74E20E94D048CE010E942F3FB8
:107E2000DF91CF910895EF92FF920F931F93CF931D
:107E3000DF93EC018B017A010E944B3FF886EF82C1
:107E4000C80166E575E00E94723FDF91CF911F91F6
:107E50000F91FF90EF9008950E94543F08950E9463
:107E6000615A0895FC01A781B0852D913C91F901DB
:107E700009950895DC011796ED91FC911897028001
:107E8000F381E02D309709F0099508958EE79EE083
:107E90000E94BE410895FC01738362838EE79EE0D9
:107EA000BF010E9449420895BC018EE79EE00E94F6
:107EB00010420895CF93DF93EC018EE79EE00E947D
:107EC000C24108C0828193818C179D0739F0CF0190
:107ED0000E948842E82FF92F3097A1F7CF01DF9158
:107EE000CF9108950F931F93CF93DF938B010E943F
:107EF0005A3FEC01009731F01D830C83C8010E94AA
:107F0000B95C8E83DF91CF911F910F9108951F93DC
:107F1000CF93DF93EC01162F888580FF1DC0EC8185
:107F2000FD813097C9F0D093830EC093820E82E01A
:107F30008887CE0106960995992787FD9095029727
:107F40008230910510F0133829F4CE01BE010E9451
:107F5000B03F02C081E08887DF91CF911F910895E3
:107F6000CF92DF92EF92FF920F931F93CF93DF9305
:107F7000EC017B01C090820ED090830E0091800EA8
:107F80001091810EF80103C00190F081E02DEC17F3
:107F9000FD0719F03097C1F746C0209709F443C098
:107FA0008885882309F118860BC0C017D10729F0EE
:107FB000C80167E8AE010E94873FF8010081118186
:107FC0000115110591F7EC81FD81309769F0CE150F
:107FD000DF0551F0D093830EC093820ECE0106963A
:107FE00063E840E050E00995E091800EF091810E49
:107FF000CE17DF0791F4888199819093810E809349
:10800000800E0DC0808191818C179D0729F4888195
:1080100099819183808303C0FC01309799F7D092B6
:10802000830EC092820EDF91CF911F910F91FF902E
:10803000EF90DF90CF9008951F93CF93DF9310922E
:10804000840EC091800ED091810E11E00EC0898502
:10805000882341F018871986CE0162E840E050E09D
:108060000E94873F0990D881C02D209781F7DF912A
:10807000CF911F91089580912F0F982F9F5F90931C
:108080002F0F08956091820E7091830E0E94B03F71
:1080900008958AE880932F0F1092860E1092850E15
:1080A0001092810E1092800E1092830E1092820E0A
:1080B00008958091840E882311F00E941C407091D5
:1080C000850E772309F455C02091860E30E0F90122
:1080D000EE0FFF1FEE0FFF1FE20FF31FE957F14FE7
:1080E000608160932E0F4181528150932D0F4093F8
:1080F0002C0F8381948190932B0F80932A0F2F5FF5
:108100003F4F2F7130702093860E71507093850E03
:10811000009741F58091800E9091810E18C080915A
:10812000840E882311F00E941C4040912C0F509126
:108130002D0F8091280F9091290F60912E0F0E9492
:10814000873FE091280FF091290F808191819093D2
:10815000290F8093280F8091280F9091290F009765
:10816000F1F607C0613819F421E0FC0120870E9474
:10817000873F8091840E2091850E30E0280F311DBD
:10818000C90108958091840E2091850E30E0280F5A
:10819000311DC90108957091850E7032D9F020917A
:1081A000860E270F2F712093270F30E0F901EE0F75
:1081B000FF1FEE0FFF1FE20FF31FE957F14F608320
:1081C00052834183948383837F5F7093850E20E085
:1081D00030E002C021E030E0C9010895CF93DF9381
:1081E000C091820ED091830E0E94873FD093830E60
:1081F000C093820EDF91CF910895FC01AB01909165
:10820000800E8091810E9C01A32FB22F03C00D9090
:10821000BC91A02DAE17BF0791F01097C1F7309712
:1082200071F090838183F093810EE093800E81E062
:10823000808717821682CF0161E80E94EE40089580
:10824000FC01009741F080858150823020F481E06C
:1082500081878093840E089521E030E0FC018085C1
:10826000882311F420E030E0C9010895CF93DF9313
:10827000EC014A815B818C819D8160E070E00E940D
:108280007B7D4A815B8188819981489F9001499FCC
:10829000300D589F300D11248E819F8160E070E079
:1082A000A9010E947B7DDF91CF910895FC0182811D
:1082B000938120E030E019C0A481B581A20FB31FE3
:1082C0004C91442381F481E08C9340815181249F1F
:1082D000C001259F900D349F900D11242681378178
:1082E000280F391F07C02F5F3F4F2817390720F38A
:1082F00020E030E0C9010895FC01268137814281E8
:10830000538180E090E018C02617370781F4A481DC
:10831000B581A80FB91F2C91121614F421502C937B
:108320000480F581E02DE80FF91F80810895A08178
:10833000B1812A0F3B1F01968417950728F38FEF11
:108340000895FC01CB01268137816217730790F0F5
:10835000A081B18162817381A69FA001A79F500D6A
:10836000B69F500D1124420F531F21E030E08417B7
:10837000950710F020E030E0C9010895FC0111825A
:1083800010820895FC01808191810895FB01208174
:108390003181FC01318320830895FC0120813181EA
:1083A0002115310511F407C09C01F90180819181EB
:1083B0000097D1F702C020E030E0C9010895CF93C3
:1083C000DF93DC012D913C91119721153105A9F026
:1083D000F90180819181009729F411961C921E92D7
:1083E0000EC0F90120813181D9018D919C911197A5
:1083F0000097B9F71182108202C020E030E0C90175
:10840000DF91CF910895DC01ED91FC9111973097A8
:1084100029F08081918111969C938E93CF010895CC
:10842000CF93DF93FC01A081B1811097D9F0C0E018
:10843000D0E016C0A617B70771F48D919C911197E3
:10844000209719F49183808302C0998388831196C1
:108450001C921E9207C0ED0198818981A92FB82F27
:10846000109741F7DF91CF9108950F931F93CF930A
:10847000DF938C01EB010E941042F8018081918111
:1084800099838883D183C083DF91CF911F910F910E
:108490000895EF92FF920F931F93CF93DF93EC0118
:1084A0007B010E941042F70111821082CE010E94CE
:1084B000CD41FC01009719F4E882F98202C0F182F3
:1084C000E082DF91CF911F910F91FF90EF9008957F
:1084D000DC01ED91FC91119720E030E005C02F5FA9
:1084E0003F4F0190F081E02D3097C9F7C901089501
:1084F000FB01309721F4BA010E9435420895DA0158
:108500008081918111969C938E935183408308952D
:10851000009721F0FC012081318102C020E030E091
:10852000C90108958091300F9091310F009729F47F
:108530001092330F1092320F08950E944E51E09125
:10854000300FF091310F2281338140815181240F0E
:10855000351F281B390B0CC042815381608171810A
:10856000460F571F481B590B4217530708F49A012F
:108570000480F581E02D309779F7280F391F30936B
:10858000330F2093320F089584E695E00E94204136
:108590000895CF92DF92EF92FF920F931F93CF93A4
:1085A000DF937C01FC0180819181009729F08A355D
:1085B000910509F06EC00BC01092310F1092300F70
:1085C0008AE590E0F7019183808381E066C0673897
:1085D00049F5CA01E091300FF091310F03C00480DA
:1085E000F581E02D309741F326813781281739072F
:1085F000B1F3E093300FF093310F0FC016962D9129
:108600003C9117972817390739F414962D913C910E
:10861000159735832483DF01FD01A481B58110976F
:1086200069F7CECF623861F6C091300FD091310F2B
:1086300000E010E02BC0CE010E94B1600097F1F085
:108640008E819F8168E8AE010E94CB400097A1F423
:108650001F821E828C819D810115110521F0F80178
:108660009583848304C09093310F8093300F1D82D3
:108670001C820E949242D8CF0E94C4428E019C81EB
:108680008D81C92EE6016E01D82EE601209799F65C
:1086900097CFF7011182108283E0DF91CF911F9174
:1086A0000F91FF90EF90DF90CF900895CF93DF93DD
:1086B000EC010E94C4428E819F81009769F0E09195
:1086C000300FF091310F06C0EC17FD07A9F00480C0
:1086D000F581E02D3097C1F78091820E9091830E45
:1086E0009F838E838091300F9091310F9D838C8377
:1086F000D093310FC093300F0E949242DF91CF91FF
:108700000895CF93DF93EC010E949160CE010E9407
:108710005643DF91CF910895CF93DF93EC010E94F0
:108720009D60CE010E945643DF91CF910895CF9373
:10873000DF93EC010E94A760CE010E945643DF91B7
:10874000CF910895FC0180819181860F971F9183BD
:1087500080830E949242089521E030E0FC018681EE
:108760009781009711F020E030E0C9010895FC01E5
:108770002281338180819181280F391FC901089599
:10878000FC0180819181089521E030E08091300FDB
:108790009091310F009711F420E030E0C901089565
:1087A0008091300F9091310F009729F02091320F76
:1087B0003091330F02C020E030E0C9010895CF931B
:1087C000DF93EC01E091300FF091310F8E179F078E
:1087D00041F48C819D819093310F8093300F14C0B0
:1087E000FC01309731F0848195818C179D07C1F78A
:1087F00007C01D821C821F821E82DF91CF910895C7
:108800008C819D81958384830E949242F2CFCF9286
:10881000DF92EF92FF920F931F93CF93DF938C0120
:108820007A01FC0180819181009729F08B349105B8
:1088300009F051C01EC085E39FE00E94C241C82ECE
:10884000E6017E01F92EE70109C06C817D81CE0130
:1088500002960E9481430990D881C02D2097A9F7E4
:1088600081E08093340F8BE490E0F8019183808362
:1088700037C06838A9F585E39FE00E94C241C82E41
:10888000E6016E01D92EE60123C0CE010296E8165C
:10889000F906D9F485E39FE0BE010E941042E09002
:1088A000820EF090830E8A859B859093830E809331
:1088B000820EEC85FD85309719F08E859F85099590
:1088C000F092830EE092820ECECF0990D881C02D17
:1088D0002097D9F6C8CFF8011182108283E001C039
:1088E00081E0DF91CF911F910F91FF90EF90DF908A
:1088F000CF9008951092340F85E39FE00E94BE410F
:108900008DE795E060E070E00E94FD4008950F93D0
:108910001F93CF93DF93EC010091820E1091830E91
:108920001B870A875D874C873F872E878091340F8E
:10893000882379F08DE795E09093830E8093820EE3
:10894000CE0102960E9481431093830E0093820E03
:1089500002C07D836C8385E39FE0BE010E941042CC
:1089600085E39FE0BE010E944942DF91CF911F91B4
:108970000F9108950F931F93CF93DF93EC01809194
:10898000340F882391F00091820E1091830E8DE7B1
:1089900095E09093830E8093820ECE0102960E9402
:1089A0008C431093830E0093820E85E39FE0BE01FB
:1089B0000E94104285E39FE0BE010E944942DF9180
:1089C000CF911F910F9108950F931F93CF93DF9332
:1089D000EC018091340F882391F00091820E109168
:1089E000830E8DE795E09093830E8093820ECE01E7
:1089F00002960E9497431093830E0093820E85E3A4
:108A00009FE0BE010E94104285E39FE0BE010E94EC
:108A10004942DF91CF911F910F910895CF93DF933A
:108A2000EC018091340F882329F0CE0102960E9438
:108A3000DF4304C01F821E821986188685E39FE0EB
:108A4000BE010E941042DF91CF910895CF93DF9332
:108A5000EC018091340F882331F0CE0102960E9400
:108A6000AC439C0114C085E39FE00E94C241E82F03
:108A7000F92F06C0EC17FD0741F00190F081E02DC1
:108A80003097C1F721E030E002C020E030E0C901BA
:108A9000DF91CF9108950F931F930091D5241091EA
:108AA000D6240E947B512DB73EB7225530400FB6D9
:108AB000F8943EBF0FBE2DBFEDB7FEB7319628EE3E
:108AC0003DE0ADB7BEB712963C932E93119702834B
:108AD00013821483158266837783808791878091C0
:108AE000C8269091C926A091CA26B091CB2682872C
:108AF0009387A487B5878091CC269091CD26A091AD
:108B0000CE26B091CF2686879787A08BB18B809198
:108B1000D0269091D126A091D226B091D326828BD7
:108B2000938BA48BB58B8091D4269091D526A09160
:108B3000D626B091D726868B978BA08FB18F809148
:108B4000D8269091D926A091DA26B091DB26828F83
:108B5000938FA48FB58F8091DC269091DD26A09114
:108B6000DE26B091DF26868F978FA0A3B1A38091D8
:108B7000E0269091E126A091E226B091E32682A31F
:108B800093A3A4A3B5A38091E4269091E526A09198
:108B9000E626B091E72686A397A3A0A7B1A7809168
:108BA000E8269091E926A091EA26B091EB2682A7CB
:108BB00093A7A4A7B5A78091EC269091ED26A0914C
:108BC000EE26B091EF2686A797A7A0ABB1AB809118
:108BD000F0269091F126A091F226B091F32682AB77
:108BE00093ABA4ABB5AB8091F4269091F526A09100
:108BF000F626B091F72686AB97ABA0AFB1AF8091C8
:108C0000F8269091F926A091FA26B091FB2682AF22
:108C100093AFA4AFB5AFEDB7FEB7FF968091FC263A
:108C20009091FD26A091FE26B091FF26808391832E
:108C3000A283B383EDB7FEB7ED5BFF4F80910027B2
:108C400090910127A0910227B091032780839183FF
:108C5000A283B383EDB7FEB7E95BFF4F8091042792
:108C600090910527A0910627B091072780839183D3
:108C7000A283B383EDB7FEB7E55BFF4F8091082772
:108C800090910927A0910A27B0910B2780839183A7
:108C9000A283B383EDB7FEB7E15BFF4F80910C2752
:108CA00090910D27A0910E27B0910F27808391837B
:108CB000A283B3830E94037E0091D5241091D62411
:108CC0002DB73EB72E5A3F4F0FB6F8943EBF0FBE9A
:108CD0002DBF0E947B51ADB7BEB7D2970FB6F894A7
:108CE000BEBF0FBEADBFEDB7FEB7319629E73DE081
:108CF00012963C932E93119702831382148315824C
:108D000066837783808791878091102790911127C0
:108D1000A0911227B091132782879387A487B587E4
:108D20008091142790911527A0911627B0911727AD
:108D300086879787A08BB18B8091182790911927F0
:108D4000A0911A27B0911B27828B938BA48BB58B94
:108D500080911C2790911D27A0911E27B0911F275D
:108D6000868B978BA08FB18F8091202790912127A0
:108D7000A0912227B0912327828F938FA48FB58F44
:108D80008091242790912527A0912627B09127270D
:108D9000868F978FA0A3B1A3809128279091292730
:108DA000A0912A27B0912B2782A393A3A4A3B5A3B4
:108DB00080912C2790912D27A0912E27B0912F27BD
:108DC00086A397A3A0A7B1A78091382790913927B0
:108DD000A0913A27B0913B2782A793A7A4A7B5A754
:108DE00080913C2790913D27A0913E27B0913F274D
:108DF00086A797A7A0ABB1AB0E94037E2DB73EB765
:108E00002E5C3F4F0FB6F8943EBF0FBE2DBF1F9193
:108E10000F91089580E38093370F0895EF92FF92AA
:108E2000CF93DF932091370F30E0C0E3D0E0C21B37
:108E3000D30B245C304FB901AE010E94727DCE018C
:108E4000DF91CF91FF90EF900895AF92BF92CF92B4
:108E5000DF92EF92FF920F931F93CF93DF937C01EA
:108E6000C090380FD090390F2091370F30E0860135
:108E7000005D1F4F021B130B01381105E0F4C0E326
:108E8000D0E0C21BD30B245C304FB901AE010E946D
:108E9000727DCE0DDF1D20913A0F30913B0F8091F6
:108EA000EE0F9091EF0F280F391FCE01B901A601E7
:108EB0000E94727D02C000E010E0C801DF91CF91F6
:108EC0001F910F91FF90EF90DF90CF90BF90AF90E8
:108ED00008959091370F980F9093370F0895409110
:108EE000380F5091390F9C014817590798F080911D
:108EF000EE0F9091EF0F820F931F9093EF0F8093DF
:108F0000EE0F421B530B5093390F4093380F21E063
:108F100030E002C020E030E0C90108959093390F9D
:108F20008093380F08952091EE0F3091EF0F245960
:108F3000304FC90108952091370F30E0245C304F45
:108F4000C901089521E030E080913A0F90913B0FE4
:108F50004FE08C36940711F420E030E0C901089509
:108F60000E94A247009771F02CE63FE060913A0F13
:108F700070913B0F4091380F5091390FC9010E94F9
:108F8000727D0895A091EE0FB091EF0F1097B9F098
:108F90002091380F3091390F205D3F4FA459B04FC9
:108FA000ECE6FFE080E390E003C04D914193019631
:108FB00082179307D4F31092EF0F1092EE0F0895DB
:108FC00080913A0F90913B0F08958091380F9091C6
:108FD000390F08959091370F80E3891B089580E33E
:108FE0009091370F891B2091380F3091390F280F3E
:108FF000311DC90108951F93CF93DF93EC011091A8
:10900000370F812F90E08C179D076CF00E94EF477F
:109010008C0F9D1F8138910530F41C1B1093370F66
:1090200021E030E002C020E030E0C901DF91CF91C3
:109030001F910895CF93DF93EFEDF4E21192119217
:1090400085E2EF30F807D1F7C0E0D0E0CE01880F1D
:10905000991F89529B4D6CE475E00E948F3E2196CA
:10906000C430D10599F7DF91CF9108951092EF0F99
:109070001092EE0F1092390F1092380F80E3809308
:10908000370F8CE69FE090933B0F80933A0F0E943E
:109090001A4808950F931F93CF93DF93EC018B0130
:1090A0000E943648D0933B0FC0933A0F1093390F6C
:1090B0000093380FDF91CF911F910F910895CF92B8
:1090C000DF92EF92FF920F931F93DF93CF9300D025
:1090D000CDB7DEB78C0169837A830E9436486981F7
:1090E0007A81C62ED72E21E8C216D10418F030E8B6
:1090F000C32ED12C80913A0F90913B0FB801A6015D
:109100000E94727DD092390FC092380FC6010F9025
:109110000F90CF91DF911F910F91FF90EF90DF9013
:10912000CF900895282F392FD901EFEDF4E280E395
:1091300001900D928150E1F7862F972FDC01E7ED2A
:10914000F4E288E001900D928150E1F70895EFED8F
:10915000F4E2282F392FD90180E30D90019281503C
:10916000E1F7A7EDB4E2862F972FFC0188E001908C
:109170000D928150E1F70895E82FF0E0EE0FFF1F08
:10918000E152FB4D7183608381E090E00895E82F08
:10919000F0E0EE0FFF1FE152FB4D808191810895B9
:1091A00090E0880F991F89559B4D0E948F3E81E06A
:1091B00090E00895282F30E0220F331F29553B4DB2
:1091C000C90108958115910511F00197F1F70895EE
:1091D000E0911225F091132590818091112589232A
:1091E0000895E0910F25F09110258081909111252F
:1091F000892B8083E0911425F09115258081909131
:109200001125892B80830895E0910F25F091102579
:10921000908180911125809589238083E091142588
:10922000F091152590818091112580958923808367
:109230000895FF920F931F93E0910F25F091102551
:10924000908180911125809589238083E091142558
:10925000F0911525808190911125892B80838FEBCA
:1092600093E00E94E248FFB6F894E0911425F09153
:10927000152590818091112580958923808383E82D
:1092800090E00E94E248E0911225F09113250081C0
:1092900010911125FFBE78948BE393E00E94E24881
:1092A000E0911225F0911325808190911125892359
:1092B00019F0802F812301C081E01F910F91FF9051
:1092C00008955093152540931425709310256093AD
:1092D0000F25909313258093122581E090E002C022
:1092E000880F991F2A95E2F7809311250E9419494A
:1092F00008950F931F93182F0FB7F894E09114253A
:10930000F0911525808190911125892B808383E030
:1093100090E00E94E248112351F0E0911425F09171
:10932000152590818091112580958923808387E17F
:1093300090E00E94E248E0911225F091132580818F
:1093400090911125892309F410E089E590E00E94AD
:10935000E248E0911425F091152590818091112526
:109360008095892380830FBF8BE390E00E94E248C1
:10937000812F1F910F9108950F931F93182F08E0CD
:10938000812F81700E9479491695811110680150D2
:10939000B9F7812F1F910F9108958FEF0E94BC495B
:1093A0000895DF92EF92FF920F931F93CF93DF9375
:1093B000182FEB010E941949882389F580EF0E943C
:1093C000BC49EE2400E498EFD92ED00E81E00E9433
:1093D0007949F82E81E00E947949882319F0FF200D
:1093E00069F020C0FF2051F4011728F0888180FF28
:1093F00005C0101719F0E02EFF24F3948F2D0E9462
:109400007949888186958883FF2011F08068888358
:1094100001500D15D9F6002339F02196D4CFEE2452
:10942000EA9402C08EEFE82E8E2DDF91CF911F912E
:109430000F91FF90EF90DF9008950F931F93CF93BC
:10944000DF93182FEB010E941949209751F085E511
:109450000E94BC4908E089910E94BC490150D9F79B
:1094600003C08CEC0E94BC49812F0E94BC49DF9153
:10947000CF911F910F9108950F931F93CF93DF9377
:10948000FB01DA01E801408150E0718160E0462B88
:10949000572B803171F4BA016E7F13E0660F771F8E
:1094A0001A95E1F796814CE050E0491B5109460FAF
:1094B000571F57FF06C091E09C93509541955F4F11
:1094C00001C01C92883289F4848190E0BC016076EE
:1094D00070706036710549F086FF02C04E7F05C08E
:1094E00085FF02C04C7F01C0487FCA0154E09695B9
:1094F00087955A95E1F7F90180834F70488380E0A2
:10950000DF91CF911F910F9108950F931F93CF93E8
:10951000DF938C01EB01F8018081BE010E94D149EB
:10952000F801808381508D3F28F48881883211F0C2
:10953000803189F7DF91CF911F910F9108951F938B
:10954000CF93DF93EC010E94194984EBBE010E9486
:109550001D4A81E00E947949182F0E94194981E033
:10956000112309F480E0DF91CF911F9108951F939B
:10957000CF93DF93182FEB010E9419490E94E8480E
:10958000882349F084E4BE010E941D4A113029F06D
:109590000E94F14802C082E001C080E0DF91CF91DB
:1095A0001F9108956F927F928F929F92AF92BF9278
:1095B000CF92DF92EF92FF920F931F93DF93CF939F
:1095C000CDB7DEB729970FB6F894DEBF0FBECDBF7B
:1095D0007C014B013A0159010E9419498EEBB701F8
:1095E0000E941D4A8E010F5F1F4F8AE0C82ED12CAA
:1095F000CC0EDD1E0E94CD49F80181938F01EC1540
:10960000FD05C1F78E010F5F1F4FC80169E070E0D3
:109610000E946265882351F4F7018081B801A4019A
:10962000930185010E943C4A80E001C083E02996B5
:109630000FB6F894DEBF0FBECDBFCF91DF911F9163
:109640000F91FF90EF90DF90CF90BF90AF909F90E1
:109650008F907F906F9008957F928F929F92AF929C
:10966000BF92CF92DF92EF92FF920F931F93DF93FF
:10967000CF93CDB7DEB729970FB6F894DEBF0FBEF4
:10968000CDBF782E5B014A0179018EEB60E070E07E
:109690000E941D4A8E010F5F1F4F9AE0C92ED12CE8
:1096A000CC0EDD1E0E94CD49F80181938F01EC158F
:1096B000FD05C1F78E010F5F1F4FC80169E070E023
:1096C0000E946265882349F4872DB801A5019401A1
:1096D00087010E943C4A80E001C083E029960FB6D2
:1096E000F894DEBF0FBECDBFCF91DF911F910F91D8
:1096F000FF90EF90DF90CF90BF90AF909F908F90B2
:109700007F9008950F931F93DF93CF93CDB7DEB76C
:1097100028970FB6F894DEBF0FBECDBF182F062FC7
:10972000DE011196EFE8F5E088E001900D9281509E
:10973000E1F7242F332727FD309541E752E0249F9E
:10974000C001259F900D349F900D112464E670E0B8
:109750000E946D7AAB0164E6069FB0011124460FAA
:10976000571FFE013196CE010996619170E02617D0
:10977000370719F44F5F5F4F03C0E817F907A9F7E0
:10978000112319F0509541955F4FCA0128960FB6E5
:10979000F894DEBF0FBECDBFCF91DF911F910F9127
:1097A00008950F931F93DF93CF93CDB7DEB72B9719
:1097B0000FB6F894DEBF0FBECDBF182F092F885FFC
:1097C000612F792F0E94B74A882309F049C066E4C7
:1097D00071E48FE090E00E943E4C812F902FBE01FB
:1097E0006F5F7F4FAE014E5F5F4F9E012D5F3F4F1A
:1097F0000E94D24A8823A1F5DE011496E7E8F5E03D
:1098000088E001900D928150E1F74B81642F70E068
:1098100021E732E0629FC001639F900D729F900D1F
:10982000112464E670E00E946D7A9A8184E6989F24
:10983000C0011124680F791FFE013496CE010C96E9
:109840002191421719F46F5F7F4F03C0E817F907A2
:10985000B9F78981882331F0709561957F4F02C0F7
:1098600064E371E2CB012B960FB6F894DEBF0FBE16
:10987000CDBFCF91DF911F910F910895DC01CB01F6
:1098800081159105A105B10529F081509040A040B6
:10989000B040D9F708951092B90080E28093B800E3
:1098A000089594EA9093BC0020EA36E841E050E045
:1098B00005C02150304040405040F1F09091BC0034
:1098C00097FFF7CF1DC09031B9F48093BB0084E8B7
:1098D0008093BC0080EA96E8A1E0B0E004C0019764
:1098E000A109B10959F02091BC0027FFF8CF0EC0A3
:1098F00081E0903421F40FC081E0089581E0089563
:109900009091B900987F9830F1F6DFCF9091B9002F
:10991000987F983169F780E0089544EA34E824E9B3
:109920004093BC009091BC0097FFFCCF9091B90090
:10993000987F983011F0903199F78093BB00309365
:10994000BC009091BC0097FFFCCF9091B900987F2C
:10995000903211F0983539F42093BC009091BC00FE
:1099600094FDFCCFDDCF08950E94514C089584E909
:109970008093BC008091BC0084FDFCCF089580934F
:10998000BB0084E88093BC008091BC0087FFFCCFC3
:109990009091B900987F81E0983209F480E00895B1
:1099A00084EC8093BC008091BC0087FFFCCF809149
:1099B000BB00089584E88093BC008091BC0087FFC1
:1099C000FCCF8091BB000895E82FF92F80E19191A1
:1099D00090933F018150D9F780913C018F7D809316
:1099E0003C0180913C01877F80933C01862F972F1B
:1099F000FC0180E1919190933E018150D9F78091D3
:109A00003C01806880933C0180913D0180FFFCCF48
:109A10004051504080913C01806280933C01809194
:109A20003C01877F80933C0114C0862F972FFC0157
:109A300080E1919190933E018150D9F780913C0152
:109A4000806880933C0180913D0180FFFCCF4051B4
:109A50005040141615064CF3822F932FFC0180E121
:109A600090913E0191938150D9F781E090E0089563
:109A70000F931F93CF93DF938C018CE70E948D4C43
:109A80008CE70E94BF4CC0E0D0E0F80181918F01CB
:109A90000E94BF4C2196C031D105B9F70E94B74C46
:109AA000DF91CF911F910F910895813039F48CE7A8
:109AB00090E060E070E040E050E006C08CE790E0AD
:109AC00060E070E040EC50E00E94EA1108958130BF
:109AD00039F48CE790E060E070E04EE050E006C0C2
:109AE0008CE790E060E070E048E050E00E94EA110E
:109AF00008958CE790E060E070E041E050E00E9463
:109B0000EA116AE67AE080E090E00E943E4C089517
:109B10008CE790E060E070E048E350E00E94EA11DA
:109B20008CE790E060E070E049E350E00E94EA11C9
:109B30008CE790E060E070E044E150E00E94EA11C0
:109B40008CE790E060E070E048E750E00E94EA11A6
:109B50008CE790E060E070E04EE550E00E94EA1192
:109B60008CE790E060E070E04DE650E00E94EA1182
:109B70006CE17AE186E090E00E943E4C8CE790E058
:109B800060E070E04CE050E00E94EA118CE790E069
:109B900060E070E041E050E00E94EA118CE790E064
:109BA00060E070E046E050E00E94EA116AE67AE088
:109BB00080E090E00E943E4C0895DF93CF93CDB7B4
:109BC000DEB7A2970FB6F894DEBF0FBECDBFDE01A1
:109BD0001196E7E9F5E081E101900D928150E1F7FE
:109BE000DE015296E8EAF5E081E101900D928150A4
:109BF000E1F70E94884DCE0101960E94384D82E027
:109C00000E94554D6AE67AE080E090E00E943E4C6A
:109C1000CE0142960E94384D60E17EEA88E290E0F3
:109C20000E943E4C80E00E94674D60E17EEA88E23F
:109C300090E00E943E4C81E00E94674DA2960FB6D4
:109C4000F894DEBF0FBECDBFCF91DF910895E6E45B
:109C5000F1E0808120819081308182958695869582
:109C6000837022952F70822B832B92959F70892B66
:109C70000895DF92EF92FF920F931F93DF93CF939C
:109C800000D0CDB7DEB780E06CE046E00E940F5216
:109C900089E18093C4001092C50082E08093C000E7
:109CA00080E00E94B9520E943E5184B784B784B7C5
:109CB00084B784B7E6E9FDE222E432E4318320830D
:109CC0003A968DB79EB70A97E817F907B8F300D010
:109CD00000D085E39FE0ADB7BEB712969C938E93FC
:109CE000119789EB95E014969C938E9313970E949D
:109CF000037E0F900F900F900F900E947B610E9447
:109D0000494084E695E060E070E00E94FD400E94DA
:109D10007A44E0910406F091050609950E94274EC9
:109D200090E00E94B961CE0101960E946C50882398
:109D300059F000D085E19FE0EDB7FEB792838183B3
:109D40000E94037E0F900F908E010F5F1F4FC8017E
:109D50000E94AA3E0E9476507C010E947B50BC016A
:109D6000C701A8010E94C6550E94D44F0E94AB555E
:109D70000E9480500E94335700D088E09FE0ADB72A
:109D8000BEB712969C938E9311970E94037E00D0CB
:109D9000EDB7FEB7319604E01FE0ADB7BEB712963F
:109DA0001C930E9311978A81828313820E94037EF3
:109DB000EDB7FEB73196ADB7BEB712961C930E93B2
:109DC00011978981828313820E94037E0F900F90E6
:109DD00082E09FE0EDB7FEB7928381830E94037E0D
:109DE0000F900F900E94BF61E0918706F091880666
:109DF0000995E0916E06F0916F060995E0913006A5
:109E0000F09131060995E0906C06F0906D06009196
:109E10008506109186060E94A855D82E0E943B57B1
:109E20002DB73EB72A5030400FB6F8943EBF0FBE54
:109E30002DBFEDB7FEB7319627EE3EE0ADB7BEB70A
:109E400012963C932E931197F382E282158304833A
:109E5000D6821782808711860E94037EE091910648
:109E6000F09192062DB73EB7265F3F4F0FB6F8949C
:109E70003EBF0FBE2DBF3097D1F00995BC0100D079
:109E800000D084ED9EE0ADB7BEB712969C938E9342
:109E9000119780E890E00E94597AEDB7FEB774837D
:109EA00063830E94037E0F900F900F900F9000D05D
:109EB00082ED9EE0ADB7BEB712969C938E9311973C
:109EC0000E94037E0F900F9080EB96E060E070E0C0
:109ED0000E94FD4082E395E00E94656000D08AEC1C
:109EE0009EE0EDB7FEB7928381830E94037E0F90C0
:109EF0000F900F900F90CF91DF911F910F91FF90D6
:109F0000EF90DF900895EF92FF920F931F9380E8F8
:109F100080936100109261000E94394E0E94594066
:109F20000E94DA528091162590911725009729F00A
:109F300001979093172580931625E0901825F090AF
:109F4000192500911A2510911B250E947B51E616B8
:109F5000F7060807190711F30E947B516093182533
:109F60007093192580931A2590931B25D7CF00D085
:109F700000D000D0EDB7FEB7319624EC3EE0ADB78F
:109F8000BEB712963C932E93119793838283758369
:109F900064830E94037E8DB79EB706960FB6F89431
:109FA0009EBF0FBE8DBF08950F931F93DF93CF9376
:109FB000CDB7DEB7A2970FB6F894DEBF0FBECDBF08
:109FC00083E490E00E94467F89839A83982F9B5078
:109FD000903108F08A839A819095891709F470C0AE
:109FE00000D080E79FE0ADB7BEB712969C938E93EA
:109FF00011970E94037E8E010D5F1F4F0F900F90EF
:10A00000D80180E090E0FC01E05BF04FE491ED933B
:10A01000019688309105B9F7F894CE01039661E274
:10A0200070E048E050E00E944C7FD80180E090E072
:10A03000FC01E85AF04FE491ED9301968E309105C2
:10A04000B9F7CE01039669E270E04EE050E00E945D
:10A050004C7F80E090E0FC01EA59F04FE491D80198
:10A06000ED938D0101968A309105A9F7CE010396F3
:10A0700067E370E04AE050E00E944C7F85E490E0A6
:10A080006DEC7BEA0E94647F87E490E060E070E022
:10A090000E94647F89E490E060E00E94567F81E442
:10A0A00090E060E070E00E94647F8AE1898385EE41
:10A0B0008A8369817A8183E490E00E94647F789446
:10A0C0008981A2960FB6F894DEBF0FBECDBFCF91A7
:10A0D000DF911F910F910895F89461E270E042E0E2
:10A0E00050E00E942E7F789480E0089585E490E00F
:10A0F0000E94467F089587E490E00E94467F08957D
:10A1000089E490E00E943E7F0895209124253091BB
:10A110002525409126255091272590E0A0E0B0E02C
:10A12000280F391F4A1F5B1F2093242530932525B4
:10A1300040932625509327252091202530912125D5
:10A140004091222550912325280F391F4A1F5B1F5C
:10A1500020932025309321254093222550932325B9
:10A160002091C4262223A1F020911C2530911D2589
:10A1700040911E2550911F25280F391F4A1F5B1F34
:10A1800020931C2530931D2540931E2550931F2599
:10A1900008951F920F920FB60F920BB60F921124D3
:10A1A0002F933F934F935F936F937F938F939F93DF
:10A1B000AF93BF93EF93FF938091F00F9091F10FC6
:10A1C00001969093F10F8093F00F8091F20F8F5FC3
:10A1D0008093F20F8091F20F8038A9F41092F20F61
:10A1E0008091242590912525A0912625B0912725A1
:10A1F0000196A11DB11D8093242590932525A09340
:10A200002625B09327258091C4268823F1F08091DC
:10A21000F30F8F5F8093F30F8091F30F8038A9F4D1
:10A220001092F30F80911C2590911D25A0911E2561
:10A23000B0911F250196A11DB11D80931C259093FF
:10A240001D25A0931E25B0931F250E94C44300978F
:10A2500011F00E94C442FF91EF91BF91AF919F9185
:10A260008F917F916F915F914F913F912F910F90BF
:10A270000BBE0F900FBE0F901F901895F894109280
:10A28000B60016BC83EF87BD82E084BD94E095BD27
:10A2900095B395BB80936E00789408952091F00F4C
:10A2A0003091F10F8091F00F9091F10F281739073D
:10A2B000A9F7C901089507C022E330E0000021504A
:10A2C0003040E1F701970097B9F708950F931F9376
:10A2D000CF93DF938C010E944E51EC010E944E51AE
:10A2E0008C1B9D0B80179107C8F3DF91CF911F91B5
:10A2F0000F910895089520912425309125254091AE
:10A300002625509127258091242590912525A091DF
:10A310002625B0912725281739074A075B0759F7E3
:10A32000B901CA0108951F920F920FB60F9211241E
:10A330001092DD050F900FBE0F901F9018951F9281
:10A340000F920FB60F920BB60F9211242F933F93DB
:10A350004F935F936F937F938F939F93AF93BF932D
:10A36000EF93FF93E091D305F091D4058081E091C4
:10A37000DE05F091DF05309709F00995FF91EF9127
:10A38000BF91AF919F918F917F916F915F914F910D
:10A390003F912F910F900BBE0F900FBE0F901F900B
:10A3A00018951F920F920FB60F9211241092EA0582
:10A3B0000F900FBE0F901F9018951F920F920FB61F
:10A3C0000F920BB60F9211242F933F934F935F93ED
:10A3D0006F937F938F939F93AF93BF93EF93FF936D
:10A3E000E091E005F091E1058081E091EB05F091CD
:10A3F000EC05309709F00995FF91EF91BF91AF916E
:10A400009F918F917F916F915F914F913F912F918C
:10A410000F900BBE0F900FBE0F901F90189590E0FD
:10A420002DE030E0829FF001839FF00D929FF00DB0
:10A430001124ED52FA4FA281B3811C92A481B581FF
:10A440006C93A681B78188ED8C93A085B1854C93E0
:10A45000128614861386089590E02DE030E0829FE6
:10A46000F001839FF00D929FF00D1124ED52FA4FF1
:10A4700081E08287A081B1816C933A9680818823A4
:10A48000E9F708951F93182F8A3031F48091F40F63
:10A490006DE00E942C5202C08D3029F08091F40FA3
:10A4A000612F0E942C5280E090E01F910895EF925E
:10A4B000FF921F93CF93DF93182FE62EE7017E01C3
:10A4C000F72EE7010CC08A3021F4812F6DE00E9445
:10A4D0002C5269916D3019F0812F0E942C52888185
:10A4E000882389F7DF91CF911F91FF90EF90089516
:10A4F0000F931F93DF93CF93CDB7DEB7FE013A964C
:10A5000005EF1FE0C80160E470E0488559859F01B0
:10A510000E94987E8F81B8010E945752CF91DF919F
:10A520001F910F9108951F93CF93DF93182FEB0185
:10A5300004C0812F0E942C522196FE016491662353
:10A54000C1F7DF91CF911F91089590E02DE030E0A9
:10A55000829FF001839FF00D929FF00D1124ED5228
:10A56000FA4F748763870895682F80E00E942C5209
:10A5700008958093F40F85EC95E09093912D80934E
:10A58000902D089584B7877F84BF88E10FB6F89433
:10A5900080936000109260000FBE08952FE088E164
:10A5A00090E00FB6F894A895809360000FBE2093BA
:10A5B00060000895A895089588E10FB6F8948093F7
:10A5C0006000109260000FBE0895F89428E088E1C2
:10A5D00090E00FB6F894A895809360000FBE20938A
:10A5E0006000FFCF8091372590E0FC01EE0FFF1F48
:10A5F0009695982F882797958795E80FF91FE85C1F
:10A60000FA4D1082089580912F2580912F2590E09A
:10A6100008958091390181FD0CC081E491E06FE1E2
:10A6200040E00E94DC58813039F021E030E0813197
:10A6300029F020E030E002C021E030E0C9010895B7
:10A640008091390181FD12C081E491E06FE140E029
:10A650000E94DC58982F8151823050F09F3141F098
:10A66000913041F081E0923031F402C081E00895F0
:10A6700080E0089580E008950E9420538823E1F34C
:10A68000089581E491E06FE140E00E94DC58089574
:10A69000E9E3F1E0808180818D7F80838DE090E02F
:10A6A0000197F1F782E491E06FE140E023E00E943E
:10A6B000E65883E090E00197F1F708950E943C533B
:10A6C0001092C4260E944853809139018260809381
:10A6D0003901809147278823E9F180919400909176
:10A6E0009500209158273091592782179307A0F49D
:10A6F0008091242790912527A0912627B091272784
:10A700008C57914EAF4FBF4F8093242790932527AE
:10A71000A0932627B09327278091940090919500CD
:10A72000821B930BA0E0B0E02091242730912527D5
:10A730004091262750912727820F931FA41FB51FF2
:10A740008093242790932527A0932627B09327272B
:10A7500010924727809149278823E9F1809194003E
:10A760009091950020915C2730915D278217930787
:10A77000A0F480912C2790912D27A0912E27B091A5
:10A780002F278C57914EAF4FBF4F80932C2790931C
:10A790002D27A0932E27B0932F278091940090917E
:10A7A0009500821B930BA0E0B0E020912C27309104
:10A7B0002D2740912E2750912F27820F931FA41FE2
:10A7C000B51F80932C2790932D27A0932E27B0930D
:10A7D0002F271092492708958091C426882381F05D
:10A7E00080913510882321F40E942053882331F46E
:10A7F00081E08093B81021E030E004C00E945E53F5
:10A8000020E030E0C90108950F931F93182F88307E
:10A8100049F0863039F0893029F0863119F08931D4
:10A8200009F041C08091390181FD40C00E943C5334
:10A830000E944153082F181709F43BC0183019F42F
:10A840000E94485329C0193141F48631A9F482E4A9
:10A8500091E06FE140E029E009C0163169F48931E7
:10A8600059F482E491E06FE140E026E00E94E6586E
:10A87000E3E0F0E03197F1F782E491E06FE140E04E
:10A88000212F0E94E658083019F4E9E6F1E002C0F1
:10A89000E3E0F0E03197F1F70E944153811749F06E
:10A8A00023E430E008C022E430E005C024E430E0D6
:10A8B00002C020E430E0C9011F910F9108958091FA
:10A8C00094009091950090935D2780935C2721E000
:10A8D000209349278091390181FF15C02093C32619
:10A8E00080919400909195009093592780935827D8
:10A8F00020934727809139018D7F80933901809182
:10A90000C3268823E1F786E10E94045481E0809306
:10A91000C42608958091C426882351F4809135106F
:10A92000882321F081E08093B71002C00E945F5419
:10A9300081E090E008951F93DF93CF930F92CDB7FE
:10A94000DEB78FB7898380913510882331F5F8946D
:10A950008091C426882351F08091390181FD1BC06C
:10A960000E9420538823B9F080E003C00E948A54DB
:10A9700081E0909147019E3010F010E001C01FEF80
:10A98000882311F00E94EC5316FF05C089818FBF08
:10A9900021E030E004C089818FBF20E030E0C901B0
:10A9A0000F90CF91DF911F9108958091B710882368
:10A9B00021F00E945F541092B7108091B810882344
:10A9C00021F00E945E531092B81010923510089535
:10A9D000EF92FF92CF93DF93B82FA92FF62FE72F97
:10A9E00081E080933510209108273091092740910C
:10A9F0000A2750910B272F5F3F4F4F4F5F4F2093F8
:10AA000008273093092740930A2750930B27862F56
:10AA10008E5F87FF0CC08091C1269091C22601965F
:10AA20009093C2268093C126CFEFDFEF0BC026E3C1
:10AA300030E1C9016B2F7A2F4F2F5E2F0E94727D5C
:10AA4000C0E0D0E00E94D554CE01DF91CF91FF90BD
:10AA5000EF9008959091390191FD0AC0282F80311F
:10AA600008F02FE085E491E06FE040E00E94E658B6
:10AA700008958093BA1008950E9441538250813105
:10AA800030F4E82FF0E0E85EF94F8081089581E02E
:10AA9000089508958FEF80934E018CE691E060EF6A
:10AAA00044E022E00E94E6588CE290E06EE041E053
:10AAB00025E00E94E65880E880936F01809146016E
:10AAC00080936D0184E491E060E245E021E00E9422
:10AAD000E6580895CF93DF93CDEFD3E0CE010197F1
:10AAE000F1F70E94D258109238251092BA25109290
:10AAF0003C261092372510923625E9E3F1E080815B
:10AB00008E7F808380818D7F80838DE090E00197B0
:10AB1000F1F780818160808382E491E06FE140E021
:10AB200023E00E94E6582197F1F780915D01809122
:10AB30005E010E944A558AEF95E060E070E00E9455
:10AB4000FD400E945F5481E090E0DF91CF91089535
:10AB50008091B9100895DF93CF930F92CDB7DEB7F0
:10AB600089830E943C5329812093B91088E491E0A5
:10AB70006FE140E00E94E6580F90CF91DF91089579
:10AB80000E94AB5586E00E940454089580936201B0
:10AB900090936301609360017093610141155105C9
:10ABA00031F1FA01819180936B01DA0111968C9158
:10ABB00080936A01DF011196818180936901FD0113
:10ABC000319611968C9180936801DF0111968181F5
:10ABD00080936701FD01319611968C9111978093B6
:10ABE000660181818093650182818093640108956B
:10ABF0008AEF95E00E94204181E080932F2580918B
:10AC00003025909131250196909331258093302500
:10AC100081E090E00895EF92FF92CF93DF935091FF
:10AC20003725252F30E0F901EE0FFF1F3695322F23
:10AC3000222737952795E20FF31FE85CFA4D4081F4
:10AC4000442309F4CEC02091390121FDCAC02091CE
:10AC5000C426222309F4C5C047FF16C00E94F25241
:10AC60008091F8269091F926A091FA26B091FB26C2
:10AC70000196A11DB11D8093F8269093F926A0930B
:10AC8000FA26B093FB26ADC04330B0F40E94F252D6
:10AC90008091F4269091F526A091F626B091F726A2
:10ACA0000196A11DB11D8093F4269093F526A093E3
:10ACB000F626B093F72695C0C42FD0E022976C17E4
:10ACC0007D07B0F40E94F2528091F0269091F12617
:10ACD000A091F226B091F3260196A11DB11D80939B
:10ACE000F0269093F126A093F226B093F32679C034
:10ACF000652F70E09B01220F331F7695762F662714
:10AD000077956795260F371F275C3A4DB90150E0BC
:10AD10000E94727D20913725822F90E0FC01EE0F7A
:10AD2000FF1F9695982F882797958795E80FF91F0D
:10AD3000E854FA4D808180932825822F90E0FC0111
:10AD4000EE0FFF1F9695982F882797958795E80F08
:10AD5000F91FE85CFA4D10822F5F209337252330CE
:10AD600010F0109237258091372590E0FC01EE0F0E
:10AD7000FF1F9695982F882797958795E80FF91FBD
:10AD8000E85CFA4D8081882311F00E94F8556091AB
:10AD900047016093292580912E25882311F068179B
:10ADA00010F460932E2584E070E00E94BC4860910E
:10ADB000282583E070E00E94BC4880910C27909188
:10ADC0000D27A0910E27B0910F270196A11DB11D4F
:10ADD00080930C2790930D27A0930E27B0930F27F5
:10ADE00002C0C0E0D0E0CE01DF91CF91FF90EF90A4
:10ADF0000895CF93DF93EC0188819981009729F022
:10AE000024E08B3F920739F505C08BEF94E09983DE
:10AE1000888325C0623819F510922F250E94364884
:10AE20000E94934760E870E00E940B5618161906BE
:10AE300044F40E948E47E0918B06F0918C060995B0
:10AE4000E4CF80912C2590912D25019690932D256E
:10AE500080932C25DACF1982188283E001C081E02B
:10AE6000DF91CF91089591E0909335100E942A557B
:10AE70000E94D55408958091390181FD07C085E471
:10AE800091E06FE040E00E94DC58089580E1089571
:10AE9000CF92DF92EF92FF920F931F93CF93DF93A6
:10AEA000182F21E0209335100091C426809139019C
:10AEB00081FF16C08091940090919500909359273E
:10AEC00080935827209347272093C32680913901E8
:10AED0008D7F809339018091C3268823E1F700E0BC
:10AEE0000E943C538091C426882309F441C080917C
:10AEF00049278823E9F120919400309195008091B1
:10AF00005C2790915D2728173907A0F420912C2702
:10AF100030912D2740912E2750912F272C57314EBD
:10AF20004F4F5F4F20932C2730932D2740932E2790
:10AF300050932F272091940030919500281B390BB6
:10AF400040E050E0C0902C27D0902D27E0902E2795
:10AF5000F0902F272C0D3D1D4E1D5F1D20932C279B
:10AF600030932D2740932E2750932F271092492757
:10AF700089E10E94045486E00E94C748009751F07E
:10AF80000E943B57C82F86E00E94C74881500E940C
:10AF90002A5502C0C0E0D0E08091940090919500C5
:10AFA00090935B2780935A2781E080934827F894F9
:10AFB00080913901826080933901809139018D7FC0
:10AFC00080933901612F6E5F86E390E10E941759EB
:10AFD00078948091BE269091BF2601969093BF26CB
:10AFE0008093BE260E943C5382E491E060EE45E0EF
:10AFF0000E94DC58182F86E00E94C748009719F07D
:10B000008C2F0E942A55002319F00E945F5402C021
:10B010000E945E53809148278823E9F18091940033
:10B020009091950040915A2750915B27841795077E
:10B03000A0F48091282790912927A0912A27B091E8
:10B040002B278C57914EAF4FBF4F8093282790935B
:10B050002927A0932A27B0932B2720919400309181
:10B060009500241B350B40E050E0809128279091FB
:10B070002927A0912A27B0912B27280F391F4A1F73
:10B080005B1F209328273093292740932A2750932A
:10B090002B27109248278091C426882361F0809145
:10B0A00094009091950090935D2780935C2781E0B8
:10B0B0008093492707C082E491E06FE140E023E0FC
:10B0C0000E94E6580E94D5541130E1F01330A9F4E3
:10B0D0008091002790910127A0910227B09103272A
:10B0E0000196A11DB11D8093002790930127A09385
:10B0F0000227B093032712E00AC0153029F0173059
:10B1000031F404C010E003C013E001C011E0812F4E
:10B1100090E0DF91CF911F910F91FF90EF90DF9022
:10B12000CF900895CF93DF93EB010E94E8549C01E8
:10B13000009731F4CE010E9448579C01009749F0D6
:10B140008091C1269091C22601969093C226809349
:10B15000C126C901DF91CF9108950F931F9380916C
:10B16000C426882321F40E948A5411E001C010E013
:10B170000E944153863111F0813119F40091470149
:10B1800009C086E491E06FE140E00E94DC58082F9E
:10B19000000F080F112311F00E94EC53802F1F9114
:10B1A0000F9108951092BC101092BB10EFE6F0E0E2
:10B1B0008081806280830895FC018081862390E0F5
:10B1C00002C0959587954A95E2F70895F894FC0199
:10B1D0009081862F8095892330E002C0220F331F93
:10B1E0004A95E2F72623282B208378940895DC01E2
:10B1F000119620917B01FC012083215030E0A901B0
:10B200004F575E4FE0E8F1E061916D93E417F50769
:10B21000D9F7FC01E058FF4F2F573E4FD9012C9131
:10B2200020838F579F4F21E0FC0120830895FC016C
:10B230006093800101966350860F911DA1E8B1E0F3
:10B2400021912D93E817F907D9F708951F920F92CE
:10B250000FB60F920BB60F9211242F933F934F937B
:10B260005F936F937F938F939F93AF93BF93EF936E
:10B27000FF9380914701809329252091362530E066
:10B28000C901880F991F3695322F222737952795A8
:10B29000820F931F885C9A4D0E94F7588091362543
:10B2A0008F5F80933625833010F0109236250E94F0
:10B2B000F855FF91EF91BF91AF919F918F917F9141
:10B2C0006F915F914F913F912F910F900BBE0F9017
:10B2D0000FBE0F901F9018951F920F920FB60F92EE
:10B2E00011240F900FBE0F901F9018951F920F9270
:10B2F0000FB60F9211240F900FBE0F901F9018954C
:10B300001F920F920FB60F9211240F900FBE0F9045
:10B310001F9018951F920F920FB60F921124109242
:10B32000C3260F900FBE0F901F9018951F920F927B
:10B330000FB60F9211241092C3260F900FBE0F90DC
:10B340001F9018951F920F920FB60F9211248F9392
:10B3500081E080932F258F910F900FBE0F901F904B
:10B3600018951F920F920FB60F9211241092C326B8
:10B370000F900FBE0F901F9018951F920F920FB64F
:10B380000F9211248F939F938091BB109091BC10CA
:10B3900001969093BC108093BB109F918F910F905A
:10B3A0000FBE0F901F9018950F931F93CF93DF93AD
:10B3B0008091CC269091CD26A091CE26B091CF261B
:10B3C0000196A11DB11D8093CC269093CD26A0930C
:10B3D000CE26B093CF260E94855CEC018DEB90E1E8
:10B3E0000E94C2410BC0D8011296ED91FC911397B7
:10B3F000309709F00995C8010E948842082F192F3B
:10B400000115110581F7209719F0CE010E94323FF6
:10B41000DF91CF911F910F9108950E94BF610E940B
:10B4200036480E948F5A8CE696E09093C726809308
:10B43000C6260E94825C82E090E060E074E040E01A
:10B440005EE12FEF31E00E94435C0895CF92DF92DE
:10B45000EF92FF920F931F93CF93DF936C01EB0159
:10B460008A018DEB90E10E94C2410CC0D701149675
:10B47000ED91FC911597309711F0CE010995C70118
:10B480000E948842E82EF92EE114F10479F7C601F2
:10B49000BE01A8010E943A3FDF91CF911F910F9109
:10B4A000FF90EF90DF90CF900895BC018DEB90E17D
:10B4B0000E9449420895BC018DEB90E10E94104228
:10B4C0000895CF93DF93EC018091C8269091C9260F
:10B4D000A091CA26B091CB260196A11DB11D8093E3
:10B4E000C8269093C926A093CA26B093CB26CE0136
:10B4F0000E949C5C009769F00E94B047E091700642
:10B50000F091710686E29AE5BE01099521E030E0EE
:10B5100002C020E030E0C901DF91CF9108958FEBA8
:10B5200090E10E94BE4108950F93CF93DF93EC0109
:10B530007B836A8318865F834E838FEB90E1BE0125
:10B540000E944942E091C110F091C210309749F039
:10B550004C815D818A819B81688520E030E001E03B
:10B560000995DF91CF910F910895BC018FEB90E188
:10B570000E94104208950F93DC0118961C921897B0
:10B58000E091C110F091C210309759F012968D9150
:10B590009C91139760E040E050E020E030E000E054
:10B5A00009950F9108950F93DC01AB0114962D912D
:10B5B0003C91159781E018968C93189715967C937B
:10B5C0006E931497E091C110F091C210309739F04A
:10B5D00012968D919C91139761E000E009950F916F
:10B5E00008950F93DC01E091C110F091C2103097E3
:10B5F00069F014962D913C91159712968D919C911E
:10B60000139718966C91A90101E009950F9108957F
:10B61000E091C310F091C410309709F00995089596
:10B620009093C4108093C31008959093C210809398
:10B63000C11008958FEB90E10E94C2410895EF92EE
:10B64000FF920F931F93CF93DF938C01EB017A014D
:10B650008FEB90E10E94C24115C0DC0112962D9142
:10B660003C9113972C173D0759F41696ED91FC91D8
:10B670001797309761F0B801AE019701099507C09F
:10B680000E948842282F392FC901009731F7DF9196
:10B69000CF911F910F91FF90EF9008950895AF9271
:10B6A000BF92CF92DF92EF92FF920F931F93DF939F
:10B6B000CF9300D0CDB7DEB75B010E949347FC016A
:10B6C000008111811A8309830C30110518F4EE24CE
:10B6D000FF242EC000D000D084E396E0EDB7FEB783
:10B6E00092838183148303830E94F17D0F900F90D6
:10B6F0000F900F9020C00E949347F701EE0FFF1F9D
:10B70000EE0FFF1FE80FF91FC280D3800E949347FE
:10B710000894E11CF11CF701EE0FFF1FEE0FFF1F55
:10B72000E80FF91F40815181C501B6010E941F5BDE
:10B73000E016F10600F30F900F90CF91DF911F916B
:10B740000F91FF90EF90DF90CF90BF90AF90089552
:10B75000CF93DF93C0EED0E16091F6107091F710B7
:10B76000CE014AED5BE520E030E00E9487440E9474
:10B77000BC616091F6107091F7100E94597ABC017B
:10B78000CE0140974FEE5BE520E030E00E94874419
:10B79000DF91CF9108950F93013051F48091F01013
:10B7A0009091F1109093F7108093F6100E94A85B8F
:10B7B0000F9108958091F6109091F7102091F41058
:10B7C0003091F510880F991F2817390708F4C9011F
:10B7D0009093F7108093F6100E94A85B0895EF9263
:10B7E000FF92CF93DF930E9436480E949347E82E42
:10B7F000E7017E01F92EE701198218820E941A5B87
:10B8000026C028813981F901EE0FFF1FEE0FFF1FBF
:10B81000EC0FFD1FDC0112964D915C911397538341
:10B8200042832F5F3F4FF901EE0FFF1FEE0FFF1F07
:10B83000EC0FFD1F14964D915C9115975183408339
:10B84000398328830E948842282F392FC901009705
:10B8500021F0FC0120852223A1F688819981880F9F
:10B86000991F880F991F02960E948E47888199819F
:10B87000009721F085EC90E10E94053FDF91CF9188
:10B88000FF90EF900895EF92FF920F931F93CF9345
:10B89000DF93FC018B017A01E90185EC90E1BF01A6
:10B8A00041E556E00E94E73E1093F1100093F0103E
:10B8B000F092F310E092F210D093F510C093F410D0
:10B8C0008BEC9BE50E94155BDF91CF911F910F914F
:10B8D000FF90EF900895CF93DF93C0EED0E1CE01BB
:10B8E0000E940E45CE0140970E940E45CE014B9717
:10B8F0000E94023FDF91CF9108958091F6109091C0
:10B90000F71008950E94463F0895EF92FF92CF935B
:10B91000DF93E0915506F09156060995EC010097EA
:10B9200029F06A817B8181E00E94BC48CE01DF91D1
:10B93000CF91FF90EF9008950F931F93CF93DF93D4
:10B940008C01E0915706F09158060995EC01F80139
:10B950006281738181E00E94BC4821E030E0209741
:10B9600011F420E030E0C901DF91CF911F910F91D8
:10B970000895E0915906F0915A0609950895FC0141
:10B9800020E030E004C08181280F311D3296808193
:10B990008823C9F7C9010895FC01818190E03081B5
:10B9A00020E0822B932B02C0880F991F6A95E2F743
:10B9B000892F9927FA01E55AF94F208130E0822337
:10B9C000932328E030E0241B350B02C09695879521
:10B9D0002A95E2F708956F927F928F929F92AF928D
:10B9E000BF92CF92DF92EF92FF920F931F93CF936C
:10B9F000DF936C017B015A0189012830310544F441
:10BA0000CB01BA01A9010E94CC5CF601808341C040
:10BA1000390133E0759467943A95E1F74115510582
:10BA200021F04C01C0E0D0E016C0DB01FC01C0E019
:10BA3000D0E08D9181932196C615D705D4F3A80146
:10BA4000477050704115510521F1C7018C0F9D1FA2
:10BA500060E070E019C0C7018C0F9D1FB50148E080
:10BA600050E00E94CC5CF40181934F012196C615F1
:10BA7000D7058CF3A801477050704115510549F066
:10BA8000C7018C0F9D1FB5010E94CC5CCC0DDD1D44
:10BA90008883DF91CF911F910F91FF90EF90DF90FE
:10BAA000CF90BF90AF909F908F907F906F900895B0
:10BAB0004F925F926F927F928F929F92AF92BF92BE
:10BAC000CF92DF92EF92FF920F931F93DF93CF936A
:10BAD00000D000D0CDB7DEB70E949347E82E092FE3
:10BAE00082E090E00E946F47009709F464C0EE2D59
:10BAF000F02F918180E02081820F911D0E945A3F9A
:10BB00007C01009709F459C00E9493473C01F7015A
:10BB10004681242F30E02770307081E090E02115BD
:10BB2000310511F480E090E0469546954695840FE6
:10BB3000911D0E946F470097F1F1F7010481158173
:10BB4000CC24DD2453E0452E512C4C0E5D1E4E01BD
:10BB50000894811C911C2AC0F801A180BB24B60165
:10BB600043E0759567954A95E1F7660D771DA60147
:10BB700047705070883150F0C40195010E94EB5C11
:10BB8000F8018081B4010E94D0480CC01C821B8245
:10BB9000C20195010E94EB5C6B817C81F801808180
:10BBA0000E94BC48CA0CDB1C0E5F1F4FF80180814D
:10BBB000882391F602C0EE24FF24C7010F900F9056
:10BBC0000F900F90CF91DF911F910F91FF90EF9009
:10BBD000DF90CF90BF90AF909F908F907F906F90AD
:10BBE0005F904F900895FC0150E080E190E0861B4B
:10BBF000970B821B930B02C0440F551F8A95E2F7E7
:10BC00008081852B80838181842B818308956F922D
:10BC10007F928F929F92AF92BF92CF92DF92EF92DC
:10BC2000FF920F931F93CF93DF938C015B016A0107
:10BC300079012830310524F4C801FA01408156C049
:10BC4000390163E0759467946A95E1F7A114B10432
:10BC500021F04A01C0E0D0E021C0DA01F80180E023
:10BC600090E02D912193019686159705D4F39701C5
:10BC70002770307021153105D9F1F601E80FF91F51
:10BC8000408150E068E070E0621B730B02C0559584
:10BC900047956A95E2F7800F911F26C0F401419104
:10BCA0004F01C8018C0F9D1FB50128E030E00E94B4
:10BCB000F35D2196C615D7058CF397012770307078
:10BCC00021153105A9F0F601EC0FFD1F408150E070
:10BCD000C5010896821B930B02C0559547958A951E
:10BCE000E2F7C8018C0F9D1F60E070E00E94F35DD9
:10BCF000DF91CF911F910F91FF90EF90DF90CF9048
:10BD0000BF90AF909F908F907F906F9008954F92CB
:10BD10005F926F927F928F929F92AF92BF92CF92DB
:10BD2000DF92EF92FF920F931F93DF93CF9300D098
:10BD3000CDB7DEB78C01DC0116964C911697842F97
:10BD400090E08770907021E030E0009711F420E0DF
:10BD500030E04695469546957901E40EF11CC70101
:10BD600002960E94FB47009709F453C00E949B472C
:10BD7000FC01D80112968C911297808313968C91B6
:10BD800081830E949B47F2E06F2E712C680E791E12
:10BD9000C30160E070E0A7010E947B7DF801C480D0
:10BDA000D58000E010E02E010894411C511C2AC0EF
:10BDB000D60111968C90119799247801E3E0F594BF
:10BDC000E794EA95E1F7E60CF71C77E0A72EB12C93
:10BDD000A022B122883130F00E94DA48AC01C701BC
:10BDE000B50107C00E94C7489A838983C701B5017E
:10BDF000A20194010E94075E080D191DE2E0F0E027
:10BE0000CE0EDF1ED6018C91882391F621E030E022
:10BE100002C020E030E0C9010F900F90CF91DF9178
:10BE20001F910F91FF90EF90DF90CF90BF90AF9058
:10BE30009F908F907F906F905F904F900895E091CA
:10BE40008906F0918A0609950895E0913206F091ED
:10BE5000330609950895E0918D06F0918E060995B7
:10BE60000895E0918F06F09190060995089580E07D
:10BE700090E008950895E0911406F0911506099553
:10BE80000895009731F0E0911406F0911506099598
:10BE90000895E0911606F09117060995089580E03F
:10BEA00090E008950F931F93DF93CF93CDB7DEB744
:10BEB000E0970FB6F894DEBF0FBECDBF0E94E547F6
:10BEC0008C010E949347602FAE014F5F5F4F0E942D
:10BED0008567882309F445C088A99801281B310982
:10BEE000C9010E946F470097E1F12E81222371F171
:10BEF0008A859B853BEA8D3C930721F03FEF8F3F7E
:10BF0000930779F5223041F088E090E007C001976F
:10BF100022912F3F41F00BC082E090E0FE01E80F3C
:10BF2000F91F3C96F4CF181619068CF30FC089E15F
:10BF3000BE01645F7F4F0E94D04889E10E94DA48C9
:10BF400065ED74E20E94983E009759F088E1BE01C9
:10BF50006A5E7F4F0E94D048E0917206F0917306AE
:10BF60000995E0960FB6F894DEBF0FBECDBFCF9116
:10BF7000DF911F910F910895AF92BF92CF92DF9200
:10BF8000EF92FF920F931F93DF93CF93CDB7DEB75E
:10BF9000E0970FB6F894DEBF0FBECDBF6C018B01EA
:10BFA000FE01319680E3DF011D928A95E9F781E079
:10BFB00089838CE00E94C7488C831D821F828091F8
:10BFC000FA1089878F5F8093FA1083E0E82EE88665
:10BFD0008DEC9BEA9B878A8789E10E94DA486CE4B2
:10BFE00075E00E94983E009731F082E08E838FEFDB
:10BFF0008C878D8709C089E10E94DA48BC01CE0197
:10C000000C960E948F3EEE828DEC9BEA9D8B8C8B72
:10C01000CE01469665ED74E20E948F3E0E949347E2
:10C020009FA78EA70E94E54788AB7E010894E11C7C
:10C03000F11CC7010E947C66A82E90E00E94FB477D
:10C04000009741F10E949B47BC01C7014A2D0E9405
:10C050009A66A0900A06B0900B060E949B477C014E
:10C060000E94EF47BC01C701F5010995C114D10435
:10C0700089F0009721F08130910561F404C0C80176
:10C0800060E070E003C0C80164E070E041E050E0AF
:10C09000F6010995E0960FB6F894DEBF0FBECDBF4E
:10C0A000CF91DF911F910F91FF90EF90DF90CF9094
:10C0B000BF90AF9008950E94BC618093FA10E09108
:10C0C0001406F091150609950895EF92FF92CF930B
:10C0D000DF93E82EE7017E01F92EE70104C060E05E
:10C0E00070E00E94FD40899199910097C1F7DF911E
:10C0F000CF91FF90EF900895EF92FF92CF93DF934F
:10C10000E82EE7017E01F92EE70102C00E944240BD
:10C11000899199910097D1F7DF91CF91FF90EF909E
:10C120000895CF93DF93EC017B836A830E944E5185
:10C1300099838883DF91CF910895FC01808191815B
:10C1400022813381820F931F918380830895CF933F
:10C15000DF93EC010E944E5199838883DF91CF9148
:10C160000895CF93DF93EC010E944E5128813981CD
:10C17000821B930B019621E030E04A815B814817D6
:10C18000590710F020E030E0C901DF91CF91089508
:10C19000EF92FF92CF93DF93FC01C281D381808124
:10C1A0009181C80FD91F0E944E51C81BD90BCE01D7
:10C1B000DF91CF91FF90EF900895CF93DF93EEE45E
:10C1C000F7E2C0E1D7E2A2E4B7E21192119219922C
:10C1D0001992199219921D9287E2E636F807A9F78B
:10C1E000DF91CF9108950F931F93CF93DF93FC01BD
:10C1F000DC01AE5BB84D8C91882339F1009194003D
:10C2000010919500EF01CC0FDD1FCC0FDD1FC05F3B
:10C21000D84DDF01AA0FBB1FA25BB84D8D919C9139
:10C2200011979801281B390B40E050E06881798113
:10C230008A819B81260F371F481F591F2883398306
:10C240004A835B8311961C930E93EE0FFF1FEE0F34
:10C25000FF1FE05FF84D6081718182819381DF91E2
:10C26000CF911F910F91089560E070E0CB01089588
:10C27000FC01EE0FFF1FEE0FFF1FE05FF84D408344
:10C280005183628373830895EF92FF920F931F93FC
:10C29000CF93DF9322E437E2C0E1D7E2EEE4F7E2A6
:10C2A000D9018D919D018823C9F04091940050914E
:10C2B0009500808191817A01E81AF90A00E010E086
:10C2C00088819981AA81BB818E0D9F1DA01FB11FFE
:10C2D00088839983AA83BB835183408324963296B3
:10C2E000B7E22E343B07E1F6DF91CF911F910F911A
:10C2F000FF90EF9008950E94F96508950F931F93A2
:10C30000FC01CB014091FB105091FC103383228340
:10C310001583048371836083F093FC10E093FB101A
:10C320004115510511F40E94136680E090E01F91C1
:10C330000F9108958091FB109091FC100097C1F02F
:10C340001092FC101092FB10DC0114966D917C9100
:10C3500015971296ED91FC9113970995E091FB10BA
:10C36000F091FC10309721F0808191810E9413663A
:10C3700008950E94477B08950E94427B089583E9B7
:10C3800096E00E9436418BE996E00E94364108957E
:10C39000EF92FF92CF93DF930E94A2470097C9F0DC
:10C3A0008BE996E00E945641E82EE7017E01F92EC6
:10C3B000E701209731F10E94E547998388830E9425
:10C3C000E0479B838A83C70104960E940E478CAB8B
:10C3D00018C083E996E00E945641EC017E01F92ED7
:10C3E000E701209771F0C70102960E9425479983C3
:10C3F0008883B7016E547F4FC7018E579F4F0E94AD
:10C400009248CE01DF91CF91FF90EF900895BC014B
:10C410006E547F4F8E579F4F0E9492480895CF933E
:10C42000DF93EC0183E996E0BE010E94A1410097F1
:10C4300019F083E996E009C08BE996E0BE010E94FD
:10C44000A141009729F08BE996E0BE010E947C4152
:10C45000DF91CF910895EF92FF92CF93DF93EC019C
:10C4600083E996E0BE010E94A141009779F06881BE
:10C470007981CE0102960E945F48BE016E547F4FC3
:10C48000CE018E579F4F0E94A7481BC08BE996E0B4
:10C49000BE010E94A1410097A1F00E943648688128
:10C4A00079818A819B810E945F488CA990E00E94DB
:10C4B000FB470E949B474CA92496BE0150E00E9476
:10C4C000727DDF91CF91FF90EF900895EF92FF92F0
:10C4D000CF93DF93EC0183E996E0BE010E94A14176
:10C4E000009711F022960DC08BE996E0BE010E94E4
:10C4F000A141009721F00A80DB81C02D02C0C0E07D
:10C50000D0E0CE01DF91CF91FF90EF900895FC0134
:10C5100080819181089570E06F5B7F4F660F771F78
:10C52000680F791FCB010895E62FF0E0EF5BFF4F16
:10C53000EE0FFF1FE80FF91F808191810895089584
:10C5400083E597E10E94AC43009721F083E597E1F2
:10C550000E9497430895E0916017F091611730971A
:10C5600011F00995089580E00895EF92FF920F93DE
:10C570001F93CF93DF93EC018A0188819981009703
:10C5800031F023E08C30920709F006C12BC080E027
:10C590000BC0E82FF0E0EE0FFF1FEE0FFF1FEF5B69
:10C5A000F84E118210828F5F843098F380935B176E
:10C5B0008091820E9091830E909352178093511721
:10C5C0000E943B408093662783E597E160E470E03A
:10C5D0000E9481430E9414698CE093E099838883D0
:10C5E00081E0DDC0623009F4B9C0633030F4662305
:10C5F00009F489C0613081F79CC0673819F0683848
:10C6000059F741C010925C1741E4E42E47E1F42E43
:10C6100018C0F701828193818017910749F48081C6
:10C6200091810E945B6AF70111821082138212824B
:10C6300084E090E0E80EF91E80915C178F5F809394
:10C640005C1780915C17843020F3E6E7FCE2848D70
:10C65000958D8017910719F4158E148E118EB09652
:10C660009CE2E63FF90799F7ECE0FDE281859285CF
:10C670008017910711F4158214823D962DE2EE3851
:10C68000F207A1F7A9CF87E14335580709F0A4CFF6
:10C69000CA010E94AC43009709F49ECF10925C1728
:10C6A0002DC0F0E035E0EE0FFF1F3A95E1F7EA58B4
:10C6B000F34D818D8823E9F083E597E10E9497434C
:10C6C00080915C1790E025E0880F991F2A95E1F78B
:10C6D0008A58934D9093752C8093742C82E00E941D
:10C6E0008F6A8091672790916827009711F00E94C8
:10C6F000AB6280915C178F5F80935C17E0915C1751
:10C70000E43078F269CF4115510509F465CF5093B3
:10C71000752C4093742C83E00E948F6A8091672768
:10C7200090916827009711F00E94AB620E94A0626E
:10C7300053CF4115510509F44FCF5093712C4093BD
:10C74000702C85E00E948F6A8091672790916827FE
:10C75000009709F441CF0E94AB623ECF80916727DA
:10C7600090916827009709F437CF80917827863019
:10C7700031F48091902781FF02C00E94A06281E085
:10C780000E948F6A8091672790916827009709F42B
:10C7900023CF0E94DE6420CF1982188283E0DF91CC
:10C7A000CF911F910F91FF90EF9008959093611793
:10C7B0008093601708952091820E3091830E60E07F
:10C7C000E1E4F7E113C0408151814817590761F452
:10C7D000428153814217530739F460935F171182E6
:10C7E00010820E945B6A089534966F5F643058F33C
:10C7F00060935F17089540E0E1E4F7E116C0542F1D
:10C800005F5F208131812115310569F440935E1706
:10C81000918380832091820E3091830E3383228313
:10C820000E94756A08953496452F443040F3409332
:10C830005E170895FC018091820E9091830E958F72
:10C84000848F778F668F0895FC018091820E90917E
:10C85000830E92878187748763870895CF93DF93D0
:10C86000EA010E94D769FC01009741F08091820E95
:10C870009091830E92878187D487C387CF01DF9100
:10C88000CF9108950F931F93DF93CF9300D000D0E3
:10C89000CDB7DEB78C01AB018FEF89838A838B83A1
:10C8A0008C83CE010196B8010E942E64FC01009792
:10C8B00011F015830483CF010F900F900F900F900C
:10C8C000CF91DF911F910F91089580EB96E062E088
:10C8D00040E050E00E94EE401092682710926727D7
:10C8E0000895AC0180EB96E061E00E94CB40089592
:10C8F000AC0180EB96E060E00E94CB4008950F937E
:10C900001F93CF93DF93EA010E944D698C0100973A
:10C9100061F08091820E9091830EF801958F848F43
:10C92000D78FC68FC8010E947864C801DF91CF916C
:10C930001F910F910895CF93DF93A091742CB09124
:10C94000752C109719F0ED016C9605C0C091702CF4
:10C95000D091712C299680916F2C86FF22C0109265
:10C960005D1740E0E1E4F7E116C0208131811496C3
:10C970008D919C9115972817390759F482819381DD
:10C98000009739F040935D17998388831B821A8240
:10C9900006C034964F5F443040F340935D170E94C9
:10C9A000A06288819981009731F04A815B81609112
:10C9B00066270E94EE40DF91CF9108950F931F9359
:10C9C000CF93DF9380917827863009F074C08091EF
:10C9D00067279091682725E08030920709F06BC0A7
:10C9E000C4E9D2E0D0936827C093672702E00093A0
:10C9F000712714E9109372271092942710929327AD
:10CA00000E940C698095909590939427809393272A
:10CA100010927A27109279270E94FB688095909552
:10CA200090937A27809379270E94AB62D0936827EE
:10CA3000C093672700937127109372279091722CEF
:10CA40008091732CE92FF82FDF01A459BD4F8CE69C
:10CA500092E00D9001920197E1F787E897E26CE68A
:10CA600072E00E949F6880916B2780938727809156
:10CA70006C278093882780916D27809389278091E8
:10CA80006E2780938A2710929427109293270E94F2
:10CA90000C6980959095909394278093932710929A
:10CAA0007A27109279270E94FB6880959095909341
:10CAB0007A27809379270E94AB62DF91CF911F91F3
:10CAC0000F910895282F392FF90120E030E080E000
:10CAD000A8E112C0419198E0542F5827B52FB170AA
:10CAE00050FD8A278695B13009F48068915011F085
:10CAF0004695F2CF2F5F3F4F2617370759F7089516
:10CB00001F920F920FB60F920BB60F9211242F9314
:10CB10003F934F935F936F937F938F939F93AF93C5
:10CB2000BF93EF93FF938091940090919500909321
:10CB300053278093522781E080934427809171008E
:10CB4000807D809371000E949A61809144278823A0
:10CB5000E9F18091940090919500209152273091B5
:10CB6000532782179307A0F48091182790911927D3
:10CB7000A0911A27B0911B278C57914EAF4FBF4FF2
:10CB80008093182790931927A0931A27B0931B27F7
:10CB90008091940090919500821B930BA0E0B0E0EF
:10CBA000209118273091192740911A2750911B275F
:10CBB000820F931FA41FB51F8093182790931927E6
:10CBC000A0931A27B0931B2710924427FF91EF914F
:10CBD000BF91AF919F918F917F916F915F914F9195
:10CBE0003F912F910F900BBE0F900FBE0F901F9093
:10CBF00018959FB7F894E1E7F0E08081807D80830D
:10CC000088B38F6288BB10929000E1E9F0E0108257
:10CC1000109292001092950010929400808185608D
:10CC200080839FBF08952FB7F894909399008093C5
:10CC3000980088B38F6288BBE1E7F0E08081826072
:10CC400080832FBF0895EF92FF92CF93DF93FC0173
:10CC5000DB0185E0EB0119928A95E9F7858190E087
:10CC600083709070009711F082E08C93878190E040
:10CC700083709070009721F082E012968C93129747
:10CC8000858190E083709070009799F0878190E0A3
:10CC900083709070009769F023893489818592852B
:10CCA0002817390731F481E0848312961C92129779
:10CCB00001C01482858183708250823030F4C82F85
:10CCC000D0E0C654D94F888101C080E011968C9382
:10CCD0001197E781E370E250E23028F4F0E0E65487
:10CCE000F94F808101C080E013968C931397DF91F8
:10CCF000CF91FF90EF900895DF93CF9300D000D0B5
:10CD00000F92CDB7DEB7BE016F5F7F4F0E942366E3
:10CD100089819A81890F8D5F9B81890F9C81890F01
:10CD20009D81890F0F900F900F900F900F90CF91D2
:10CD3000DF910895AF92BF92CF92DF92EF92FF9270
:10CD40000F931F93DF93CF9300D000D000D0CDB7C7
:10CD5000DEB78C017B01BE016F5F7F4F4E830E9467
:10CD60002366C9809A81A92EBB24DB808C81682F21
:10CD700070E095012C0D311D2D5F3F4F2D0D311DA4
:10CD8000260F371F5D81250F311D4E8150E0421760
:10CD900053070CF4A8C0D80111964C91119750E09C
:10CDA00041705070E3E0440F551FEA95E1F7129689
:10CDB0002C91129730E02170307054E0220F331F15
:10CDC0005A95E1F7242B3C913770232B13963C9115
:10CDD0001397E32FF0E0E170F07045E0EE0FFF1FD6
:10CDE0004A95E1F72E2B14963C911497E32FF0E02F
:10CDF000E170F07036E0EE0FFF1F3A95E1F72E2B51
:10CE0000F701208315964C91159750E043705070B0
:10CE1000440F551F440F551F16962C91169730E05E
:10CE20002370307054E0220F331F5A95E1F7242B02
:10CE300017963C9117973295330F330F307C322B76
:10CE4000318318962C9118972283FC2DF23069F4C7
:10CE500019962C91D70113962C931397F8012285DC
:10CE600014962C93149745E001C043E0E92FF0E0BD
:10CE70003B96E00FF11F542F0AC09701250F311D7B
:10CE8000C290D901CC925F5F0894A108B108A114A7
:10CE9000B10499F7940FBD2DB23089F4F701E90F71
:10CEA000F11DD80153962C91539720839F5FF70172
:10CEB000E90FF11D54962C91549720839F5FE82F22
:10CEC000F0E07596E00FF11F292F08C0D701A20FDF
:10CED000B11D32913C932F5F615070406115710517
:10CEE000A9F7890F01C080E026960FB6F894DEBF3F
:10CEF0000FBECDBFCF91DF911F910F91FF90EF90AB
:10CF0000DF90CF90BF90AF900895BF92CF92DF9205
:10CF1000EF92FF920F931F93CF93DF937C01D62E56
:10CF2000EA01633008F4ADC0FC018081B82EB294F0
:10CF3000B694B694B3E0BB22F1E0BF22F701918131
:10CF4000292F269526952370C92EC294C694C6947F
:10CF5000A3E0CA22382F37703883382F369536959C
:10CF6000369531703983382F329531703A838295F6
:10CF7000869581708B83BC822D83892F82958370E7
:10CF80008E83CF828281888787010D5F1F4F222386
:10CF900061F1F801918180E0F7013381830F911DE8
:10CFA0009A87898787010B5F1F4F223081F4CA015E
:10CFB0000B966CE475E00E948F3EF80181818B87AF
:10CFC000F70185818C878701095F1F4F16C02330C9
:10CFD000A1F4F7013D96DA011B9682918D93E0173B
:10CFE000F107D9F7085F1F4F08C0CA010B966CE420
:10CFF00075E00E948F3E1A861986CC2089F1BB20ED
:10D0000059F4F801918180E02081820F911D9C8B61
:10D010008B8B0E5F1F4F04C089859A859C8B8B8BF1
:10D02000FC2DF23071F4CE0145966CE475E00E945F
:10D030008F3EF80181818D8B80818E8B0E5F1F4F1B
:10D0400017C0FC2DF330A1F4085F1F4FD801FE017B
:10D05000759680E09E9191938F5F8830D9F708C0D4
:10D06000CE0145966CE475E00E948F3E1C8A1B8AB7
:10D07000802F8E199D2D981B9FA71EA70DA7D81630
:10D0800008F480E0DF91CF911F910F91FF90EF9016
:10D09000DF90CF90BF9008959C0141505040460FC3
:10D0A000571FDB0110C0FC91E0E011968C911197A5
:10D0B000BF01680F711D260F371F2617370710F4A1
:10D0C0002F5F3F4F1296A417B50768F3A417B50753
:10D0D00049F49C9180E0280F391F2817390710F474
:10D0E0002F5F3F4FC9010895CF93DF93909172272F
:10D0F000C92FD0E064973091712720E0C20FD31F71
:10D100009E01280F311DC9016BE777E248E050E02E
:10D110000E944C6863E877E2AE010E944C68009779
:10D1200019F0382F292F02C02FEF3FEFC901DF91EF
:10D13000CF91089590937117809370170895FC0113
:10D140004381460F40936E27872F99272281280F0E
:10D1500020936D27A181A0936C27508150936B275A
:10D1600030E02817390748F48A2F8F5F80936C27A7
:10D17000882319F45F5F50936B27842F90E07070C1
:10D180008617970798F480916D278F5F80936D279E
:10D19000882361F480916C278F5F80936C278823AC
:10D1A00029F480916B278F5F80936B270895BC01D2
:10D1B0008091742C9091752C08960E949F68E09144
:10D1C000742CF091752C80916B27808780916C274F
:10D1D000818780916D27828780916E27838708954C
:10D1E0009C01AB0180E090E0B9010E944C68382FAF
:10D1F000292FC901089580E090E06FE677E244E1CD
:10D2000050E00E944C68009719F0382F292F02C077
:10D210002FEF3FEFC901089586E00E9474680895DA
:10D2200081E10E947468089580E009C0E82FF0E071
:10D23000EE0FFF1FEA50F34D118210828F5F843092
:10D24000A8F380E00BC0E82FF0E095E0EE0FFF1FA1
:10D250009A95E1F7EA58F34D118E8F5F843098F379
:10D2600080E094E0909373178093721740E08DE014
:10D2700090E00EC0242F30E0289FF001299FF00D90
:10D28000389FF00D1124E45FF24D158214824F5F38
:10D290004A3080F340936E170895209172173091B1
:10D2A00073172F5F3F4F4DE72030340710F020E019
:10D2B00030E1522F432FA0E013C0EA2FF0E0B5E099
:10D2C000EE0FFF1FBA95E1F7EA58F34DB18DBB237E
:10D2D00031F00480F581E02DE417F50711F3AF5F1D
:10D2E000A43059F7309373172093721710926E176A
:10D2F00020E0E0E0F0E01EC0A22FB0E035E0AA0F91
:10D30000BB1F3A95E1F7AA58B34D59963C915997EE
:10D31000332321F420936E17FD0110C0373049F4F8
:10D32000309731F05A964C915A97328D341708F451
:10D33000FD012F5F243000F320936E173097A9F181
:10D3400022E0218F20916817248720916917258773
:10D3500020916A17268720916B17278728ED34E0E4
:10D36000338B228B358B248B21E030E0318B208B6B
:10D37000138E21E0228F23E0208F168A20E1278B55
:10D380002091721730917317322723273227358364
:10D39000248377836683DC012D913D914D915C91CF
:10D3A00013972083318342835383CF0108950F93D2
:10D3B0001F93CF93DF9320917217309173174DE035
:10D3C00050E02F5F3F4FADE720303A0710F020E0EC
:10D3D00030E1B22FA32F10E012C0C12FD0E0C49FC4
:10D3E000F001C59FF00DD49FF00D1124E45FF24DC4
:10D3F0000480F581E02DEA17FB0719F31F5F1A304F
:10D4000061F7309373172093721710E02DE030E02E
:10D410001AC0012F0F5FC12FD0E0C29FF001C39F40
:10D42000F00DD29FF00D1124E45FF24DDF01149650
:10D43000448155814115510529F410936E17309799
:10D4400049F433C0102F1A3020F310936E17E0E028
:10D45000F0E02BC0209172173091731732272327E9
:10D46000322711963C932E9377836683009729F495
:10D47000108211821282138209C0DC012D913D912C
:10D480004D915C9120833183428353838DE090E002
:10D49000C89FD001C99FB00DD89FB00D1124A45FC3
:10D4A000B24D80E418968C931897CF01DF91CF91FD
:10D4B0001F910F91089540E013C0E42FF0E0542F26
:10D4C0005F5FEE0FFF1FEA50F34D20813181281777
:10D4D000390729F440936E17118210820895452F61
:10D4E000443058F340936E17089540E013C0E42F82
:10D4F000F0E0542F5F5FEE0FFF1FEA50F34D2081E5
:10D5000031812115310529F440936E179183808371
:10D510000895452F443058F340936E170895EF92C5
:10D52000FF920F931F93CF93DF93C091742CD091F0
:10D53000752C843009F4F7C107E917E21093732CB6
:10D540000093722C10936A2700936927833071F43B
:10D55000898D90E08F7090708330910509F074C0D0
:10D5600088899989009709F02FC78DC0823009F00A
:10D570008EC080916B178F5F80936B17882399F40F
:10D5800080916A178F5F80936A17882361F4809176
:10D5900069178F5F80936917882329F48091681732
:10D5A0008F5F8093681710926827109267271092F8
:10D5B0000B2D10920A2D898D873011F0853041F4A2
:10D5C0008A8D8F5F8A8F843109F0FEC6198EFCC662
:10D5D000882309F4F9C6288939892115310509F408
:10D5E0004EC09A8D292F21502A8F992309F0ECC61D
:10D5F0009B8D983031F0282F2150223048F49530FF
:10D6000039F4198E80E880936F2C0E949B6495C535
:10D61000953048F423E030E0092E02C0220F331F7A
:10D620000A94E2F701C020E32A8F9F5F9B8F90E06E
:10D630008F70907083309105E1F0843091054CF447
:10D640008130910509F461C38230910509F0BCC6AF
:10D650000DC08630910509F40CC58830910509F498
:10D6600008C58430910509F0AFC603C51092902714
:10D670004FC384E080936F2C0E949B6490C58F7091
:10D68000833009F0A1C688E080936F2C4BC58530AC
:10D6900019F5E091702CF091712C8481958100979F
:10D6A00009F492C61092752C1092742C0C501040F4
:10D6B0001093732C0093722C10936A2700936927A0
:10D6C00010920B2D10920A2D109268271092672746
:10D6D00088E080936F2C25C10852104080916F27FD
:10D6E000853409F071C69091712780E020917227EE
:10D6F0007C01E20EF11C80916727909168278E15BE
:10D700009F0508F461C6F0926827E0926727809130
:10D71000752790E08F739070009709F055C680913F
:10D720007627882309F050C68091062D9091072D09
:10D73000C091C006D091C1068C179D0759F4409145
:10D74000082D5091092D2091C2063091C306421731
:10D750005307A1F020917F273091802728173907A0
:10D7600009F032C620918127309182278091082DBF
:10D770009091092D2817390709F026C60E94FB68E9
:10D780002FEF8F3F920709F01FC6809178278630D0
:10D7900009F431C18131E9F1813009F015C6809178
:10D7A0008327883009F010C610928327809185273F
:10D7B000909186274FEF873F940710F0099601C09C
:10D7C0000896909386278093852780917B27909158
:10D7D0007C27A0917D27B0917E2780937F2790930F
:10D7E0008027A0938127B09382278091062D909166
:10D7F000072DA091082DB091092D80937B27909340
:10D800007C27A0937D27B0937E2780E4F801808752
:10D81000B8C5C7014C9790936827809367278BE81A
:10D8200097E29093732C8093722C8091892790912A
:10D830008A27009739F00E941069FFEF8F3F9F07FA
:10D8400009F0C2C520918527309186272115310521
:10D8500009F4BAC58CE09DE29093712C8093702CF2
:10D860006091C2067091C3064091BC065091BD06FE
:10D870000091BE061091BF0639C084819581009742
:10D8800081F12817390769F586819781009739F06A
:10D89000A0918327B0918427A817B90711F580813B
:10D8A00091818C179D0729F4A281B381A617B70730
:10D8B00039F18417950729F4A281B381A017B10724
:10D8C000F9F0A0917B27B0917C27A817B90749F4FC
:10D8D000A0917D27B0917E2782819381A817B907F7
:10D8E00079F03D96F093712CE093702CE091702CC0
:10D8F000F091712C8DE2EE38F80708F4BECF64C5C4
:10D900001092752C1092742C82E080936F2C8BE80F
:10D9100097E290936A278093692710920B2D1092BB
:10D920000A2D0E949B6480910A2D90910B2D0097E7
:10D9300009F44AC59C01245E3F4F30936827209329
:10D9400067273093712720937227E091702CF09114
:10D95000712C20852093772721E120937827089642
:10D960009827892798279093882780938727109254
:10D970008A271092892784819581909384278093A8
:10D98000832786819781909386278093852780912E
:10D99000062D9091072DA091082DB091092D80930F
:10D9A0007B2790937C27A0937D27B0937E2780814F
:10D9B0009181A281B38180937F2790938027A09348
:10D9C0008127B093822787E997E29093732C809305
:10D9D000722C0E9410698095909590938A2780936D
:10D9E0008927009709F0CDC48FEF9FEF90938A2786
:10D9F00080938927C6C40E940C69EFEF8F3F9E0772
:10DA000009F0E2C48091852790918627009709F458
:10DA1000DBC420918327309184272115310509F437
:10DA2000D3C4C6E7DCE2498D4423E9F06C817D81F3
:10DA300086179707C1F46E817F812617370799F4FF
:10DA4000E0917B27F0917C2768817981E617F707C1
:10DA500051F4E0917D27F0917E276A817B81E61762
:10DA6000F70709F46DC1A096FCE2C63FDF07D9F6BF
:10DA7000209190272F732230B9F490936D178093E3
:10DA80006C1740E00DC0E42FF0E0EE0FFF1FEA50EE
:10DA9000F34D208131814F5F8217930709F46EC0E7
:10DAA000443088F340936E178091902782FD8CC498
:10DAB00084E1F80181A388E290E090936827809345
:10DAC000672780E580A380918A2790918E27938F86
:10DAD0003091892790918D27928F368F20918827BA
:10DAE00090918C27918F258F9091872790936E1717
:10DAF00040918B27408F948F8F5F878F882361F4AD
:10DB0000832F8F5F868F882339F4822F8F5F858FD5
:10DB1000882311F49F5F948F8091832790918427AD
:10DB200090936D1780936C172091852730918627ED
:10DB3000F801358B248B978B868B80917B27909176
:10DB40007C27A0917D27B0917E2780937F2790939B
:10DB50008027A0938127B09382278091062D9091F2
:10DB6000072DA091082DB091092D80937B279093CC
:10DB70007C27A0937D27B0937E27E8C310926E1771
:10DB800080E0C0E0D0E022C0E82FF0E075E0EE0FCA
:10DB9000FF1F7A95E1F7EA58F34D918D992321F40F
:10DBA00080936E17EF0116C0973079F4209721F01B
:10DBB000228D9A8D921748F4C82FD0E065E0CC0FE3
:10DBC000DD1F6A95E1F7CA58D34D8F5F8430E0F2CC
:10DBD00080936E17209709F4F7C3D093752CC093E8
:10DBE000742C83E08A8F888F1E8A84E08F8B1B8E33
:10DBF00080918527909186279D838C8380918327B0
:10DC0000909184279F838E8380917B2790917C279E
:10DC1000A0917D27B0917E2788839983AA83BB83B7
:10DC200081E0898F809168178C87809169178D8733
:10DC300080916A178E8780916B178F8781E090E0C3
:10DC4000998B888B80918A278B87809189278A87F7
:10DC500080918827898780918727888781E090E055
:10DC60000E94D76880918F27282F30E0207F307066
:10DC7000213531050CF449C082958F7090E00597ED
:10DC8000880F991F880F991F50916F1740E034C07B
:10DC9000F901E159F84D50A5552329F440936E1729
:10DCA00010926F1732C0513011F44F5F25C05230BF
:10DCB000E1F461A56430C9F440936E1750936F1777
:10DCC00032A520E083A590E0822B932B90936D17D3
:10DCD00080936C17F4E0893D9F0710F088ED94E085
:10DCE0009B8B8A8B9D8B8C8B10C02159384DF901F1
:10DCF00021A5222331F0420F242F30E028173907C5
:10DD00003CF240936E1750936F1780E180939027F9
:10DD10008091902782608093902782E0809397275C
:10DD200084E0809398278093992788ED80939A27A1
:10DD30008CE290E0909368278093672780E6B3C2D7
:10DD4000D093752CC093742C10926F2C80919027D7
:10DD500090E082FF03C0198E80E24EC220918F278F
:10DD600022952F70220F220F20936E17B701621B8E
:10DD700071099B0124513040309368272093672715
:10DD800050E04F7050704230510539F4AC014F7380
:10DD900050704231510551F42AC04130510531F4DF
:10DDA000AC014F7350704230510509F12115310516
:10DDB00031F49C012370307021153105C1F0309190
:10DDC00087272885321709F064C230918827298572
:10DDD000321709F05EC2309189272A85321709F07F
:10DDE00058C230918A272B85321709F052C284FF1E
:10DDF0004AC0688979896115710509F444C0CE016A
:10DE00000C960E949F6830918B2780916B27381762
:10DE1000D1F520918C2780916C272817A1F590913E
:10DE20008D2780916D27981771F580918E274091ED
:10DE30006E27841741F53C872D879E878F878B8DB2
:10DE40008823D1F42E89888D9A8D891B922F9695DF
:10DE500096959695891B280F2E8B87FD81959F8916
:10DE6000392F36953695931B980F9F8B822F869569
:10DE700086958695890F888F81E080936F2C888D99
:10DE80008A8F198A188A298D30E0C9018F709070A5
:10DE90008430910509F4B5C18530910564F4823070
:10DEA0009105C9F1833091050CF0B9C0813091051D
:10DEB00009F08AC211C08630910509F4E2C18630AA
:10DEC00091050CF4BEC18730910509F4E2C1883098
:10DED000910509F079C28AC180916F2C80FF14C02E
:10DEE00083E0898F80E480936F2C198A188A80914F
:10DEF000672790916827009709F410C122E42093C6
:10DF00006F2C0E94D7680AC1809190278F7382304E
:10DF100009F05AC2FACE80916F2C80FF75C08091B3
:10DF200090278F73823109F06FC080918F27282F3F
:10DF300030E0207F3070213531050CF449C08295E6
:10DF40008F7090E00597880F991F880F991F509147
:10DF50006F1740E034C0F901E159F84D50A5552341
:10DF600029F440936E1710926F1732C0513011F49C
:10DF70004F5F25C05230E1F461A56430C9F440938D
:10DF80006E1750936F1732A520E083A590E0822B87
:10DF9000932B90936D1780936C1774E0893D9707CE
:10DFA00010F088ED94E09B8B8A8B9D8B8C8B10C03E
:10DFB0002159384DF90121A5222331F0420F242F98
:10DFC00030E0281739073CF240936E1750936F17D3
:10DFD00083E0898F80918727888780918827898728
:10DFE000809189278A8780918A278B8781E090E0BA
:10DFF0000E94D76882E480936F2C198A188A109245
:10E000006827109267278AC080E280936F2C0E9455
:10E010009B64E091742CF091752C118E45CD80910C
:10E02000902780FF2AC024FD28C0888999890097FD
:10E0300009F0CAC1809167279091682701960E94D4
:10E04000D76820916F2C822F806180936F2C8091F4
:10E05000672790916827009719F0226120936F2C11
:10E060000E949B6481E090E0998B888B88E0898F87
:10E070001B8E81E1809390270FC185FF1CC05091BA
:10E08000952740E08091962790E0842B952B409136
:10E09000722C5091732C480F591F5093732C40933E
:10E0A000722C4091672750916827481B590B509359
:10E0B000682740936727809167279091682700978A
:10E0C00049F024FD07C020916F2C226020936F2C13
:10E0D0000E94D7689091912780E020919227820F2B
:10E0E000911D90936D1780936C172C893D8928178B
:10E0F000390710F0009721F430936D1720936C17B7
:10E1000080916C1790916D179B8B8A8B80916F2CEF
:10E1100090E083709070009709F456C110920B2D17
:10E1200010920A2D0E949B6480916F2C85FF07C07E
:10E1300010920B2D10920A2D198E84E19BCF84FF33
:10E140000AC010920B2D10920A2D81E090E0998B5D
:10E15000888B84E08CCF20910A2D30910B2D2115D6
:10E160003105E1F080FF02C0198A188A88899989EF
:10E17000009781F48A899B898217930720F49093F2
:10E180000B2D80930A2D80910A2D90910B2D998B48
:10E19000888B04C090930B2D80930A2D1B8E809149
:10E1A000692790916A279093732C8093722C8091A9
:10E1B0000A2D90910B2D009759F088899989009725
:10E1C00039F08896909368278093672788E10BC081
:10E1D00080916F2C81FFF8C088E290E090936827CF
:10E1E0008093672780E1809390275CC080916F2C9B
:10E1F00080FFEAC0198E80E180936F2C0E949B649F
:10E20000E3C08091672790916827009711F00E94E2
:10E21000D7689091902780916F2C90FF0BC080FF62
:10E2200006C087E0898F1A8E198A188A19C086E07D
:10E23000898F16C080FF1EC085E0898F198A188AD1
:10E24000C3C08091672790916827009711F00E94C2
:10E25000D7688091902780FF0DC087E0898F1A8E44
:10E2600081E090E00E94D76880E180936F2C0E944B
:10E270009B640FC08091672790916827009749F4AD
:10E28000A3C080916F2C80FF9FC087E0898F1A8E7A
:10E290009BC080E1F80181A388E290E09093682719
:10E2A0008093672780E580938F27888580938B27CD
:10E2B000898580938C278A8580938D278B85809391
:10E2C0008E278C85809387278D85809388278E85E0
:10E2D000809389278F8580938A2786E0809378278B
:10E2E0008C819D8190938427809383278E819F8149
:10E2F00090938627809385278091062D9091072DF6
:10E30000A091082DB091092D80937B2790937C27B5
:10E31000A0937D27B0937E2788819981AA81BB81B4
:10E3200080937F2790938027A0938127B0938227A3
:10E33000898D84FF05C0109292271092912706C004
:10E3400084E08093912788ED8093922780E48093E6
:10E350007727809167279091682790937127809302
:10E360007227109296271092952710929427109258
:10E3700093270E940C6980959095909394278093A1
:10E38000932785E480936F27109270271092762749
:10E390001092752780917017909171170196909344
:10E3A000711780937017909373278093742710923E
:10E3B0007A27109279270E94FB6880959095909318
:10E3C0007A278093792704C01092682710926727D4
:10E3D00010926F2CDF91CF911F910F91FF90EF90D2
:10E3E0000895382F292FC9010895382F292F40E08B
:10E3F00050E076276727762780E090E0CB017727EB
:10E400006627262B372B482B592BB901CA010895B3
:10E41000AC01E0916927F0916A27222733272E1B50
:10E420003F0B2159334D621773070CF49B011216F1
:10E43000130664F420930A2D30930B2D4E175F07BB
:10E4400029F0CF01BA01A9010E94727D08950F93AE
:10E45000DF93CF93CDB7DEB760970FB6F894DEBFEA
:10E460000FBECDBF002309F459C029833A834B83E3
:10E470005C836D837E838F839887E0E2E01B298134
:10E480003A814B815C811E16BCF019861A861B8668
:10E490001C868E2F992787FD9095909581959F4F8B
:10E4A00004C0220F331F441F551F8A95D2F72D87B2
:10E4B0003E874F87588B2AC0CA01B901002E04C07D
:10E4C000660F771F881F991F0A94D2F769877A878A
:10E4D0008B879C87DA01C90104C0B695A7959795EB
:10E4E0008795EA95D2F72D813E814F81588504C0EA
:10E4F000220F331F441F551F0A95D2F7822B932BEF
:10E50000A42BB52B8D879E87AF87B88B29853A853D
:10E510004B855C856D857E858F85988960960FB665
:10E52000F894DEBF0FBECDBFCF91DF910F9108955C
:10E53000A0E1B0E0EEE9F2E70C94C57A29833A83D2
:10E540004B835C836D837E838F839887A986BA868D
:10E55000CB86DC86ED86FE860F87188B2D813E816B
:10E560004F8158858D859E85AF85B88928173907D5
:10E570004A075B07C8F082179307A407B50790F016
:10E5800029813A814B815C8189859A85AB85BC85DF
:10E59000281739074A075B0738F082179307A40743
:10E5A000B50720F482E003C080E001C081E06096FE
:10E5B000EAE00C94E17A2F923F924F925F926F9231
:10E5C0007F928F929F92AF92BF92CF92DF92EF9203
:10E5D000FF920F931F93DF93CF93CDB7DEB763976F
:10E5E0000FB6F894DEBF0FBECDBF6C017F876E877C
:10E5F000FC0117821682838181FD04C06FC34C85A4
:10E600005D8504C01E010894211C311CF601938114
:10E61000EE85FF8593FD859193FF8191FF87EE87BE
:10E62000882309F457C3853241F493FD859193FF04
:10E630008191FF87EE87853259F490E0B6014A8BCD
:10E640005B8B0E94C57D4A895B895D874C87D7CFEC
:10E6500010E0FF2400E00032B0F48B3269F08C321D
:10E6600028F4803251F0833271F40BC08D3239F0CE
:10E67000803349F401602CC00260046029C0086046
:10E6800027C0006125C007FD2EC0282F20532A3047
:10E6900098F406FF08C0812F880F182F110F110F53
:10E6A000180F120F15C08F2D880FF82EFF0CFF0CBE
:10E6B000F80EF20E00620CC08E3221F406FD0AC381
:10E6C000006406C08C3611F4006802C0883659F424
:10E6D000EE85FF8593FD859193FF8191FF87EE87FE
:10E6E000882309F0B8CF982F9554933018F400611F
:10E6F000805E06C0982F9556933008F09BC10F7E20
:10E7000006FF16E06FE3E62EE022853619F4F0E40A
:10E71000EF2A07C0863619F420E8E22A02C0111158
:10E720001150E7FE06C01C3340F4912E939427E06D
:10E730000BC0183030F4212F06C027E03CE3932EA5
:10E7400003C027E017E09924CA0104969D878C87AF
:10E75000FA016081718182819381A101092D0E945A
:10E76000827C5C016980262D30E0398B288B60FE2D
:10E7700003C0388933FF06C0E1FC06C0E2FE06C0D4
:10E7800000E205C00DE203C00BE201C000E0888991
:10E7900099898C7090700097C1F1002311F084E08A
:10E7A00001C083E08F1558F4F81AE3FC09C080E239
:10E7B00090E0B6010E94C57DFA94C9F701C0FF241C
:10E7C000002329F0802F90E0B6010E94C57D888942
:10E7D00083FD03C001EA1FE00EC00DE91FE00BC07E
:10E7E000A114B10409F0805290E0B6010E94C57DE9
:10E7F0000F5F1F4F05C0AE2CBB2490E1A922BB24A4
:10E80000F8018491882361F762C2E7FE0EC09A0C7A
:10E81000F889F4FF04C08A81813309F49A941914A9
:10E8200054F5292D293050F52DC0E6FC2BC0812F41
:10E8300090E08A159B054CF03CEFA3163FEFB30622
:10E8400024F080E8E82A01C01150112349F0E2E0E9
:10E85000F0E0EC0FFD1FE10FF11D80818033A1F38B
:10E86000E7FE10C0912E9394812F90E0A816B90670
:10E8700044F41A1907C09924939404C098E0992E7F
:10E8800001C010E0E7FE07C01A141B043CF4950118
:10E890002F5F3F4F05C025E030E002C021E030E0AF
:10E8A000002311F02F5F3F4F112329F0812F90E0BB
:10E8B0000196280F391F8F2D90E02817390714F47F
:10E8C000F21A01C0FF244E2C5524C20189709070A9
:10E8D000009749F406C080E290E0B6010E94C57D31
:10E8E000FA94FF20C1F7002329F0802F90E0B601B1
:10E8F0000E94C57D43FC09C006C080E390E0B601DC
:10E900000E94C57DFA94FF20C1F7E7FE46C035019D
:10E91000B7FE02C06624772425010894411C511CCF
:10E9200046185708420C531CF501E919F1094F012B
:10E93000812F90E000271127081B190BFFEF6F169E
:10E94000FFEF7F0629F48EE290E0B6010E94C57DBC
:10E95000A614B70434F0861497041CF4F2018081E5
:10E9600001C080E30894610871080894411C511C9F
:10E97000601671062CF090E0B6010E94C57DDECFD6
:10E980006A147B0441F49A81963320F4953319F488
:10E99000F889F4FF81E390E049C08A81813311F066
:10E9A0002FEE622290E0B6010E94C57D112389F00E
:10E9B0008EE290E0B6010E94C57D02E0F101E00F19
:10E9C000F11D0F5F808190E0B6010E94C57D11505E
:10E9D000A9F744FE03C085E490E002C085E690E01C
:10E9E000B6010E94C57DB7FC05C0A114B10441F475
:10E9F00064FE06C0B094A194B108B3948DE201C046
:10EA00008BE290E0B6010E94C57D80E305C08F5F78
:10EA1000E6EFFFEFAE0EBF1EFAE0AF16B104BCF793
:10EA200090E0B6010E94C57DC501C096B6010E9466
:10EA3000C57D4DC1833631F0833789F0833509F0C8
:10EA400059C022C09A012E5F3F4F3D872C87FA01A3
:10EA500080818983310181E0A82EB12C13C09A01F5
:10EA60002E5F3F4F3D872C87FA016080718006FF43
:10EA700003C0612F70E002C06FEF7FEFC3010E94FF
:10EA80008B7D5C010F7714C09A012E5F3F4F3D874D
:10EA90002C87FA016080718006FF03C0612F70E04F
:10EAA00002C06FEF7FEFC3010E94627D5C010068CE
:10EAB00003FD1CC006C080E290E0B6010E94C57D47
:10EAC000FA948F2D90E0A816B906A8F30FC0F301B1
:10EAD00007FD859107FF81913F0190E0B6010E94FB
:10EAE000C57DF110FA940894A108B108A114B104ED
:10EAF00071F7EDC0843611F0893661F507FF0BC060
:10EB00009A012C5F3F4F3D872C87FA01608171810C
:10EB1000828193810CC09A012E5F3F4F3D872C87E5
:10EB2000FA0160817181882777FD8095982F0F7693
:10EB300097FF08C090958095709561957F4F8F4F96
:10EB40009F4F0068A1012AE030E00E94D07E982EFD
:10EB5000921841C0853721F40F7E2AE030E020C0B2
:10EB6000097F8F36A9F0803720F4883509F0B2C0CC
:10EB70000BC0803721F0883709F0ACC001C00061BC
:10EB800004FF09C0046007C004FF08C0066006C097
:10EB900028E030E005C020E130E002C020E132E0B2
:10EBA00007FF0AC0CA0104969D878C87FA0160811D
:10EBB00071818281938109C0CA0102969D878C87E9
:10EBC000FA016081718180E090E0A1010E94D07E15
:10EBD000982E92180F7706FF09C00E7F911630F419
:10EBE00004FF06C002FD04C00F7E02C0E92C01C074
:10EBF000E12E802F90E004FF0CC0FE01E90DF11D15
:10EC00002081203311F4097E09C0E39402FF06C07D
:10EC100004C086789070009709F0E394A02EBB247E
:10EC200003FD14C000FF0FC0EF1428F4192D1F0DB1
:10EC30001E19EF2C08C0192D06C080E290E0B60125
:10EC40000E94C57DE394EF14C0F304C0EF1410F4E8
:10EC5000FE1801C0FF24A4FE0FC080E390E0B601BF
:10EC60000E94C57DA2FE1FC0A1FE03C088E590E002
:10EC700010C088E790E00DC0C501867890700097BD
:10EC800091F0A1FC02C080E201C08BE207FD8DE2A1
:10EC900090E0B6010E94C57D06C080E390E0B60119
:10ECA0000E94C57D11509116C0F39A94F101E90DAF
:10ECB000F11D808190E0B6010E94C57D9920A9F7E1
:10ECC00006C080E290E0B6010E94C57DFA94FF2064
:10ECD000C1F795CCF6012681378102C02FEF3FEFB7
:10ECE000C90163960FB6F894DEBF0FBECDBFCF91BA
:10ECF000DF911F910F91FF90EF90DF90CF90BF9029
:10ED0000AF909F908F907F906F905F904F903F90CB
:10ED10002F9008955058BB27AA270ED0CBC1BCD145
:10ED200030F0C1D120F031F49F3F11F41EF48CC1BA
:10ED30000EF4E095E7FB82C1E92FCDD180F3BA173D
:10ED4000620773078407950718F071F49EF5E5C113
:10ED50000EF4E0950B2EBA2FA02D0B01B9019001F6
:10ED60000C01CA01A0011124FF27591B99F0593F3A
:10ED700050F4503E68F11A16F040A22F232F342F82
:10ED80004427585FF3CF469537952795A795F040D0
:10ED90005395C9F77EF41F16BA0B620B730B840BE5
:10EDA000BAF09150A1F0FF0FBB1F661F771F881F9D
:10EDB000C2F70EC0BA0F621F731F841F48F48795F5
:10EDC00077956795B795F7959E3F08F0B3CF9395E4
:10EDD000880F08F09927EE0F9795879508955CD1D5
:10EDE00058F080E891E009F49EEF5DD128F040E80A
:10EDF00051E059F45EEF09C027C18FC1E92FE078D7
:10EE00006AD168F3092E052AC1F326173707480788
:10EE1000590738F00E2E07F8E02569F0E025E06488
:10EE20000AC0EF6307F8009407FADB01B9019D01FE
:10EE3000DC01CA01AD01EF9347D03CD10AD05F910C
:10EE4000552331F02BED3FE049E450FD49EC63CF11
:10EE50000895DF93DD27B92FBF7740E85FE31616EB
:10EE6000170648075B0710F4D92F5ED19F938F9345
:10EE70007F936F930FD2E0E2F1E0E9D01BD12F91A5
:10EE80003F914F915F9163D1DD2349F09058A2EA01
:10EE90002AED3FE049EC5FE3D0785D274DDFDF915D
:10EEA00009C1A8D008F481E008950CD003C1FBD0BB
:10EEB00040F0F2D030F021F45F3F19F0BFC05111A3
:10EEC0002DC1C2C008D198F39923C9F35523B1F3DA
:10EED000951B550BBB27AA2762177307840738F0C9
:10EEE0009F5F5F4F220F331F441FAA1FA9F333D028
:10EEF0000E2E3AF0E0E830D091505040E695001CDC
:10EF0000CAF729D0FE2F27D0660F771F881FBB1F97
:10EF1000261737074807AB07B0E809F0BB0B802D71
:10EF2000BF01FF2793585F4F2AF09E3F510568F0BD
:10EF300085C0F4C05F3FECF3983EDCF3869577958F
:10EF40006795B795F7959F5FC9F7880F911D9695BF
:10EF5000879597F90895E1E0660F771F881FBB1F1B
:10EF6000621773078407BA0720F0621B730B840BC8
:10EF7000BA0BEE1F88F7E0950895E89409C097FB57
:10EF80003EF490958095709561957F4F8F4F9F4F80
:10EF90009923A9F0F92F96E9BB279395F6958795C4
:10EFA00077956795B795F111F8CFFAF4BB0F11F487
:10EFB00060FF1BC06F5F7F4F8F4F9F4F16C088232E
:10EFC00011F096E911C0772321F09EE8872F762F64
:10EFD00005C0662371F096E8862F70E060E02AF0A5
:10EFE0009A95660F771F881FDAF7880F9695879591
:10EFF00097F90895990F0008550FAA0BE0E8FEEF66
:10F0000016161706E807F907C0F012161306E407EC
:10F01000F50798F0621B730B840B950B39F40A26E5
:10F0200061F0232B242B252B21F408950A2609F4C3
:10F03000A140A6958FEF811D811D089597F99F67C7
:10F0400080E870E060E008959FEF80EC0895DF9322
:10F05000CF931F930F93FF92EF92DF927B018C016E
:10F06000689405C0DA2EEF0172D0FE01E894A591F4
:10F070002591359145915591AEF3EF015DDEFE018D
:10F080009701A801DA9479F7DF90EF90FF900F9144
:10F090001F91CF91DF91089500240A941616170648
:10F0A00018060906089500240A9412161306140679
:10F0B00005060895092E0394000C11F4882352F0DC
:10F0C000BB0F40F4BF2B11F460FF04C06F5F7F4F94
:10F0D0008F4F9F4F089557FD9058440F551F59F07B
:10F0E0005F3F71F04795880F97FB991F61F09F3F35
:10F0F00079F087950895121613061406551FF2CF5E
:10F100004695F1DF08C0161617061806991FF1CFAD
:10F1100086957105610508940895E894BB276627D4
:10F120007727CB0197F908959B01AC0160E070E06F
:10F1300080E89FE3BACE0BD0BDCFAEDF28F0B3DFBF
:10F1400018F0952309F07ACF7FCF1124E7CFC3DFE2
:10F15000A0F3959FD1F3950F50E0551F629FF001EA
:10F16000729FBB27F00DB11D639FAA27F00DB11D43
:10F17000AA1F649F6627B00DA11D661F829F2227CC
:10F18000B00DA11D621F739FB00DA11D621F839F53
:10F19000A00D611D221F749F3327A00D611D231F29
:10F1A000849F600D211D822F762F6A2F11249F5777
:10F1B00050408AF0E1F088234AF0EE0FFF1FBB1F9A
:10F1C000661F771F881F91505040A9F79E3F510539
:10F1D00070F034CFA3CF5F3FECF3983EDCF386951D
:10F1E00077956795B795F795E7959F5FC1F7FE2BE4
:10F1F000880F911D9695879597F90895FA01EE0F5E
:10F20000FF1F30962105310599F16115710561F4F3
:10F210008038BFE39B0749F168949038810561F01D
:10F220008038BFEF9B0741F0992342F5FF3FE1058E
:10F230003105210511F1E8940894E795D901AA2335
:10F2400029F4AB2FBE2FF85FD0F310C0FF5F70F42E
:10F25000A695E0F7F73950F019F0FF3A38F49F77A8
:10F260009F930CD00F9007FC905808953EF0ECCE81
:10F2700060E070E080E89FE308954FE79F775F9339
:10F280004F933F932F9375D02F913F914F915F9163
:10F2900052DF08C09B01AC014ECF19F40EF0CECE68
:10F2A0003CCFD2CE20DFC8F39638C0F707F80F92D4
:10F2B000E8942BE33AEA48EB5FE74BDF0F920F92BB
:10F2C0000F924DB75EB70F9294D0EDE4F1E0BFDE40
:10F2D0004F915F91EF91FF91E595EE1FFF1F49F070
:10F2E000FE57E0684427EE0F441FFA95E1F7419579
:10F2F000550B06D00F9007FE17CF08959FCEACC0D8
:10F30000F2DEE8F39923D9F3940F511DBBF391502A
:10F31000504094F059F0882332F0660F771F881F11
:10F3200091505040C1F79E3F510544F7880F911D01
:10F330009695879597F908955F3FACF0983E9CF0BD
:10F34000BB27869577956795B79508F4B160939537
:10F35000C1F7BB0F58F711F460FFE8CF6F5F7F4F25
:10F360008F4F9F4FE3CFDACE0EF076C06DCE68940C
:10F3700065CEB9DEC8F39923D1F3C6F3DF93CF93FB
:10F380001F930F93FF92C92FDD2788232AF021971F
:10F39000660F771F881FDAF720E030E040E85FEB68
:10F3A0009FE3883920F0803E30F021968F77B3DCE0
:10F3B000E5E7F1E003C0AFDCE2EAF1E048DE8B0113
:10F3C000BE01EC01FB2E6F5771097595771F880BF5
:10F3D000990BD5DD28E132E741E35FE3B8DEAF2DDD
:10F3E0009801AE01FF900F911F91CF91DF91A4DCA6
:10F3F00061CEFA01DC01AA0FBB1F9B01AC01BF5714
:10F4000028F422273327442750781FC0B75188F4A7
:10F41000AB2F0024469537952795011CA395D2F371
:10F42000002069F0220F331F441FB395DAF30DD08B
:10F4300071CC61307105A0E88A07B94630F49B01B0
:10F44000AC016627772788279078309621F02083B3
:10F4500031834283538308959F3F31F0915020F4CC
:10F46000879577956795B795880F911D96958795A0
:10F4700097F90895629FD001739FF001829FE00D7C
:10F48000F11D649FE00DF11D929FF00D839FF00D23
:10F49000749FF00D659FF00D9927729FB00DE11DCF
:10F4A000F91F639FB00DE11DF91FBD01CF011124AC
:10F4B0000895AA1BBB1B51E107C0AA1FBB1FA617BB
:10F4C000B70710F0A61BB70B881F991F5A95A9F70D
:10F4D00080959095BC01CD01089597FB092E0726D4
:10F4E0000AD077FD04D0E5DF06D000201AF470952D
:10F4F00061957F4F0895F6F7909581959F4F0895F8
:10F50000A1E21A2EAA1BBB1BFD010DC0AA1FBB1F27
:10F51000EE1FFF1FA217B307E407F50720F0A21B99
:10F52000B30BE40BF50B661F771F881F991F1A9406
:10F5300069F760957095809590959B01AC01BD0130
:10F54000CF01089597FB092E05260ED057FD04D054
:10F55000D7DF0AD0001C38F450954095309521959E
:10F560003F4F4F4F5F4F0895F6F7909580957095F8
:10F5700061957F4F8F4F9F4F08952F923F924F92EB
:10F580005F926F927F928F929F92AF92BF92CF9233
:10F59000DF92EF92FF920F931F93CF93DF93CDB73C
:10F5A000DEB7CA1BDB0B0FB6F894DEBF0FBECDBFB4
:10F5B00009942A88398848885F846E847D848C8485
:10F5C0009B84AA84B984C884DF80EE80FD800C818E
:10F5D0001B81AA81B981CE0FD11D0FB6F894DEBF71
:10F5E0000FBECDBFED010895AF92BF92CF92DF92D3
:10F5F000EF92FF920F931F93CF93DF93EC016881FB
:10F6000079818A819B81611571058105910521F4BC
:10F6100064E279ED8BE597E02DE133EF41E050E0D6
:10F620000E94A27A79018A0127EA31E440E050E0A1
:10F630000E943A7A5B016C01C801B7012CEE34EFED
:10F640004FEF5FEF0E943A7A6A0D7B1D8C1D9D1D66
:10F6500097FF04C061507040804090486883798370
:10F660008A839B837F77CB01DF91CF911F910F918D
:10F67000FF90EF90DF90CF90BF90AF9008950E94E1
:10F68000F47A089584EC96E00E94F47A0895A0E05C
:10F69000B0E08093C4069093C506A093C606B093CD
:10F6A000C70608952F923F924F925F926F927F927A
:10F6B0009F92AF92BF92CF92DF92EF92FF920F9301
:10F6C0001F93CF93DF933B01EA016115710519F098
:10F6D000FB0180839183209739F09E0122503040B6
:10F6E0002332310508F0D5C0C82ED92EF60111916C
:10F6F0006F017F01812F90E00E945A7D0097B1F742
:10F700001D3231F4F60111917F019924939406C0C2
:10F710001B3219F4F60111917F019924209719F0F9
:10F72000C031D105D1F4103389F4F70180818837D5
:10F7300011F0883559F4F701118182E090E0E80E6C
:10F74000F91E92E0992AC0E1D0E007C0209729F481
:10F750001033B1F0CAE0D0E02BC0CA30D10541F17E
:10F76000C031D10521F0C830D105A9F409C02FEF6F
:10F77000A22E2FEFB22E2FEFC22E2FE0D22E20C0BE
:10F78000C8E0D0E09FEFA92E9FEFB92E9FEFC92EC2
:10F790009FE1D92E15C09E01442737FD4095542F77
:10F7A0006FEF7FEFCB010E94807A59016A0108C098
:10F7B00089E9A82E89E9B82E89E9C82E89E1D82ED1
:10F7C00060E020E030E0A9011E01442437FC4094B1
:10F7D000542C012F00530A3060F0812F81548A315C
:10F7E00010F4075006C0812F81568A3150F5012F41
:10F7F0000755802F90E08C179D071CF56F3FE9F0AF
:10F80000A216B306C406D506A8F0CA01B901A20122
:10F8100091010E943A7A9B01AC01802F90E0A0E018
:10F82000B0E0280F391F4A1F5B1F281739074A0706
:10F830005B0710F46FEF01C061E0F70111917F01E8
:10F84000C8CF6114710481F0662339F00894E1088F
:10F85000F108F301F182E08207C091FE05C0C70103
:10F860000297F3019183808390FE07C050954095E5
:10F87000309521953F4F4F4F5F4F67FF0DC082E29C
:10F8800090E09093952D8093942D2FEF3FEFA90159
:10F8900003C020E030E0A901B901CA01DF91CF9196
:10F8A0001F910F91FF90EF90DF90CF90BF90AF909E
:10F8B0009F907F906F905F904F903F902F90089512
:10F8C000662777270C94697FFC0188279927E8949D
:10F8D00021912032E9F3293010F02E30C8F32B3279
:10F8E00041F02D3239F4689404C00E94BD7D820F2E
:10F8F000911D219120532A30C0F31EF490958195DB
:10F900009F4F0895283008F027E03327DA01990F38
:10F91000311D87FD916000966105710539F43260F3
:10F920002E5F3D9330E32A95E1F708959F3F30F035
:10F9300080387105610509F03C5F3C5F3D93913073
:10F9400008F08068911DDF93CF931F930F93FF9270
:10F95000EF92192F987F9695E92F96959695E90F36
:10F96000FF27E150F04F99273327EE24FF24A7010A
:10F97000E70105900894079428F4360FE71EF81E57
:10F98000491F511D660F771F881F991F0694A1F705
:10F990000590079428F4E70EF81E491F561FC11D55
:10F9A000770F881F991F661F0694A1F7059007948B
:10F9B00028F4F80E491F561FC71FD11D880F991F25
:10F9C000661F771F0694A1F70590079420F4490F4E
:10F9D000561FC71FD81F990F661F771F881F0694D1
:10F9E000A9F784911095177041F0D695C795579552
:10F9F0004795F794E7941A95C1F7E5EAFFE0689414
:10FA00001590159135916591959105907FE27395CB
:10FA1000E118F10A430B560BC90BD009C0F7E10CF2
:10FA2000F11E431F561FC91FD01D7EF4703311F401
:10FA30008A95E6CFE894015030F0080F0AF40027C9
:10FA4000021708F4202F2395022F7A3328F079E348
:10FA50007D932A95E9F710C07D932A9589F606943F
:10FA600097956795379517951794E118F10A430B09
:10FA7000560BC90BD00998F023957E9173957A3374
:10FA800008F070E37C932013B8F77E9170617D934A
:10FA900030F0839571E37D9370E32A95E1F71124AB
:10FAA000EF90FF900F911F91CF91DF91992787FDE4
:10FAB0009095089591119BC3803219F0895085501B
:10FAC000D0F70895FC010590615070400110D8F7FF
:10FAD000809590958E0F9F1F089544E757E10E94EF
:10FAE000967D0895FB01DC0102C001900D9241500A
:10FAF0005040D8F70895DC0101C06D93415050404B
:10FB0000E0F70895FB01DC018D910190801901104F
:10FB1000D9F3990B0895FC016150704001900110D8
:10FB2000D8F7809590958E0F9F1F0895FA01A191A7
:10FB3000B081009719F41097E1F0CD01DC01CD01FF
:10FB40000D90002011F4C00113C0FB01219122236C
:10FB500019F02015D9F7F3CFFB012191201519F4E5
:10FB60001E92119606C02223C1F70D900020A1F726
:10FB7000D001FA01A193B08308957AE0979F902D68
:10FB8000879F802D910D112408950F931F93CF937C
:10FB9000DF938C01EB018B8181FF1BC082FF0DC0C5
:10FBA0002E813F818C819D812817390764F4E8817B
:10FBB000F9810193F983E88306C0E885F985802FF0
:10FBC0000995009731F48E819F8101969F838E83E2
:10FBD00002C00FEF1FEFC801DF91CF911F910F916E
:10FBE0000895DF93CF93CDB7DEB7FE0135966191CF
:10FBF00071918091902D9091912DAF010E94DB72B7
:10FC0000CF91DF910895DF93CF93CDB7DEB7FE019B
:10FC10003596619171918091902D9091912DDC019B
:10FC200013962C911397286013962C93AF010E9482
:10FC3000DB72E091902DF091912D2381277F23831A
:10FC4000CF91DF910895EF92FF920F931F93CF937F
:10FC5000DF938C01E091902DF091912D838181FFB4
:10FC60001FC0C0E0D0E00AC0DB011896ED91FC9106
:10FC700019970995009711F0CFEFDFEFF801819107
:10FC80008F016091902D7091912D882369F7DB0190
:10FC90001896ED91FC9119978AE00995009711F05B
:10FCA000CFEFDFEFCE01DF91CF911F910F91FF904A
:10FCB000EF9008950F931F93DF93CF93CDB7DEB7E7
:10FCC0002E970FB6F894DEBF0FBECDBF0D891E89EB
:10FCD0008F89988D26E02C831A83098397FF02C0B1
:10FCE00080E090E801979E838D839E01255E3F4FC3
:10FCF000CE010196698D7A8DA9010E94DB724D813A
:10FD00005E8157FD0AC02F813885421753070CF4D6
:10FD10009A01020F131FF80110822E960FB6F89465
:10FD2000DEBF0FBECDBFCF91DF911F910F91089520
:10FD30000F931F93DF93CF93CDB7DEB72E970FB6F8
:10FD4000F894DEBF0FBECDBF8C01CB01BA0146E0F7
:10FD50004C831A83098397FF02C080E090E80197E3
:10FD60009E838D83CE010196A9010E94DB724D8195
:10FD70005E8157FD0AC02F813885421753070CF466
:10FD80009A01020F131FF80110822E960FB6F894F5
:10FD9000DEBF0FBECDBFCF91DF911F910F910895B0
:10FDA000FA01AA27283051F1203181F1E8946F93AC
:10FDB0006E7F6E5F7F4F8F4F9F4FAF4FB1E03ED052
:10FDC000B4E03CD0670F781F891F9A1FA11D680FF0
:10FDD000791F8A1F911DA11D6A0F711D811D911D23
:10FDE000A11D20D009F468943F912AE0269F112498
:10FDF0003019305D3193DEF6CF010895462F4770FC
:10FE0000405D4193B3E00FD0C9F7F6CF462F4F7056
:10FE1000405D4A3318F0495D31FD4052419302D0B4
:10FE2000A9F7EACFB4E0A69597958795779567955A
:10FE3000BA95C9F700976105710508959B01AC015A
:10FE40000A2E06945795479537952795BA95C9F781
:10FE5000620F731F841F951FA01D0895DC01CB0145
:10FE6000FC01F999FECF06C0F2BDE1BDF89A3196CA
:10FE700000B40D9241505040B8F70895F999FECF63
:10FE800092BD81BDF89A992780B50895A8E1B0E0A8
:10FE900042E050E00C94307FDC01CB0103C02D9197
:10FEA0000E94577F41505040D0F70895262FF9996E
:10FEB000FECF1FBA92BD81BD20BD0FB6F894FA9A4D
:10FEC000F99A0FBE019608950E94567F272F0C9431
:10FED000577F6F927F928F929F92AF92BF92CF92F5
:10FEE000DF92EF92FF920F931F93DF93CF930F92C6
:10FEF000CDB7DEB75B016115710521F0DB018C9395
:10FF000011969C93482F592F6A01F601E1906F01D9
:10FF10008F018E2D90E00E945A7D0097B1F7FE2D43
:10FF2000FD3229F4D601ED908D0121E007C0BE2DF0
:10FF3000BB3219F4F601E1908F0120E068010894CA
:10FF4000C108D108C6016FE970E143E050E02983A0
:10FF50000E94FA802981009711F572E0E72EF12CBA
:10FF6000E00EF11EC70162EA70E145E050E00E9438
:10FF7000FA802981009729F467E0E62EF12CE00E43
:10FF8000F11EA114B10421F0D5011196FC92EE925C
:10FF900020FF0FC130E020E090E88FEF12C1C601D2
:10FFA00067EA70E143E050E029830E94FA802981EA
:10FFB000009731F060E070E0CB01662477240AC03E
:10FFC000A114B10409F4F9C00E5F1F4FF5011183AC
:10FFD0000083F3C03E2D30533A30A0F52260E22F6B
:10FFE000F0E0AF014870507022FF07C04115510585
:10FFF00071F50894611C711C2AC04115510519F056
:020000021000EC
:100000000894610871086B017C0152E0CC0CDD1C86
:10001000EE1CFF1C5A95D1F76C0D7D1D8E1D9F1D8A
:10002000660F771F881F991F630F711D811D911D1A
:100030006839F9E97F07F9E98F07F9E19F0738F097
:10004000246005C03E3F39F423FD3FC02860D8013D
:10005000ED908D01BFCF353311F03531B1F5F80199
:1000600031913D3211F4206102C03B3241F4D8019C
:1000700011963C911197319642E050E002C041E068
:1000800050E030533A3020F08F01041B150B1DC097
:1000900040E050E0BCE040385B075CF4DA01AA0FB6
:1000A000BB1FAA0FBB1F4A0F5B1F440F551F430FF7
:1000B000511D319130538F013A3060F324FF03C05A
:1000C000509541955F4F640E751EC22EDD2421FFB1
:1000D00008C0A114B10429F001501040F5011183AA
:1000E00000830E94BD777B018C01F3E0CF22DD24E9
:1000F00033E0C316D10421F417FB109517F91095BE
:10010000C801B70120E030E0A9010E94517788239F
:1001100009F44AC077FE09C04EEBC42E40E1D42E4C
:10012000709461947108739404C036EDC32E30E16D
:10013000D32E26E0822E912C90E2A92EB12C0FC056
:10014000F6012591359145915491C801B7010E945E
:100150009B78E62EF72E082F192F6A187B086A1451
:100160007B0474F7B594A7940894810891088114CE
:10017000910429F08CEF9FEFC80ED91EF0CFB70184
:10018000C801282F220F292F221F2F3F39F020E0EE
:1001900030E0A9010E945177882331F482E290E097
:1001A0009093952D8093942D3E2D2F2D902F812F60
:1001B00008C030E020E090E803C030E020E090ECA0
:1001C0008FE7F901AC016F2F722F852F942F0F90BD
:1001D000CF91DF911F910F91FF90EF90DF90CF9023
:1001E000BF90AF909F908F907F906F9008959927C8
:1001F00088270895FB01DC014150504088F08D9123
:1002000081341CF08B350CF4805E659161341CF0F8
:100210006B350CF4605E861B611171F3990B0895C8
:08022000881BFCCFF894FFCF0E
:1002280054696D656F757420414444523D252D64B1
:100238002E252D64205345513D252D6420525353BE
:10024800493D252D75204C51493D252D750A00261F
:100258003A202573205B414444523D252D642E25C8
:100268002D64205345513D252D6420525353493D5B
:10027800252D75204C51493D252D75204452503D62
:10028800252D642E253032645D0A00523D252D75DA
:10029800204C3D252D7520533D252D6420002845F3
:1002A800787450777229000065756936343D0025E9
:1002B80030327800253032780A00736E3D00413ABA
:1002C800202564202564202564200A00433A20253F
:1002D8006420256420256420613D25352E31660A79
:1002E800007374617475733D3078253032780A2054
:1002F800006669726D776172653D53322D342E3414
:100308002D323031342D30312D3036006565707224
:100318006F6D006F6E006F66660061310072657305
:100328006574006E6F6E6500613200765F696E00FD
:100338007374617473003100320033003400350087
:100348003600636820706B74730025327520252D84
:100358003130750A006175746F00666C75736800DA
:10036800414444523D252D642E252D64205345518A
:100378003D252D6420525353493D252D75204C5160
:10038800493D252D750A006465657000666F7263C6
:10039800655F69646C65007472696D007465737477
:1003A8000043683D252D642054785077723D252DF3
:1003B800640A004572726F72205458204C656E674B
:1003C80074683D25640A0049443D004536343D00C3
:1003D8002050533D25640020543D252D362E32668D
:1003E800002054313D252D362E32660020545F4DB5
:1003F80043553D252D352E31660020565F4D43551A
:100408003D252D342E3266002050303D252D6C5868
:10041800002050305F543D252D372E336600205084
:10042800313D252D6C58002050315F543D252D3726
:100438002E3366002055503D252D6C58002052481B
:100448003D252D342E31660020565F494E3D252D21
:10045800352E32660020565F41313D252D352E322E
:10046800660020565F41323D252D352E326600202C
:10047800565F41333D252D352E30660020503D25F1
:100488002D6C64002050413D252D372E3266002604
:100498003A2025730A00545820706B74206C656EDE
:1004A800203D2025640A000100D734EF3C22FFCC10
:1004B8003B22FFCC3B1A20090D009604616263645D
:1004C80065666768696A6B6C6D6E6F70269400006C
:1004D8003C000A001A636D642070726F6365737361
:1004E800000000B504A43500000000737464696E50
:1004F8002070726F63657373000000CB04D70F0020
:1005080000000062726F6164636173742070726FBF
:1005180063657373000000E3048436000000005331
:100528006C6565702070726F63657373000000FFFF
:1005380004C91000000000506572696F6469632087
:1005480070726F636573730000001705E21700008F
:100558000000C104D904F50428050D05000024098C
:1005680000001D004000FE063E0710000000BE3ED1
:10057800B23E1810000000004576656E742074695C
:100588006D65720000005805C94200000000437400
:10059800696D65722070726F636573730000006E19
:1005A80005074400000000020306070A0B0E0F02AD
:1005B8000306070A0B0E0F28432920323031322058
:1005C8004865726A756C660055747665636B6C690C
:1005D8006E6720202020202000436F6E74696B69AD
:1005E80020322E35000000000200000000425200B8
:1005F800000000C600C500C400C100C20000000021
:10060800CE00CD00CC00C900CA000000005246321E
:10061800333020647269766572000000ED05F95682
:10062800000000006A55E854485792580B569B54EE
:10063800095303538A54EC530001010101010101DC
:1006480001010101010101010052696D65002906DE
:100658000D5AD45961646174612E6E756D2077618D
:1006680079206F75742074686572653A2025640A6C
:10067800004F5B4E5B585D875EBF5C0080C0E0F05A
:10068800F8FCFEFF6E756C6C6D61630064063A5F82
:100698001F5F255F2B5F315F375F736963736C6F13
:1006A800776D6163007A065B60BC5F525F3B5F41B8
:1006B8005F4F5FBA000800FD10051135000200D534
:1006C80016D7165443502F495020737461636B003A
:1006D8000000A306B562000000000208FFFFFFFF4C
:0806E800000000000100000009
:00000001FF
